:020000040800F2
:1000000000000220991A0B081D1B0B08F19006082E
:100010001D1B0B081D1B0B081D1B0B0800000000FF
:100020000000000000000000000000001D1B0B0885
:100030001D1B0B08000000001D1B0B08B54E05081A
:100040001D1B0B081D1B0B081D1B0B081D1B0B0884
:100050001D1B0B081D1B0B08C12D0508C52D050810
:10006000C92D0508CD2D0508D12D0508A943040883
:10007000B9430408C9430408D9430408ED430408FC
:1000800001440408154404081D1B0B081D1B0B0824
:100090001D1B0B081D1B0B081D1B0B08D52D050870
:1000A0001D1B0B081D1B0B081D1B0B08054F04080F
:1000B000194F04082D4F0408414F0408D93504088E
:1000C000CD35040809360408FD3504081D1B0B084E
:1000D0001D1B0B0865590408715904087D59040853
:1000E000D92D05081D1B0B08000000007D4F0408DA
:1000F000CD4F0408F54F0408694F0408294404084B
:100100001D1B0B08AD6A0408554F04081D1B0B0886
:10011000895904081D1B0B081D1B0B08B19F0408FF
:100120003D44040851440408654404087944040823
:100130008D4404081D1B0B081D1B0B081D1B0B0801
:1001400000000000000000000000000000000000AF
:10015000A1440408B5440408C94404089559040896
:10016000393604082D3604081D1B0B081D1B0B080F
:100170001D1B0B081D1B0B081D1B0B08000000009E
:100180001D1B0B081D1B0B08A1590408AD590408C1
:100190001D1B0B081D1B0B081D1B0B081D1B0B0833
:1001A0001D1B0B081D1B0B081D1B0B081D1B0B0823
:1001B0001D1B0B081D1B0B081D1B0B081D1B0B0813
:1001C0001D1B0B081D1B0B081D1B0B081D1B0B0803
:1001D0001D1B0B08C98D04081D1B0B081D1B0B08DC
:1001E0001D1B0B081D1B0B081D1B0B081D1B0B08E3
:1001F0001D1B0B081D1B0B081D1B0B081D1B0B08D3
:100200001D1B0B081D1B0B081D1B0B081D1B0B08C2
:10021000914F0408A54F0408B94F04081D1B0B0893
:100220001D1B0B081D1B0B081D1B0B0800000000ED
:10023000B16A04081D1B0B08000000001D1B0B0801
:100240001D1B0B081D1B0B081D1B0B081D1B0B0882
:100250001D1B0B081D1B0B081D1B0B081D1B0B0872
:100260001D1B0B081D1B0B081D1B0B081D1B0B0862
:100270001D1B0B081D1B0B081D1B0B08000000009D
:100280001D1B0B08000000001D1B0B0800000000D8
:08029000000000001D1B0B081B
:1002980081C90181008408B10000000080C9018182
:1002A800008408B10000000080C90181B0AB08B12A
:1002B80000000000C9010181B0B0AC80000000005E
:1002C800C9060181B0B0AF85000000003F1A018166
:1002D800B0AF81C90000000008B10181B0B000844E
:1002E8000000000008B10181B0B0008400000000E7
:1002F8005C3D0B0000840280C43D0B00010000003F
:10030800E03E0B00008402804C3F0B00010000001F
:100318004C3F0B007CFFFF7F00400B0080FFFF7FFE
:1003280040400B0084FFFF7F28410B00B0B0AE8037
:10033800CC420B00B0A8018014440B0078FFFF7F6B
:10034800344A0B00B0AA0580904C0B000100000055
:10035800904C0B006CFFFF7FFC570B000100000066
:10036800905A0B0068FFFF7FFC600B000100000043
:1003780084610B00B0A8018094610B0001000000AB
:10038800C4610B00B00D8480D4610B000100000033
:10039800F8610B0044FFFF7F04620B0048FFFF7FFA
:1003A80010620B00AF08B18048650B000100000027
:1003B80054650B00A908B18000670B00010000001C
:1003C800F49C0B00A908B1801C9D0B0001000000E3
:1003D800E89D0B00B0A902807C9E0B00B0B0A880FD
:1003E800CC9E0B0001000000D49E0B00B0B0AA8088
:1003F800089F0B00AE71B280CC9F0B00AB3F3880DA
:100408002CA00B000100000034A00B00B0B0AA80A3
:1004180070A00B000100000010A10B00AA0DB28013
:100428008CA10B00B0AF08802CA40B0001000000C9
:100438003CA40B00AD3F0280B8A60B0001000000F1
:10044800E8A60B00B0AD04808CA90B0001000000E9
:10045800A85A01240201000002001400C85A01240D
:100468000202000002001400E85A0124020A0000F7
:1004780002001400085B01240203000004001400B9
:10048800285B01240208000004001400485B0124D2
:10049800010B000000017700685B0124010C0000DB
:1004A80000017600885B012401100000000176003D
:1004B800A85B0124010D010000017700C85B01243D
:1004C8000112000000017600E85B0124011400001D
:1004D80000001E00085C0124011A000000000D0045
:1004E800285C01240115000000000C00485C012470
:1004F8000116000000000C00685C0124011B0000CC
:1005080000000E00885C0124011C000000001E0091
:10051800A85C01240117000000000C00C85C01243D
:100528000118000000000E00E85C01240119000019
:1005380000000C00085D0124011E000000000C00F2
:10054800285D0124011F000000000C00485D012403
:100558000128010000011800685D01240120000045
:1005680000014800885D01240121000000014900C4
:10057800A85D01240122000000014A00C85D012491
:100588000123000000014B00E85D01240124000064
:1005980000014C00085E01240125000000014D0007
:1005A800285E01240126000000014E00485E012457
:1005B8000127000000014F00685E0124012B0000A4
:1005C80000002900885E0124012C01000000290098
:1005D800A85E0124012D010000007000C85E0124FE
:1005E800012E010000005200E85E0124012F0100E5
:1005F80000012800085F01240130010000012800E3
:10060800285F01240133000000003C00485F0124FA
:08061800013600000000200083
:020000040804EE
:10000000836B5A6D12F0500F5A6D1AD1196842F471
:1000100000725A650A6812F0080FCA6816D012F406
:10002000406F15D1CA68920412D45A6D22F48072BE
:100030005A655A6DD1040BD45A6D42F001025A65CB
:100040007047D20604D4DB6CDB6C18479007ECD009
:10005000704700BF704700BF836B5A6D42F040028B
:100060005A659A6D42F004029A657047026838B585
:10007000524B9A4248D018339A4245D03033504CB4
:100080005049A24218BF9A4204F148040CBF012310
:1000900000238A4208BF43F001033031A24208BF67
:1000A00043F0010330348A4208BF43F0010301F5F5
:1000B0005C71A24208BF43F0010304F55C748A42FC
:1000C00008BF43F001033031A24208BF43F00103EF
:1000D00030348A4208BF43F001033031A24208BFE6
:1000E00043F0010330348A4208BF43F0010330314A
:1000F000A24208BF43F001038A4208BF43F0010354
:1001000013B9314B9A4208D1042380F83530136873
:1001100023F001031360002038BD2C4B2C4D1168D7
:10012000AA4218BF9A422B4C21F00E0105F13C0562
:100130000CBF012300231160A24208BF43F001035A
:1001400011682834AA4208BF43F0010321F00101DD
:10015000A24208BF43F0010314341160A24208BF59
:1001600043F001031C498A4208BF43F0010313B95D
:100170001A4B9A4217D10123856DD0E917142268D2
:1001800001F01F0122F480728B4022606B60C36E0D
:10019000D0E91921516033B11A68D0E91C1422F456
:1001A00080721A604C6000210122036D80F83410C7
:1001B00080F83520002BAED09847ACE71000024005
:1001C0004000024070000240B80402401C54025833
:1001D000085402583054025880540258945402581B
:1001E000002280F8422090F84130292B04D090F86A
:1001F00041302A2B18D070474FF0280C212301687A
:1002000080F841C0036390F8413003EA0C03634572
:100210000B680CBF6FF0420C6FF0F20C03EA0C039A
:100220000B6080F84020704710B422232824016816
:1002300080F84140036390F841302340A3420C68AA
:100240000CBF6FF044036FF0F40323405DF8044BE0
:100250000B6080F8402070470023202210B4174C18
:100260004363C462036380F8412080F842304B0747
:1002700012D50268436A526A1A70436A028D0133CA
:1002800043624AB1438D013A013B02859BB24385EB
:10029000436C43F0040343640368102490F8412046
:1002A000002190F841201A6822F0FE021A60DC61F9
:1002B0005DF8044B80F84010704700BF0000FFFF5E
:1002C00010B54FF0000C90F84130444A044680F8D5
:1002D00042C0283BC262A0F82AC0022B426C41EA0D
:1002E000020141643CD890F841204FF0280C90F86E
:1002F000413002F0280203F02803282A0CBF4622CE
:10030000F622282B03684FF000000CBFD1436FF09A
:10031000F6011A680A401A60314A84F841C06263E3
:1003200020631A6812F4804231D01A68A06B22F45C
:1003300080421A6098B100222A4B036584F840205D
:1003400090F83520022A3CD080224265BDE810405A
:10035000184794F84130602B3AD084F8401010BD13
:10036000036890F8412090F841201A6822F0FE02BC
:100370001A6090F84120602A02D0202280F84120A3
:100380000022226362631A6812F48042CDD1196898
:1003900011F40041DDD01968E06B21F400411960CF
:1003A0000028DCD00F4B036584F8402090F83520FE
:1003B000022AC9D1FFF75AFE0028D0D0E06B036DA6
:1003C000C4E7FFF753FE0028C9D0A06B036DBDE75B
:1003D000202384F8401084F8413010BD0000FFFF56
:1003E00065040408F106040803689A69196810B4E2
:1003F000D4052ED50C061FD5416C4FF4807441F006
:10040000010141645105DC6128D5416C4FF48064E1
:10041000920541F008014164DC6106D5426C4FF45D
:10042000007142F002024264D961416C11F00B0F7D
:100430000CD15DF8044B70475405F6D49405F4D5FF
:100440000906EBD4416C11F00B0FF2D05DF8044BB0
:1004500036E75405F2D50906D7D4E6E79205DDD490
:10046000E3E700BF2DE9F84390F84030C66A012B5E
:1004700000F0D980012304460D46914680F84030B3
:10048000880602D512F0200F62D1EF0621D519F0AF
:10049000100F1ED0638D9BB2002B40F0AA8094F801
:1004A0004130B6F1007FDBB202D1282B00F017817A
:1004B00094F841301022292B2368DA6103D116F514
:1004C000803F40F0D2800023184684F84030BDE8D9
:1004D000F88369071DD42A0703D519F0080F40F0E7
:1004E0009880AB07EFD519F0020FECD0638D9BB26B
:1004F000002B00F0A380616A236811F8010B228DA4
:100500009862638D013A6162013B22859BB26385EB
:10051000D9E719F0040FDED0638D9BB26BB122686E
:10052000636A526A1A70638D616A228D013B0131E0
:10053000013A9BB2616222856385638D9BB2002B79
:10054000C1D116F5803FBED02046FFF749FEBAE77D
:1005500023682021644A1F68D96194F8411094F8F7
:100560004110186820F0FE001860586840F4004000
:1005700058605968114059609969890701D500216F
:1005800099629969CA0703D4996941F00101996197
:1005900078044BD5A16B19B10868416889B26185AF
:1005A0006A0749D5596A25F00408636A1970636AB5
:1005B00001336362238D002B50D1638D9BB21BB13D
:1005C000636C43F0040363640023236384F84230C4
:1005D000676C6363002F56D1E36ADFF810814345EF
:1005E00031D194F84130202384F8407084F84130B0
:1005F0004BE723681022DA61636C43F00403636401
:1006000036F080737FF45FAF616C2046FFF758FED1
:1006100059E794F8413003F02803282B236840D091
:100620000822DA614FE70220BDE8F8833904B7D524
:10063000E16B0029B0D1B3E7A846BEE736F080737E
:100640007FF441AF80E72046FFF7CAFD2023C4F8BE
:100650002C8084F8407084F8413016E7013B2385F4
:10066000638D013B9BB26385A7E79A69950701D526
:1006700000229A629A69D0073FF566AF9A6942F004
:1006800001029A6160E7616C2046FFF719FE94F859
:100690004130282B7FF4F9AE41462046FFF7DCFDC0
:1006A000F3E6E1689A69022998699A68DD6811D1D0
:1006B000C2F3C21282EA104212F006020AD1A16C01
:1006C0000131A164A16C02297FF4FDAE0821A2646E
:1006D000D961F8E61A6822F0B8021A60F3E62946F2
:1006E0002046FFF7B9FDEEE600E800FE0000FFFF40
:1006F000836B0022D3E90E0102650A6593F841205D
:10070000602A02D1202283F841207047026870B429
:10071000D4072DD597490B69896A03F03803102B4C
:1007200000F0F180182B00F0E9804368B3F5803FBA
:1007300000F05581002B00F05B81B3F5A02F8D4BAD
:10074000196800F0328221F480311960196821F4AF
:1007500080211960884B41F2883C864C1D6804E07A
:100760001968491B614500F2408121688E03F7D565
:1007700091072DD57F490B69896A13F0380300F082
:10078000A680182B00F0A080C3687A4C002B00F0E4
:100790006981216821F019011943774B21601D6897
:1007A00004E01968491B022900F21F8121684907EA
:1007B000F7D5724941F203030968B3EB114F63683F
:1007C0000169C0F0238223F47C3343EA0133636080
:1007D000D5064CD4150713D54369664C002B00F0A1
:1007E0009E80616F644B41F0010161671D6804E008
:1007F0001968491B022900F2F880616F8907F7D553
:10080000940613D583695B4C002B00F007812168A7
:10081000594B41F4805121601D6804E01968491B5F
:10082000022900F2E28021688904F7D5540700F11B
:10083000A780436AC3B14F490A6902F03802182AF7
:1008400000F085810A68022B4B4B22F080720A600F
:1008500000F01E81186804E01A68121A022A00F2D9
:10086000C4800A689201F7D4002070BC70474149E7
:100870000B69896A03F03803082B63D0182B5DD00D
:10088000C3693C4C002B00F0D88021683A4B41F002
:10089000800121601D6804E01968491B022900F2EB
:1008A000A4802168C905F7D5344941F203030968DA
:1008B000B3EB114FC0F097816368016A23F0F843EE
:1008C00043EA8163636085E78D077FF45DAF294B61
:1008D0001B685C0701D5C368F3B1284941F20303E3
:1008E00004690968B3EB114F22494B68C0F0B4802A
:1008F00023F47C3343EA04334B6069E701F00301DE
:1009000002297FF412AF1B4B1B689B037FF530AFAE
:100910004368002B7FF42CAF012070BC7047616FDF
:10092000154B21F0010161671D6803E01968491B3F
:1009300002295AD8616F8E07F8D461E701F00301EC
:1009400001299DD10B4B1B68DC0502D5C369802BA7
:10095000E2D10A4941F20303046A0968B3EB114F7B
:100960000449C0F08E804B6823F0F84343EA846367
:100970004B602FE700440258602B00240010005CFD
:100980009D499E4B0A6842F480720A601C6803E02D
:100990001A68121B642A28D80A68D505F8D5826817
:1009A000012A00F03981002A00F00781052A944AC3
:1009B000116F00F0378121F001011167116F21F0F3
:1009C000040111671D6841F288348D4903E01A68FB
:1009D000521BA24209D80A6F9207F8D529E7884925
:1009E0000B6843F480330B60B4E6032070BC70479F
:1009F000834C41F28835814B216821F4803121609C
:100A0000216821F4802121601E6803E01968891B98
:100A1000A942EAD821688903F8D4A9E62168774B6E
:100A200021F4805121601D6803E01968491B0229E7
:100A3000DBD821688E04F8D4F8E621686F4B21F0EA
:100A4000800121601D6803E01968491B0229CCD888
:100A50002168CE05F8D4BDE623F0FE4343EA0463E3
:100A60004B60B5E62168654B21F0010121601D68EE
:100A700003E01968491B0229B7D821684E07F8D44A
:100A8000A6E6CB6823F07C5343EA0463CB60A1E67F
:100A90001C6803E01A68121B022AA6D80A6895018E
:100AA000F8D48C6A574A2240846A2243C46A42EAD4
:100AB00004128A62D0E90D24013A013C5202240456
:100AC00092B204F4FE042243046B013CC4F3080414
:100AD0002243C46B013C240604F0FE4422430A6313
:100AE000CA6A22F00102CA62474A4D6B846C2A40EE
:100AF00042EAC4024A63CA6A046C22F00C0222432E
:100B00003F4CCA62CA6A406C22F002020243CA62C7
:100B1000CA6A42F48032CA62CA6A42F40032CA62C5
:100B2000CA6A42F48022CA62CA6A42F00102CA62F8
:100B30000A6842F080720A60196804E01A68521A62
:100B4000022A3FF652AF22689001F7D58CE6012BBE
:100B50008A6A0C6B3FF4E0AE02F00303816A8B42B9
:100B60007FF4DAAEC2F30512C36A9A427FF4D4AEC0
:100B7000036BC4F30802013B9A427FF4CDAE436B92
:100B8000C4F34622013B9A427FF4C6AE836BC4F3A2
:100B90000642013B9A427FF4BFAEC36BC4F30664C6
:100BA000013B9C423FF460AEB6E641F480211960FF
:100BB000196841F480311960CCE5114941F288355A
:100BC0000A6F22F001020A670A6F22F004020A6724
:100BD0001C6804E01A68121BAA423FF606AF0A6FAF
:100BE0009607F7D425E6E368016A23F07C5343EACD
:100BF0000163E360EEE500BF00480258602B00246B
:100C0000004402580CFCFFFF0700FFFF23F0FE43E7
:100C100043EA01636360DBE506490A6F42F00102C3
:100C20000A67CFE641F004011167116F41F001013D
:100C30001167C7E600440258454B30B49A6A9C6A73
:100C4000DD6A14F47C7F596BC4F3051038D0C1F30E
:100C5000CC0105F0010502F0030205FB01F1012AB8
:100C600007EE901AB8EEE77A02D0022A4ED04AB3C5
:100C700007EE900ADFED376AF8EEE77A1B6B86EE37
:100C8000A76A9FED355AC3F3080306EE903AF7EED4
:100C9000005AF8EEE66AE7EE056A76EEA56A66EEB9
:100CA000266A2B4B1B6BC3F34623013307EE903AA6
:100CB000B8EEE77AC6EE877AFCEEE77A17EE900A8E
:100CC00030BC70471A68920627D5196807EE900A5B
:100CD000224AF7EE005A1B6BC1F3C101F8EEE77A26
:100CE0009FED1D5AC3F30803CA4006EE903A06EE84
:100CF000102AF8EEE66AB8EEC66AE7EE056A86EEF6
:100D0000277A76EEA56A66EE876ACAE707EE900A4A
:100D1000DFED136AF8EEE77AB0E707EE900A9FED91
:100D2000115A1B6BB7EE006AF8EEE77ADFED0A5A4C
:100D3000C3F30803C5EE276A07EE903AF8EEE77AA8
:100D4000E7EE257A77EE867A66EEA76AA9E700BF16
:100D5000004402580024744A000000390090D00377
:100D600020BCBE4B0024744C836ADA0710B406D54D
:100D70000168C46A4A6822F4003222434A609C0730
:100D800006D50168046B4A6822F4803222434A6027
:100D9000590706D50168446B4A6822F48022224331
:100DA0004A601A0706D50168846B4A6822F400423B
:100DB00022434A60DC0606D50168C46B8A6822F4C7
:100DC000805222438A60990606D50168046C8A68BD
:100DD00022F4005222438A605A060AD50168446C04
:100DE0004A68B4F5801F22F4801242EA04024A6085
:100DF0000BD01B0606D50268C16C536823F4002390
:100E00000B4353605DF8044B70474A68846C22F4CE
:100E1000C00222434A60ECE70022836BA3F85E2005
:100E2000A3F85620704700BF134B41F2883C134A89
:100E300001461B68A2FB0332520A0CFB02F2531E4E
:100E400042B14A6B013B12F0450F01D0920404D528
:100E5000581CF6D14FF0004070474B6B5B0707D42E
:100E6000486B10F0010014BF0123054B8B637047E2
:100E7000042318468B63704700000024D34D621092
:100E8000C5002000036942681F2B70B430D9A3F15C
:100E9000200520215468A940214227D08169087C7F
:100EA000022835D048681F2BC9681B4D4E68016960
:100EB000C1F30324194951F8244015F804C005680A
:100EC00056F80C4024F0010446F80C40407901EB40
:100ED0004001098C01F4F050E96821EA0001E96061
:100EE00010D9A3F1200120238B40D36070BC704740
:100EF0002021146899402142F8D08169087C022899
:100F0000D0D105E0202101FA03F370BC9360704753
:100F100000200874C6E700BF9CB20B0838B10B086C
:100F2000436BDA69910670B5044614D5586AE36AD2
:100F3000C0B2002B00F0F080216B9847636B1A68F9
:100F400022F480721A609A6822F001029A609A690B
:100F500042F008029A61DA69D20701D501221A62C9
:100F6000DA69960701D502221A62DA69550701D5B6
:100F700004221A62DA69100701D508221A62DA69B6
:100F8000110613D5D4F8B420212A0FD0D4E90912C0
:100F90008A4200F0CD80A169895C0132C9B29962B0
:100FA0002169B2FBF1F001FB1022A262DA6952065C
:100FB00000D470BDDA6940F60F0C1D6804F13400EE
:100FC00012EA0C0F996826D1960607D505F020067F
:100FD00001F0805C56EA0C0640F0C980D60202D5CA
:100FE0004E0200F1C980160606D501F4000105F095
:100FF0008006314340F0A8805106DAD56A06D8D57C
:101000001A682020002122F040021A60C4F8B400BF
:10101000C4F8A41070BD604E01EA060C5F4E05EAEC
:10102000060E5EEA0C06D9D0D60709D5EE0507D51F
:1010300001261E62D4F8BC6046F00106C4F8BC600C
:10104000960700F18680560709D5CE0707D50426F6
:101050001E62D4F8BC6046F00206C4F8BC601607F5
:101060000CD505F0200656EA0C0607D008261E62AD
:10107000D4F8BC6046F00806C4F8BC6016050AD572
:101080006E0108D54FF400661E62D4F8BC6046F0CD
:101090002006C4F8BC60D4F8BC60002E89D0960647
:1010A0000BD505F0200501F0805155EA010204D06E
:1010B000D4F8A0200AB19047636BD4F8BC109A68AA
:1010C00001F0280102F040020A4362D01968202092
:1010D000334A21F49071196099680A4000219A609E
:1010E000C4F8B8009A68C4F8A01052067FF561AF42
:1010F0009A68D4F8AC0022F040029A6000283FF4CD
:1011000058AF90F83520274B022A036538D080224B
:101110004265BDE870401847E3696269D054E369ED
:10112000E2680133B3FBF2F102FB1133E36105E73F
:101130000022A4F88A201A6822F080021A60DA6974
:1011400052067FF536AF35E7D4F8A430002BE0D156
:101150002FE7CE0783D502261E62D4F8BC6046F086
:101160000406C4F8BC6056077FF579AF6FE7D4F882
:10117000A030002BCDD11CE74FF480121A6270BD55
:10118000FEF774FF00283FF414AFD4F8AC00036DF1
:10119000BFE7C4F8BC2070BD0100001020010004AE
:1011A000FEFFFFEF190E0408D0E907239A4201D38E
:1011B000D01A7047C0681044C01A7047D0E909239C
:1011C0009A4204D30069D31A0138C01A70470069E3
:1011D00002440138D31AC01A704700BFD0E909028F
:1011E000101AB0FA80F04009704700BF016A034648
:1011F00040694A1C405CD9688A4228BF00221A62B2
:10120000704700BF436A826910B4D154436A416B8E
:10121000046901330A68A34228BF00235DF8044B28
:1012200042F0800243620A60704700BF436BD86996
:1012300010F0100002D0102201201A62704700BF87
:101240002DE9F047046982B0C3681C4044D0814650
:1012500088464FF0004501F1500701F13806B4FA15
:1012600084F325FA03F21B3BD2431440C9F8102043
:10127000B8F1000F5DD0042B2CD8DFE803F0504606
:101280003B300300D8F81030D9F82CA033B19B685C
:1012900023B11FFA8AF108F108009847D8F82830DE
:1012A00033B19B6823B11FFA8AF108F120009847F7
:1012B000D8F840302BB19B681BB11FFA8AF1304639
:1012C0009847D8F858302BB19B681BB11FFA8AF1A8
:1012D00038469847002CC2D102B0BDE8F087D8F854
:1012E000103008F10800D9F834105B689847002CDA
:1012F000B5D1F1E7D8F8283008F12000D9F8381036
:101300005B689847002CAAD1E6E7D8F84030304611
:10131000D9F83C105B689847002CA0D1DCE7D8F8DE
:1013200058303846D9F840105B689847002C96D161
:10133000D2E7042B07D8DFE803F00319140F0A00E3
:10134000D9F840300193019B002C88D1C4E7D9F82B
:101350002C300193019BF7E7D9F834300193019BBE
:10136000F2E7D9F838300193019BEDE7D9F83C302A
:101370000193019BE8E700BF70B5124E124A336833
:10138000A2FB03239B09013BB3F1807F0FD24FF0F7
:10139000E0220E4900240F2853614FF0F003054668
:1013A00081F823304FF007039461136101D90120C4
:1013B00070BD01464FF0FF306BF050FE2046756067
:1013C00070BD00BF00000024D34D621000ED00E0AE
:1013D000034A0130116813685B1A8342FBD37047DC
:1013E000602B00240268354B354930B4354D364CFE
:1013F000AA4218BF9A420CBF012300238A4208BFA9
:1014000043F001033031A24208BF43F001033034FE
:101410008A4208BF43F001033031A24208BF43F0C3
:10142000010330348A4208BF43F0010301F55C71C7
:10143000A24208BF43F0010304F55C748A4208BF6E
:1014400043F001033031A24208BF43F001033034BE
:101450008A4208BF43F001033031A24208BF43F083
:10146000010330348A4208BF43F001033031A24205
:1014700008BF43F001038A4208BF43F0010313B9D8
:10148000124B9A4215D1D3B21149124C103BA1FB19
:1014900003515F2B104BC1F3021103EA02032144F5
:1014A00088BF043391F828108365C165184630BCA5
:1014B000704722F0FF038365F8E700BF1000024089
:1014C000400002402800024058000240B804024098
:1014D000ABAAAAAA38B10B0800FCFFFF2DE9F04F18
:1014E0000D6883B0002D00F0D5800023DFF86882FE
:1014F00001229A4012EA050C00F0C7804E6826F0DF
:101500001009B9F1020F40F0C88003F007044FEA58
:10151000D30E4FF00F0A4FEA840900EB8E0E0AFA41
:1015200009FADEF8204024EA0A0A0C6904FA09F4F0
:1015300006F0030944EA0A04CEF820404FEA430EBD
:101540000324D0F800A009FA0EF904FA0EF42AEAEE
:10155000040AE44349EA0A09C0F80090D0F808A058
:10156000CF6804EA0A0A07FA0EF949EA0A09C0F83C
:101570000890C6F30019D0F804A009FA03F92AEA82
:10158000020249EA02024260C268F70004EA020469
:101590008A6802FA0EF242EA0402C26075D5644C0F
:1015A00023F0030E03F00309D4F8F420C6444FEAF5
:1015B000890942F00202C4F8F420D4F8F42002F0C1
:1015C00002020192019A0F22DEF8084002FA09F2A3
:1015D00024EA0202574CA04225D004F58064A042C0
:1015E0007BD0554CA0427ED0544CA0426FD0544C7E
:1015F000A04200F08480534CA04200F08680524C00
:10160000A04276D0514CA04200F08580504CA042C0
:1016100000F087804F4CA0420CBF09240A2404FA32
:1016200009F942EA0902CEF808204FF0B0426FEA09
:101630000C0EF403D2F880204FF0B04454BF0EEAF1
:1016400002024CEA0202C4F88020B203D4F88440BB
:101650004FF0B04254BF0EEA04044CEA0404F7020F
:10166000C2F8844014684FF0B04254BF0EEA04043C
:101670004CEA04041460B40252684FF0B04454BF02
:101680000EEA02024CEA02026260013335FA03F20A
:101690007FF42EAF03B0BDE8F08F4FEA430E032472
:1016A000D0F800B006F0030A04FA0EF409F1FF398D
:1016B0000AFA0EFA2BEA040BB9F1010F6FEA0404DF
:1016C0004AEA0B0AC0F800A03FF65EAF46E70324E3
:1016D00004FA09F942EA0902A5E7012404FA09F922
:1016E00042EA09029FE7022404FA09F942EA0902E0
:1016F00099E7062404FA09F942EA090293E7042467
:1017000004FA09F942EA09028DE7052404FA09F905
:1017100042EA090287E7072404FA09F942EA0902C2
:1017200081E7082404FA09F942EA09027BE700BFCD
:10173000004402580000025800080258000C0258E9
:10174000001002580014025800180258001C0258D9
:101750000020025800240258000400580C4A136963
:1017600003F03803102B04D0182B0DD01BB10948FF
:1017700070470948704713689B0607D513680748E8
:10178000C3F3C103D8407047FFF756BA0348704708
:101790000044025800093D0040787D010090D003CC
:1017A000184A136903F03803102B10B51AD0182B00
:1017B00023D0CBB114481349144A8B69144CC3F39A
:1017C0000323134493F8303003F01F03D840206004
:1017D0008B6903F00F031A4492F8303003F01F03B3
:1017E000D84010BD0B48E6E713689B0608D5136880
:1017F0000948C3F3C103D840DDE7FFF71DFADAE774
:101800000548D8E70044025800093D0038B10B08EC
:101810000000002440787D010090D003584B70B444
:10182000996A9D6ADE6A15F47C3FC5F30532DC6B6C
:101830005CD0C4F3CC04C6F3001601F0030106FB30
:1018400004F4012907EE904AB8EEE77A03D00229A2
:1018500075D000294FD007EE902ADFED4A6AF8EEE6
:10186000E77A9B6B86EEA76A9FED475AC3F308039E
:1018700006EE903AF7EE005AF8EEE66AE7EE056AF1
:1018800076EEA56A66EE266A3D4AB7EE006A936B6D
:10189000C3F3462307EE103AB8EEC77A70BC37EEB2
:1018A000067AC6EE877AFCEEE77AC0ED007A936B93
:1018B000C3F3064307EE103AB8EEC77A37EE067A5E
:1018C000C6EE877AFCEEE77AC0ED017A936BC3F33C
:1018D000066307EE903AF8EEE77A77EE867A86EEC0
:1018E000A77ABCEEC77A80ED027A704770BCC0E977
:1018F0000022826070471968890627D51C6807EEA8
:10190000902A2249F7EE005A9B6BC4F3C102F8EE0D
:10191000E77A9FED1D5AC3F30803D14006EE903AD3
:1019200006EE101AF8EEE66AB8EEC66AE7EE056A49
:1019300086EE277A76EEA56A66EE876AA4E707EE5A
:10194000902ADFED136AF8EEE77A8AE707EE902A2D
:101950009FED105A9B6BB7EE006AF8EEE77ADFED69
:101960000A5AC3F30803C5EE276A07EE903AF8EE69
:10197000E77AE7EE257A77EE867A66EEA76A83E75E
:10198000004402580024744A000000390090D0033B
:1019900020BCBE4B0024744C584B70B4996A9D6AAD
:1019A000DE6A15F07C7FC5F305525C6C5CD0C4F335
:1019B000CC04C6F3002601F0030106FB04F4012960
:1019C00007EE904AB8EEE77A03D0022975D00029D5
:1019D0004FD007EE902ADFED4A6AF8EEE77A1B6CEB
:1019E00086EEA76A9FED475AC3F3080306EE903AC6
:1019F000F7EE005AF8EEE66AE7EE056A76EEA56ABB
:101A000066EE266A3D4AB7EE006A136CC3F34623BE
:101A100007EE103AB8EEC77A70BC37EE067AC6EE1B
:101A2000877AFCEEE77AC0ED007A136CC3F30643C5
:101A300007EE103AB8EEC77A37EE067AC6EE877A26
:101A4000FCEEE77AC0ED017A136CC3F3066307EE90
:101A5000903AF8EEE77A77EE867A86EEA77ABCEED1
:101A6000C77A80ED027A704770BCC0E900228260BC
:101A700070471968890627D51C6807EE902A224905
:101A8000F7EE005A1B6CC4F3C102F8EEE77A9FED43
:101A90001D5AC3F30803D14006EE903A06EE101A21
:101AA000F8EEE66AB8EEC66AE7EE056A86EE277AD1
:101AB00076EEA56A66EE876AA4E707EE902ADFED68
:101AC000136AF8EEE77A8AE707EE902A9FED105A3C
:101AD0001B6CB7EE006AF8EEE77ADFED0A5AC3F343
:101AE0000803C5EE276A07EE903AF8EEE77AE7EECC
:101AF000257A77EE867A66EEA76A83E70044025875
:101B00000024744A000000390090D00320BCBE4B72
:101B10000024744C2DE9F0418268044686B02368A5
:101B2000D0E904101D680A43616E0243E069024374
:101B30000A4394492940944D0A43E168AB421A6034
:101B40005A6822F4405242EA0102A1695A6000F048
:101B5000A280226A9D6811438C4A666A2A4011431A
:101B60009960DA6A22F00F023243DA62884A9342BD
:101B700025D0884A934258D0874A934200F0448245
:101B8000864A934200F0BB82854A934200F0F0807F
:101B9000844A934200F0BD82834A934200F0EF856D
:101BA000824A934200F0EA82012500234FF001129D
:101BB00028462367C4E91A2306B0BDE8F0817C4BB0
:101BC0005B6D03F03803282BEED87A4A134493F860
:101BD0004050B0F5004F35D0202D00F2EB81202D84
:101BE00000F2BA80DFE815F0AF017701B800B80065
:101BF0006F01B800B800B8004601B800B800B800DE
:101C0000B800B800B800B8001901B800B800B800B2
:101C1000B800B800B800B800B800B800B800B80004
:101C2000B800B800B800B800EA00614B5B6D03F083
:101C30000703052BB8D85F4AB0F5004F134493F85B
:101C40006C50C9D1202D00F22F82202D00F210827D
:101C5000DFE815F0B2037F040E020E024F040E02FD
:101C60000E020E02B8040E020E020E020E020E0248
:101C70000E020E0219040E020E020E020E020E02D7
:101C80000E020E020E020E020E020E020E020E02D4
:101C90000E020E02EA0398683C4A024044480A4396
:101CA0009A60DA6A616A22F00F020A43DA62836D8F
:101CB00003F00703052B3FF677AF3E4F3B4493F805
:101CC0007460202E00F2AA81012E7FF66DAFB31E44
:101CD0001E2B3FF669AF01A252F823F0AF22040891
:101CE000A91B040859220408A91B0408A91B0408FD
:101CF000A91B040837230408A91B0408A91B04080E
:101D0000A91B0408A91B0408A91B0408A91B040893
:101D1000A91B0408D7220408A91B0408A91B04084E
:101D2000A91B0408A91B0408A91B0408A91B040873
:101D3000A91B0408A91B0408A91B0408A91B040863
:101D4000A91B0408A91B0408A91B0408A91B040853
:101D5000A91B04084D23040801250023A3F1100149
:101D60004FF6EF7291423FF61FAF2268D3601CE737
:101D70000F4B5B6D03F00703052B3FF615AF0E4AC3
:101D8000D55C26E7F369FFCF000C0058FFF4FF1184
:101D9000001001400044004000480040004C00405A
:101DA000005000400014014000780040007C0040DA
:101DB0000044025838B10B08A4B10B08002E00F003
:101DC000B281012E00F09485022E00F0A785032E2B
:101DD00000F0E885042E00F00986052E00F07C86D0
:101DE000062E00F0AE86072E00F00A87082E00F0BF
:101DF0008387092E00F0A7870A2E01F0158043F68D
:101E00000953A44A0B2E18BF13466268002503EB42
:101E10005203B3FBF2F39BB2A0E79F4B1A68920602
:101E200040F183811A689D4BC2F3C102D340002E5A
:101E3000EBD0012E00F00482022E00F0DC84032E91
:101E400000F0D684042E00F04485052E00F0C286F2
:101E5000062E00F0FF86072E00F03B86082E00F0CD
:101E60006D86092E00F0A9860A2E00F0E8860B2E5A
:101E7000CBD126E06846FFF78FFD626A019B002AFE
:101E8000C3D0012A00F0DC81022A00F0B484032AC6
:101E900000F0AE84042A00F01C85052A00F01685A7
:101EA000062A00F0B285072A00F01386082A00F0FF
:101EB0004586092A00F081860A2A00F0C0860B2A8E
:101EC000A3D11B0AA1E703A8FFF7A8FC626A049B41
:101ED000002A9AD0D5E7FFF763FC6F4A704BD269AE
:101EE000616AC2F30222134493F8303003F01F03F7
:101EF000D84001B3012900F0FE84022900F0DD84FE
:101F0000032900F0D784042900F04085052900F05A
:101F10003A85062900F02286072900F06E860829F6
:101F200000F0F686092900F026870A2900F0578775
:101F30000B2908BF000A6268002500EB5203B3FBBF
:101F4000F2F39BB20AE7FFF72BFC534A544BD269DA
:101F5000C2F302121344626A93F8303003F01F0395
:101F6000D84002B3012A00F0C984022A00F0AB84F1
:101F7000032A00F0A584042A00F00285052A00F057
:101F8000FC84062A00F0E485072A00F03F86082A30
:101F900000F0AF86092A00F0DA860A2A00F04A87A4
:101FA0000B2A08BF000A626800EB5203B3FBF2F38E
:101FB0009BB2D3E6402D7FF4F7AD002E00F0DB801E
:101FC000012E00F09E84022E00F0AB84032E00F060
:101FD000E584042E00F00D85052E00F08085062E88
:101FE00000F0B285072E00F0FA85082E00F0478633
:101FF000092E00F0B9860A2E00F0F7860B2E0CBFD2
:1020000080234FF4004300E7234B5B6D03F007038D
:10201000052B3FF6C9AD234AD55CDAE5402E7FF4A7
:10202000C3AD002900F0B480012900F072840229B8
:1020300000F0A084032900F0D084042900F0428538
:10204000052900F07385062900F0BD85072900F0F9
:102050000F86082900F06B86092900F0A6860A2958
:1020600000F0DE860B290CBF80254FF4004591E07F
:1020700001250023A3F110014FF6EF7291423FF6C4
:1020800093AD23F00F02C3F3420313432268D360DE
:102090008BE500BF00093D00004402580090D003CA
:1020A00038B10B08A4B10B08402D7FF47DAD002E94
:1020B00000F0C880012E00F0C780022E00F083845B
:1020C000032E00F0EE84042E00F02485052E00F08F
:1020D0006C85062E00F0AD85072E00F02486082EB4
:1020E00000F07386092E00F097860A2E00F0DB863A
:1020F0000B2E0CBF4FF480704FF48030A4E0A74B40
:102100005B6D03F00703052B3FF64EADA44AD55C8B
:102110005FE5A24B5B6D03F03803282B3FF644AD1F
:10212000A04AD55C55E5A04B6FE6002E00F0BF83BA
:10213000012E00F00084022E00F05384032E00F0E4
:10214000C584042E00F0EF84052E00F03985062E9C
:1021500000F08B85072EE6D0082E00F0C983092EEB
:1021600000F0DC830A2E00F04184904B904A0B2E45
:1021700018BF134649E64FF4004346E6874B5B6DB4
:1021800003F00703052B3FF60FAD8A4AD55C20E527
:102190004FF40045D4F8048008EB4803AB423FF607
:1021A00003ADB5EB083F3FF6FFAC202E00F2F28204
:1021B000012E7FF6F9AC023E1E2E3FF6F5AC01A3D0
:1021C00053F826F051270408A91B04083D270408EA
:1021D000A91B0408A91B0408A91B0408DB26040882
:1021E000A91B0408A91B0408A91B0408A91B0408AF
:1021F000A91B0408A91B0408A91B04086D260408D0
:10220000A91B0408A91B0408A91B0408A91B04088E
:10221000A91B0408A91B0408A91B0408A91B04087E
:10222000A91B0408A91B0408A91B0408A91B04086E
:10223000A91B0408A91B0408A91B0408D525040828
:102240005B08E2E54FF480306268002500EB520342
:10225000B3FBF2F39BB20DE703A8FFF7DFFA636A63
:10226000049D03B3012B00F0D182022B00F0C98240
:10227000032B00F0C382042B00F03383052B00F006
:102280002D83062B00F0B983072B00F03084082B38
:1022900000F06A84092B00F0A6840A2B00F0328536
:1022A0000B2B00F06782002D3FF47FAC72E7FFF745
:1022B00077FA3A4B1B6AC3F302133B4493F830306E
:1022C00003F01F0320FA03F5636A002BCAD1002D27
:1022D0003FF46BAC5EE7314B1A68950640F19D8286
:1022E0001B68334DC3F3C103DD4000293FF452AFF7
:1022F000012900F06383022900F05A83032900F0CA
:102300005483042900F04984052900F08B840629B0
:1023100000F00185072900F03485082900F0958533
:10232000092900F09D850A2900F0D7850B297FF443
:1023300031AF2D0A2EE76846FFF72EFB636A019D39
:10234000002B8FD1002D3FF430AC23E7002900F0A3
:102350006282012900F0D982022900F00983032951
:1023600000F03883042900F0A083052900F0D88309
:10237000062900F02C84072900F06984082900F060
:10238000DF84092900F015850A2900F0618543F6EC
:102390000955054B0B2918BF1D46FBE600440258A2
:1023A000A4B10B0878B10B0800093D0090D00300E0
:1023B0000090D003A4B10B08FFF7F2F9A44AA54B93
:1023C000D269C2F302121344626A93F8303003F008
:1023D0001F03D84002B3012A00F0AB82022A00F0AA
:1023E000F582032A00F06483042A00F09183052A11
:1023F00000F0CF83062A00F02584072A00F09B8492
:10240000082A00F0DD84092A00F0FB840A2A00F083
:102410002F850B2A08BF000A6268530803EB4003AC
:10242000B3FBF2F39BB225E6002E00F01A82012ED8
:1024300000F07B82022E00F0C482032E00F02F8376
:10244000042E00F06383052E00F09E83062E00F01C
:102450000684072E00F08584082E00F0AE84092E35
:1024600000F0D7840A2E00F0F78447F612237A4A48
:102470000B2E18BF13466268002503EB5203B3FB13
:10248000F2F39BB2F6E5724B1A68910640F1EB81CC
:102490001A68724BC2F3C10223FA02F206B3012E8C
:1024A00000F0BB82022E00F02A83032E00F064832A
:1024B000042E00F0B383052E00F01684062E00F0E3
:1024C0006B84072E00F09784082E00F0F384092E09
:1024D00000F0E6840A2E00F0E0840B2E08BF120AFA
:1024E000616800254B0803EB4203B3FBF1F39BB299
:1024F000C0E503A8FFF792F9626A049902B3012AC2
:1025000000F0F481022A00F00782032A00F04182E1
:10251000042A00F06982052A00F0E582062A00F00C
:102520000983072A00F07583082A00F08683092AA8
:1025300000F024840A2A00F055840B2A08BF090AF7
:1025400062680025530803EB4103B3FBF2F39BB22F
:1025500090E5FFF725F93E4A3E4BD269616AC2F326
:102560000222134493F8303003F01F03D84001B324
:10257000012900F0DC81022900F02A82032900F001
:102580009C82042900F0C082052900F012830629EC
:1025900000F06783072900F0DD83082900F0038439
:1025A000092900F04A840A2900F067840B2908BF32
:1025B000000A62680025530803EB4003B3FBF2F303
:1025C0009BB257E56846FFF7E7F9626A0199002A6E
:1025D000B6D094E7616A002900F02782012900F053
:1025E0001283022900F09C83032900F0CD83042983
:1025F00000F00484052900F06084062900F0658459
:10260000072900F05E84082900F0A984092900F058
:10261000A2840A2900F088841148124B0B2918BFA4
:10262000184600214FEA5803424618184FF000039D
:1026300041F100016FF016FAA0F540730A4A934287
:102640003FF6B2AA23680025D860FFF7AEBA00BFF4
:102650000044025838B10B0800127A000090D003F1
:1026600000093D000000093DFFFC0F00B34A11685E
:1026700011F0200100F0DD8113680021B048C3F3A0
:10268000C103D840636A0BB3012B00F05783022BC0
:1026900000F09983032B00F0B783042B00F0EB8349
:1026A000052B00F01D84062B00F02384072B00F07F
:1026B0002A84082B00F02384092B00F048840A2B7D
:1026C00000F041840B2B01D1000A00210902030212
:1026D00041EA10614FEA5800A6E76846FFF75CF947
:1026E0000198636A002102460BB3012B00F09F8121
:1026F000022B00F01382032B00F05282042B00F017
:102700008F82052B00F02883062B00F04083072BD7
:1027100000F06F83082B00F0A983092B00F0A3833E
:102720000A2B00F0C4830B2B01D1100A0021626830
:102730000902030241EA1061500876E703A8FFF797
:102740006DF80498636A00210246002BEFD0CCE7B5
:10275000FFF726F8794A636A0021126AC2F302126F
:10276000174497F8302002F01F02D0400246002B99
:10277000DDD0BAE72D0A002D3FF417AA0AE56F4B0A
:102780005B6D03F00703052B3FF60EAA6D4AD55C7F
:10279000FFF71FBA402E7FF407AA616A002900F0F4
:1027A0004181012900F02582022900F06C82032971
:1027B00000F00F83042900F04383052900F06083B3
:1027C000062900F06683072900F05E83082900F0DF
:1027D000A683092900F09E830A2900F0A9830B290A
:1027E0004FF000010CBF4FF400404FF4000019E718
:1027F000554AA2FB03239B08FFF707BB524BA3FBE1
:102800000535AD08002D3FF4D0A9C3E46D08002DB7
:102810003FF4CBA9BEE44D4DBCE400295CD00129B6
:1028200000F0C980022900F0FA80032900F06981D4
:10283000042900F0AB81052900F0ED81062900F0A4
:102840001B820729E7D008295FD0092900F0908072
:102850000A2900F02A813E4D394B0B2918BF1D462D
:1028600098E43C4B07E6002E51D0012E00F0D380B7
:10287000022E00F04281032E00F07C81042E00F035
:10288000D681052E00F03B82062E00F0A582072E91
:10289000E7D0082E49D0092E00F093800A2E00F0D0
:1028A00035812D4B2D4A0B2E18BF1346E3E5244BE3
:1028B000FFF7ABBA244BA3FB00308008FFF73BBB0C
:1028C000214BA3FB00308008FFF76DBB244AA2FB1D
:1028D0000323DB08FFF799BA194D5BE4204BA3FBF8
:1028E0000535ED08002D3FF460A953E4490827E6BB
:1028F0001C4BFFF78ABA4008FFF71DBB4008FFF7E3
:1029000052BB4FF48043FFF780BA164D42E4134B9D
:10291000B1E54FF480453DE4890811E6124BFFF71D
:1029200074BA4FF40053FFF770BA084BA3E54008A0
:102930003FE6400870E50D4BFFF767BA00440258C8
:102940000090D003A4B10B08ABAAAAAA00093D00CD
:1029500090D0030000127A0020A107000020A107F8
:10296000CDCCCCCC80841E0040420F000048E80152
:10297000C74D0FE44FF400550CE4C64BA3FB0030E9
:10298000C008FFF710BBC34BA3FB0030C008FFF724
:10299000D2BAC14BA3FB01239908D1E541F25553AB
:1029A000FFF733BABD4BFFF730BABB4BA3FB05357E
:1029B000AD08FFF7EFBBBA4DFFF7ECBB6D08FFF7B3
:1029C000E9BBB84B57E54FF480403DE4800823E570
:1029D0008008EEE5B14DFFF7DDBB41F25555FFF73D
:1029E000D9BBB14BFFF711BAC908A9E5AF4BFFF747
:1029F0000CBA4FF48053FFF708BA0C23B5FBF3F57C
:102A0000002D3FF4D2A8FFF7C5BBA34AA2FB0323C6
:102A1000DB08FFF7FAB9A64B2DE5520860E5A24D99
:102A2000FFF7B8BB4FF40000FCE5A248FAE5400808
:102A30007DE6626A002A00F0A480012A00F09881F5
:102A4000022A00F0AE81032A00F0F281042A00F08D
:102A50004282052A00F03D82062A00F05982072AA8
:102A600000F05482082A00F06B82092A00F0658287
:102A70000A2A00F03B820B2A8F4A8D4B0EBF0021A1
:102A8000032113464FEA58004246C0184FF0000396
:102A900041F100016EF0E6FFA0F54073CEE5874BF3
:102AA000E9E442F6AA20FFF7CFBB804DFFF772BBE7
:102AB000794BA3FB00239808AEE4774BA3FB0023DC
:102AC000980876E54FF48055FFF764BB7C4BFFF721
:102AD0009CB91B09FFF799B97A4BFFF796B940F6F5
:102AE000CC43FFF792B90A23B1FBF3F128E52D0996
:102AF000002D3FF45AA8FFF74DBB694BBBE4920889
:102B0000EEE46F4DFFF746BBC00852E5604BB2E400
:102B1000C00881E44FF40050FFF796BB800806E63A
:102B2000684DFFF737BB684BFFF76FB940F6CC45F0
:102B3000FFF730BB0C23B1FBF3F101E55B09FFF7B5
:102B400064B9624BFFF761B940F6AA23FFF75DB99C
:102B5000514BA3FB0030C008FFF725BA4E4BA3FB37
:102B60000030C008FFF7E7B96D09002D3FF41DA83C
:102B7000FFF710BB564B7EE4474BA3FB02239A089A
:102B8000AEE44D4B03217DE7524B74E44E4DFFF70D
:102B900001BB0A23B0FBF3F03EE4ED08FFF7FABAFD
:102BA000062200236EF05EFFC1E541F69810FFF7A4
:102BB0004BBB0A23B0FBF3F0FBE49B09FFF725B9FD
:102BC000454BFFF722B940F6AA25FFF7E3BA3F4D80
:102BD000FFF7E0BA0A22B3FBF2F3FFF716B94FF49E
:102BE0000063FFF712B9AD09002D3EF4DEAFFFF729
:102BF000D1BA4FF48000002114E50009FFF79BB91A
:102C0000364BFFF702B9364800210BE50009FFF704
:102C1000CAB9090994E4304DFFF7BCBAD2085FE4A1
:102C2000C00884E50A23B5FBF3F5FFF7B3BA1E4BE2
:102C300021E441F25450FFF707BB490980E4DB0966
:102C4000FFF7E3B80C23B0FBF3F0FFF7E5BB234D30
:102C5000FFF7A0BA0C22B3FBF2F3FFF7D6B80F4B85
:102C600009E40C23B0FBF3F0A3E41E4BFFF7CDB84F
:102C70004FF40065FFF78EBA1A4DFFF78BBA4FF489
:102C80008063FFF7C2B84FF400100021CAE400BF10
:102C900040420F00CDCCCCCCABAAAAAA2A2C0A0069
:102CA0000048E80180841E000024F40020A10700F1
:102CB0000090D0030000093D000090D0545814004B
:102CC000AAC2A200801A060000127A00151605009A
:102CD0005485450100350C0000A8610090D0030028
:102CE0000080841E556151000A23B2FBF3F2FFF706
:102CF000F7BB4009FFF757B99B4BFFF786B89B4BD3
:102D0000FFF7B9BBED09002D3EF44FAFFFF742BA14
:102D10004009FFF710B90C23B5FBF3F5FFF73ABAFA
:102D2000934800217EE44FF48050FFF78DBA4FF4B2
:102D30008065FFF72FBA0009FFF76EBB4008C5E4B6
:102D4000894DFFF727BA4FF22443FFF75EB8800999
:102D5000FFF729B900092CE40A2200236EF082FE55
:102D6000E5E4844BFFF787BB4FF40073FFF74DB8E2
:102D7000814B114686E68009FFF7DDB88909FFF728
:102D8000DFBB2D09FFF706BA7C4800214AE40C227C
:102D900000236EF067FECAE40C23B2FBF3F2FFF7E8
:102DA0009FBB774B6EE6400903E44FF40075FFF7D5
:102DB000F1B94FF22445FFF7EDB9724BFFF75BBB5A
:102DC0004009FFF729BB800880E44FF40060FFF75B
:102DD0003BBA6D48002125E46C4BFFF74CBBC009A2
:102DE000FFF7A9B8C909FFF7ABBB4FF48073FFF732
:102DF0000CB800099BE41209FFF772BB644800217C
:102E000010E48009FFF708BB062200236EF02AFEBB
:102E10005CE4554BFFF72FBB4FF48060FFF714BA0B
:102E20004FF48075FFF7B6B947F61223FEF7EDBFF2
:102E3000584B27E6C009FFF7B6B88009FFF7B9BBC2
:102E40004FF480100021FFF7EDBB6D09FFF7A2B929
:102E500047F61225FFF79EB94FF22443FFF70BBB4D
:102E6000AD09FFF797B99009002160E440095EE4DD
:102E7000C009FFF7D1BAC00828E4C009FFF799BB21
:102E800045480021FFF7CEBB4FF400200021FFF79B
:102E9000C9BB42480021FFF7C5BBD209FFF720BBE1
:102EA0009209FFF71DBB4FF40070FFF7CDB9D009B1
:102EB00000213CE45209FFF713BB39480021FFF71A
:102EC000B1BB38480021FFF7ADBB37480021FFF701
:102ED000A9BB364BD6E5364BD4E5ED09FFF75AB919
:102EE0000A2200236EF0BEFDFFF7F0BB284B002145
:102EF000C8E50C2200236EF0B5FDFFF7E7BB4009E3
:102F00000021FFF7E3BB0009FFF7E0BB294BB9E560
:102F1000294BB7E54FF400300021FFF783BB4FF496
:102F200080200021FFF77EBB24480021FFF77ABBF9
:102F30004FF480300021FFF775BB0D4B0021A1E558
:102F40001F4B00219EE5C0090021FFF7BFBB800990
:102F50000021FFF7BBBB1B480021FFF763BB1A48EA
:102F60000021FFF75FBB00BF48E801000050C3002D
:102F70000040420F20A10700000048E8002A2C0A68
:102F8000000024F490D0030000551500AAC2A2004E
:102F90000020A10700AAC2A200CC0C0000AA0A00CF
:102FA00000801A060090D003001516050000A861E5
:102FB0000000127A0000093D0055615100127A00AC
:102FC0000080841E0024F4000048E801374A936A18
:102FD00003F00303032B63D0136830B423F0806342
:102FE000334C1360256803E023685B1B022B54D825
:102FF00013681B01F8D4936A056823F47C3343EA11
:10300000053393628368C568013B013D5B022D0473
:103010009BB205F4FE052B434568013DC5F3080549
:103020002B430569013D2D0605F0FE452B439363B7
:10303000D36A456923F0C0032B43D362D36A856901
:1030400023F020032B43D362D36A23F01003D3620F
:10305000184BD56BC0692B4043EAC003D363D36AD6
:1030600043F01003D362D36AE1B101290CBF43F4EA
:10307000801343F40013D3620C4A136843F0806357
:103080001360216803E023685B1A022B05D81368DC
:103090001B01F8D5002030BC7047032030BC7047BE
:1030A0000120704743F40023D362E5E7004402584F
:1030B000602B00240700FFFF374A936A03F00303E5
:1030C000032B63D0136830B423F08053334C136068
:1030D000256803E023685B1B022B54D813689B0010
:1030E000F8D4936A056823F07C7343EA055393622E
:1030F0008368C568013B013D5B022D049BB205F46A
:10310000FE052B434568013DC5F308052B430569C2
:10311000013D2D0605F0FE452B431364D36A456936
:1031200023F440632B43D362D36A856923F400738D
:103130002B43D362D36A23F48073D362184B556C4C
:10314000C0692B4043EAC0035364D36A43F48073DD
:10315000D362D36AE1B101290CBF43F4000343F009
:103160008073D3620C4A136843F080531360216864
:1031700003E023685B1A022B05D813689B00F8D57F
:10318000002030BC7047032030BC704701207047DE
:1031900043F48003D362E5E700440258602B002427
:1031A0000700FFFF3F4AB0F1804F0368A0EB020227
:1031B000B2FA82F230B44FEA521223D012BB3A4C28
:1031C000A04247D004F58064A04243D004F5806457
:1031D000A04249D004F57844A04245D0334C344A4B
:1031E000904218BFA0424FD002F5806290424BD06F
:1031F0004D6923F080038C680A682B430360C46226
:10320000826223E04C6823F070032343294C041BA3
:10321000B4FA84F46409CD6823F440732B434D69F8
:1032200023F080032B4303608B68C3620B688362C7
:1032300052B94CB91D4A1E4B984218BF904203D058
:1032400003F58063984201D10B690363012330BC0D
:1032500043617047174C23F070034D68041B2B43E8
:10326000B4FA84F46409D6E74D6823F07003114C76
:103270002B43114D041BA842B4FA84F44FEA5414B2
:10328000C9D0002CC7D1A9E7CC6823F440734A69A0
:1032900023438C6823F0800313430A680360C462ED
:1032A0008262C7E700000140000400400040014086
:1032B0000044014000040140000C0040474B10B4A2
:1032C0001B68474CA4FB03435B0A03FB02F24AB1B1
:1032D000531E444C426B013B224201D0920407D55D
:1032E0005A1CF7D14FF0004318465DF8044B704765
:1032F000436B5C073DD4436B13F0010334D13A4B6D
:1033000083630369DBB2994231D14269374B134081
:10331000002BE9D0002A30DB510031D4940031D4A5
:10332000D00031D4110132D4540133D4D00134D47B
:10333000110235D4540236D4900240D4D1023BD489
:10334000540336D4900331D4D10344D414043FD46D
:1033500050043AD4910435D412F0080F14BF4FF43E
:1033600000034FF48033BFE701228263BCE70123EF
:10337000BAE7042213468263B6E74FF00073B3E75F
:103380004023B1E78023AFE74FF48073ACE74FF4FD
:103390000073A9E74FF48063A6E74FF40063A3E747
:1033A0004FF48053A0E74FF400539DE74FF4802380
:1033B0009AE74FF4003397E74FF4004394E74FF454
:1033C000804391E74FF480038EE74FF400138BE7BF
:1033D0004FF4801388E74FF4002385E700000024B2
:1033E000D34D621045002000C500200008E0FFFD1D
:1033F0000B4B01E0013B10D00269002AFADA0369A5
:10340000074A43F00103036101E0013A05D0036973
:1034100013F00103F9D1184670470320704700BF2D
:10342000400D030003682DE9F041C3F31005064683
:103430000C4635BB614A934274D902F5003293427F
:103440006FD902F50032934240F2AC8002F50032AF
:10345000934240F2A98002F50032934240F2A680E6
:1034600002F50032934240F2A38002F5003293420B
:1034700040F2A080B3F1016FC0F09E80052012F0F1
:103480004FFA4F4F1D463A7E012A00F0828003F129
:1034900078434FF00108B3F5801F4FF0000387F821
:1034A0001880FB6133D3022069F076FD00284CD1EF
:1034B000444A4FF00208D2F80C3143EA0803C2F83C
:1034C0000C31BFF36F8FBFF34F8F04F1200254F81C
:1034D000043B944245F8043BF9D1BFF36F8FBFF32F
:1034E0004F8F404669F058FDB8F1010F354A54D06E
:1034F000D2F80C3123F00203C2F80C3100233B76E2
:10350000002846D1336820333360BDE8F08140465F
:1035100069F042FDC8B92B4AD36843F00203D36077
:10352000CFE70125264F3B7E012B0BD04FF0010842
:103530000023404687F81880FB6169F02DFD50B1EB
:1035400000233B764FF0FF30DFE700236FF00100F0
:103550003B76BDE8F0814046DFF86880D8F80C3053
:1035600023F4E663C8F80C30D8F80C3043EA05259C
:1035700045F0A405C8F80C5069F00EFDD8F80C20F1
:10358000114B1340C8F80C300028D9D133681D46C0
:103590007DE76FF00100BDE8F081D36823F00203FE
:1035A000D360ABE70225BDE70325BBE70425B9E7F8
:1035B0000525B7E70625B5E70725B3E7FFFF0108AF
:1035C000602B002400200052FBF8FFFF0148FCF7AD
:1035D0000BBF00BF842B0024074810B4436A846DDE
:1035E00099691A6824B1234624305DF8044B1847C2
:1035F0005DF8044B704700BF602B00240148FCF7C6
:10360000F3BE00BFD42B0024074810B4436FD0F89A
:10361000A84099691A6824B1234674305DF8044BB8
:1036200018475DF8044B7047602B00240148FCF7F5
:10363000DBBE00BF242C0024084810B4D0F8C430EE
:10364000D0F8F84099691A6824B12346C4305DF86F
:10365000044B18475DF8044B704700BF602B0024F3
:103660002DE9F04FDFF874B300EB4004430083B062
:103670000BEB84040193A368002B00F06381804668
:10368000E08969F0F1FA207B0FF0FAFB0646607BD7
:103690000FF0F6FB08F101038146DBB2002E00F0CB
:1036A000888140F60C123372F280002800F06881A5
:1036B000037240F60C23C3803368B2889A61D9F84C
:1036C0000030B9F804209A611121304609270FF023
:1036D0008BFB112148460FF087FB6525002E00F07B
:1036E00034813268B3881169194200F02E811B04BD
:1036F000936111F031FC04460D4611F02DFC001BC6
:1037000061EB0501052871F10003F6D316B13368AA
:10371000B2889A6111F020FC04460D4611F01CFCA1
:10372000001B61EB0501052871F10003F6D3013F91
:10373000D3D11EB1B38832681B04936111F00CFC25
:1037400004460D4611F008FC001B61EB050105283D
:1037500071F10003F6D3B9F1000F05D0B9F80430C8
:10376000D9F800201B04936111F0F6FB04460D46C6
:1037700011F0F2FB001B61EB0501052871F100035C
:10378000F6D316B13368B2889A6111F0E5FB0446AE
:103790000D4611F0E1FB001B61EB0501052871F1FD
:1037A0000003F6D3B9F1000F04D0D9F80030B9F80E
:1037B00004209A61019B30463E21834C03EB0806AE
:1037C0004FEA88050BEB8606F27C0FF033FBF27CA8
:1037D00048463E210FF02EFBB26808EB880304EB4D
:1037E00003135A62794B9A4200F0C580FDF7D8FF67
:1037F000774BDA69C2F30212764B134493F83030F8
:1038000003F01F03D840019B43440BEB83031B7C55
:10381000022B00F0B980032B00F0BF80012B14BFF6
:103820004FF4C8714FF4487168F0D0FF05EB0803FE
:1038300004EB0313986205EB0803002204EB031367
:10384000DA62C3E90D22C3E9102201221A6393F858
:10385000652002F0FF01002A00F0A88005EB0802B5
:10386000242704EB0212D2E9093182F86570186846
:1038700021F0706120F0010018601961996821F44D
:10388000004199604FF40041996001F1007158685E
:1038900001435960D16BD868090220F40040D86018
:1038A000D96000211960186840F0010018602020DC
:1038B000916682F86500516582F8661092F865009D
:1038C0002028C6B217D192F86400012813D082F8DC
:1038D0006570186820F001001860186820F48050A6
:1038E000186018681860186840F00100186082F8C5
:1038F000656082F86410019B02210127364E434423
:1039000045440BEB830B04EB05149BF8120069F0A4
:10391000A5FB9BF812309BF81100022103F01F0257
:103920005B0907FA02F246F8232069F097FB9BF83F
:10393000113003F01F025B0907FA02F246F8232058
:1039400084F8207003B0BDE8F08F013D0DD011F078
:1039500003FB04468A4611F0FFFA001B61EB0A01E3
:10396000052871F10003F6D3B8E6002E3FF4C1AE8E
:103970003268B388BBE6FDF713FF154B1A6A39E7C7
:103980003368B2889A619FE6642168F01FFF05EBF7
:10399000080304EB031398624DE7C82168F016FF93
:1039A00005EB080304EB0313986244E783F8641003
:1039B00054E700283FF488AE89F8083040F60C231D
:1039C000A9F806307BE600BF602B0024001C0058DD
:1039D0000044025838B10B0800E100E00000002468
:1039E0002DE9F04F441C83B09DF8346065D0044647
:1039F000BF4D00EB80004FEA840905EB001090F802
:103A00002080B8F1000F5AD0002B18BFFF2A0CBF3E
:103A1000012700273E4056D190F86560202E40F0E7
:103A2000C3809FB2002B00F0BC8090F86430012B63
:103A300000F0BA8001232E6880F86430406A04E008
:103A40002B689B1B192B00F20A81836913F4004336
:103A5000F6D109EB040A4FF0210E4FF0400C019211
:103A600005EB0A1B8BF865E0CBF858308BF866C085
:103A7000CBF868300C9BABF84E704F00CBF8483059
:103A8000436823F07F7323F4593323F47F7323F0C7
:103A9000030343EA4103974901EB0A1A9649194384
:103AA00041603146504669F04DFA002840F084816B
:103AB000DBF82410019A8A628AE04FF00008404641
:103AC00003B0BDE8F08F90F86520202A6CD190F803
:103AD0006420012A68D00122D5F800A080F8642073
:103AE000426A05E02868A0EB0A00192800F26C8100
:103AF000906910F40040F5D14F0009EB04014FF03C
:103B0000210E1FFA83FC05EB01110C9B81F865E087
:103B10004FF0100E8B6481F866E08866A1F84EC005
:103B2000B1F84E3088659BB2FF2B40F28681536816
:103B30007248034072483B431843FF23A1F84C30BE
:103B4000506009EB04026B4B05EB021B019203EB87
:103B50000218BBF84E30514640469BB2002B00F095
:103B60007C8169F0EFF9F8B9DBF84820DBF8241024
:103B700012F8010BBBF84C308862CBF84820013BAF
:103B8000BBF84E209BB2013AABF84C3092B2ABF886
:103B90004E20BBF84E2092B2002BDAD1002AD8D0AA
:103BA00073E04FF400738366B5F810314FF00008EE
:103BB000204601339BB2A5F81031FFF751FD404676
:103BC00003B0BDE8F08F2A68921B0A2A00F2E78052
:103BD0008B6913F08003F6D009EB040205EB0212A7
:103BE000B2F84E309BB2FF2B40F2FE804B68454846
:103BF000034045483B431843FF23A2F84C3048603C
:103C000009EB040305EB031B019305E0BBF84E3001
:103C10009BB2002B00F0F8803146504669F092F9D3
:103C20000028C1D1DBF84810DBF8242011F8010B83
:103C3000BBF84C309062CBF84810013BBBF84E10FB
:103C40009BB20139ABF84C3089B2ABF84E10BBF8DF
:103C50004E1089B2002BD9D10029D7D033E0A1442E
:103C60002021002205EB0919D9F8683089F8642071
:103C70000B43C9F8683089F8651089F8662093E726
:103C80002A68A2EB0A020A2A77D88B6913F080030C
:103C9000F6D0BBF84E309BB2FF2B47D94B681A4A7F
:103CA00023F07F7323F4583323F47F7323F003034B
:103CB0003B431A43FF23ABF84C304A6049E72B687B
:103CC0009B1B0A2B48D8906910F08000F7D0BBF8F6
:103CD0004E309BB2FF2B19D953680A490B400A4951
:103CE0003B431943FF23ABF84C3051608EE700BFD4
:103CF000602B0024842B002400200181009800FC0C
:103D00000020FF81009C00FC0000FF01BBF84E304A
:103D100057489BB25168ABF84C30DBB2014047EAE0
:103D200003430B4343F0007353606FE7BBF84E301F
:103D30009BB2DAB2ABF84C304B6823F07F7323F4BC
:103D4000583323F47F7323F003033B4343EA0243D6
:103D500043F000734B60FCE6A14405EB0919D9F868
:103D6000683089F8640043F02003C9F868302023E4
:103D700089F8653089F8660016E7A1449C4605EB92
:103D80000919D9F8683089F864C043F02003C9F8EC
:103D90006830202389F8653089F866C004E71A4640
:103DA00009EB0403202005EB0313996E0143996688
:103DB00083F8650083F8662009EB0403002205EB15
:103DC000031383F86420EFE609EB040320200021AD
:103DD00005EB03139A6E83F8641002439A6683F826
:103DE000650083F86610DFE6B2F84E3020489BB2DB
:103DF000A2F84C30DBB24A6847EA0343024013435F
:103E000043F000734B60FBE63146504669F070F8B2
:103E100000287FF4C9AE019B05EB0315DBF82420D5
:103E20002024144ED4615168314051608BF86540B4
:103E300085F864008BF8660041E6B1F84E300E4814
:103E40009BB2A1F84C30DBB2516847EA0343014012
:103E50000B430A491943516073E669F049F8002899
:103E60007FF4A2AE019BB04605EB0315D6E700BF79
:103E7000009C00FC00E800FE009800FC002000828E
:103E80002DE9F04F441C83B09DF8347000F0508150
:103E9000BB4C00EB800C0646850004EB0C1C9CF828
:103EA0002080B8F1000F7FD0FF2A14BF002707F051
:103EB0000107002F7CD09CF86520202A69D19CF84E
:103EC0006420012A65D00122DCF82400D4F80080A7
:103ED0008CF8642005E02268A2EB0802192A00F29F
:103EE0002D81826912F40042F5D14FEA4109A919E6
:103EF0004FF0220C1FFA83FE04EB01110C9B81F89A
:103F000065C04FF0100C8B6481F866C08A66A1F81A
:103F10004EE0B1F84E308A659BB2FF2B00F224814F
:103F2000B1F84E3042689BB2A1F84C30DBB29549F3
:103F300049EA03430A401343934A1A434260AB19C8
:103F4000924A04EB031B019302EB031ABBF84E30B9
:103F50009BB2002B00F0E581DBF824200CE0DBF8BD
:103F60002420916911F0200140F068812368A3EBBF
:103F700008030A2B00F27B819369414650465B0798
:103F800000F121819369DB06EBD568F06FFF002813
:103F9000E5D0B4F8103130464FF0000801339BB241
:103FA000A4F81031FFF75CFB404603B0BDE8F08F8A
:103FB0009CF865002028ECD198B20C9B002B00F0F7
:103FC000CC80002800F0C9809CF86430012BE0D040
:103FD000012327688CF86430DCF824C004E02368EF
:103FE000DB1B192B00F2AA80DCF8183013F4004315
:103FF000F5D105EB060E4FF0220B4FF0400A01926F
:1040000004EB0E1989F865B0C9F8583089F866A034
:104010004FEA410AC9F868300C9BA9F84E00C9F86C
:104020004830DCF8043023F07F7323F4593323F451
:104030007F7323F0030343EA4103544901EB0E1B52
:10404000534919435846CCF80410394668F07AFFB2
:10405000002840F0B180D9F82410019A8A6204E067
:104060002268D21B0A2A00F29B808B6913F040035E
:10407000F6D0AA1904EB0212B2F84E309BB2FF2B15
:1040800040F278814B683F480340424843EA0A03C4
:104090001843FF23A2F84C304860AB193E4904EBAB
:1040A00003190193D9F8240004E02268D21B0A2ADC
:1040B00000F2EA80836913F00403F6D0426AD9F86B
:1040C00048301A70B9F84E30B9F84C20013B013A2B
:1040D0009BB292B2A9F84E30D9F84830A9F84C20DA
:1040E0000133C9F84830B9F84E309BB213B1002AF9
:1040F00000F0F980B9F84E309BB2002BD2D139468E
:10410000584668F0F5FE00287FF443AF019B234D2D
:1041100004EB0312D9F824302024DC6159682940CB
:10412000596089F8654082F8640089F866003BE7C9
:104130004FF00008404603B0BDE8F08FAB192020D7
:10414000002104EB03139A6E83F8641002439A660D
:1041500083F8650083F866101BE7AB194FF4007213
:1041600004EB03139A6614E74368064A1340094AAE
:1041700043EA09031A43FF23A1F84C304260DEE60C
:10418000602B0024009800FC00240082842B002473
:10419000002001800024FF81009C00FC00E800FE5C
:1041A0001A46AB19202004EB0313996E014399665C
:1041B00083F8650083F86620AB19002204EB031333
:1041C00083F86420E5E6526ADBF848301A70BBF8E1
:1041D0004E30DBF84820013B01329BB2CBF848203F
:1041E000ABF84E30BBF84C30BBF84E20013B92B2DE
:1041F0009BB2ABF84C30002B7FF4A8AE002A3FF402
:10420000A5AEDBF8241004E02268A2EB08020A2A1B
:1042100059D88B6913F08003F6D0BBF84E309BB2AF
:10422000FF2B40D94B685B4A13405B4A43EA0903C2
:104230001A43FF23ABF84C304A6087E6936959076D
:1042400003D5BBF84C30002BBDD12021AB1953480E
:10425000D16104EB031355682840506000229A6630
:1042600083F8642083F8651083F8662091E635446E
:1042700004EB0515AB6E85F8641043F02003AB66C4
:10428000202385F8653084E6AA1904EB0212916EAA
:1042900082F8643041F020019166202182F8651097
:1042A00082F8663075E6BBF84E303A489BB24A68F1
:1042B000ABF84C30DBB2024049EA0343134343F00E
:1042C00000734B6042E61946AB1904EB03139A6E78
:1042D00083F8641042F020029A66202283F8652059
:1042E00083F8661055E6D9F8240003E02268D21B53
:1042F0000A2AC9D8836913F08003F7D0B9F84E3081
:104300009BB2FF2B27D94FF0FF03A9F84C3043682D
:104310000B4043EA0A0343F0FF7343F480334360E6
:10432000E8E64146504668F0E3FD00287FF431AEF0
:10433000019B2021194DB84604EB0314DBF824300F
:10434000D9615A682A405A608BF8651084F8640075
:104350008BF8660028E6B9F84E3042689BB20A40F6
:10436000A9F84C30DBB24AEA0343134343F000732D
:104370004360BFE6B2F84E3009489BB2A2F84C3019
:10438000DBB24A684AEA034302401343054A1A4330
:104390004A6082E6009C00FC0000FF0100E800FE8D
:1043A000009800FC002400820248836B0BB12C3083
:1043B00018477047000000240248836D0BB14C3051
:1043C00018477047000000240248836F0BB16C301F
:1043D00018477047000000240348D0F898300BB10C
:1043E0008C301847704700BF000000240348D0F805
:1043F000B8300BB1AC301847704700BF0000002444
:104400000348D0F8D8300BB1CC301847704700BF04
:10441000000000240348D0F8F8300BB1EC30184706
:10442000704700BF000000240348D0F8183113B1D2
:1044300000F5867018477047000000240348D0F844
:10444000383113B100F5967018477047000000240A
:104450000348D0F8583113B100F5A67018477047DB
:10446000000000240348D0F8783113B100F5B6708D
:1044700018477047000000240348D0F8983113B162
:1044800000F5C67018477047000000240348D0F8B4
:10449000B83113B100F5D6701847704700000024FA
:1044A0000348D0F8D83113B100F5E67018477047CB
:1044B000000000240348D0F8F83113B100F5F6707D
:1044C00018477047000000240348D0F8183213B191
:1044D00000F50370184770470000002410B54468C9
:1044E0008646464820401843CEF80400DEF8000017
:1044F00040F00100CEF80000DEF8000040F400704B
:10450000CEF80000EBB140F2E930DEF81440A40729
:1045100029D5002A46D012F8010B40F2E93C8EF86A
:10452000200002E0BCF1010C3ED0DEF81440E007B0
:10453000F8D59EF83000C0B209B101F8010B013B7B
:10454000E1D1DEF814301B07FBD5DEF8183001206E
:1045500043F01003CEF81830DEF8003023F00103EA
:10456000CEF8003010BD0138CFD1254B9E450CD080
:10457000A3F578439E453DD003F580639E453BD02F
:1045800003F578439E4533D1032000EB40031D4AD9
:10459000002002EBC302B2F8403201339BB2A2F812
:1045A000403210BDFF20B8E7154B9E450DD0A3F556
:1045B00078439E4519D003F580639E4512D003F5DC
:1045C00078439E4514D14FF0030C0E4B0CEB4C0C72
:1045D000002003EBCC0CBCF8403201339BB2ACF8AA
:1045E000403210BD4FF0020CEFE74FF0010CECE74A
:1045F000002010BD0120C8E70220C6E70000FFFF31
:1046000000300140000000242DE9F041314A82B021
:10461000314D00240746036801E052F83450AB42A4
:104620000AD001340E2CF8D100212C4A052001912A
:1046300009F0EEFB019B18E0294B03EB8408D8F846
:104640001461B6B178790021431C00EB400203EB02
:10465000430306EBC202DB00D760C2E90411F15448
:10466000182303FB006606F10803184602B0BDE8F4
:10467000F0810721682009F0BFFCC8F8140100B3DD
:104680006822314674F0FAFC1248D8F81411334607
:1046900000EBC404104A89600962896309650C60F3
:1046A00001E050F83320954205D001330E2BF8D1AC
:1046B0004E600E46C6E70B4E06EB83164E600E4666
:1046C000C0E701460190084A052009F0A1FB019BC3
:1046D000CBE700BFB4B10B080000014094500C08B8
:1046E000602B0024AC2C0024BC500C082DE9F043B6
:1046F000002587B0382224482946244F244E254CD3
:1047000074F0BCFC57F825103246002301E054F841
:104710003320914231D001330E2BF8D100200535E2
:1047200068F0A2FA462DEDD1DFF860900025DFF8A1
:104730006C80194F09F58C7699F8040009F1140979
:104740000EF09EFB044698B103683B449B0A08EBBD
:104750004303B3F8EC0068F087FAA28802232068CC
:1047600001A90595CDE90125CDE90335FCF7B6FE94
:10477000B145E1D107B0BDE8F083084A02EBC303BD
:10478000B3F88000CBE700BF742C00248C02002417
:1047900000000140B4B10B080000FEA738B10B08BF
:1047A00030B40C4C0022234603E0013214330E2AAD
:1047B0000CD093F804C08445F7D1DD68294201D1BB
:1047C0000029F2D1142000FB024000E0002030BCA0
:1047D000704700BF8C020024F0B44468A37913F042
:1047E000020266D19446036864795B689D48204460
:1047F00093F83C40012C90F8000158D0012483F834
:104800003C40022483F83D4014284AD8DFE810F0E9
:1048100055004900490049008F00490049004900FE
:104820003601490049004900C400490049004900D7
:10483000F700490049004900150018688A4E046ACB
:10484000B04224F480140462046A456824F400141D
:1048500044EA0252446D24F4E04444F4C0440ED0CF
:1048600006F58066B0420AD0804F06F58046B04219
:1048700018BFB84203D006F58066B04203D125F4D4
:10488000003545F4802545604465C1650262426D8E
:1048900042F400624265426D22F480624265426DDC
:1048A00042650121002283F83D1083F83C20F0BCD2
:1048B000704702224FF0080C95E718686C4D046AA7
:1048C000694E24F00104B0420462046A24F0020438
:1048D00042EA04024468876905EA070545F0600575
:1048E0000ED006F58066B0420AD0604F06F58046CD
:1048F000B04218BFB84203D006F58066B04207D177
:1049000022F0080244F440744CEA020C2CF0040239
:104910004460856141630262826942F008028261FB
:10492000826922F00402826182698261B9E71868B3
:10493000504D046A4C4E24F01004B0420462046AE4
:1049400024F0200444EA02124468876905EA070556
:1049500045F4C04500F0CB8006F58066B04200F01B
:10496000C680424F444EB04218BFB84203D006F54D
:104970008066B04201D144F4406444608561816343
:104980000262826942F400628261826922F480627A
:1049900082618269826184E71868334E046AB0429A
:1049A00024F480540462046A456824F4005444EA00
:1049B0000232C46924F4E64444F4C0440ED006F53F
:1049C0008066B0420AD0294F06F58046B04218BF33
:1049D000B84203D006F58066B04201D145F4804567
:1049E0004560C46101640262C26942F40062C2614E
:1049F000C26922F48062C261C269C26151E718686B
:104A0000194E046AB04224F480340462046A456892
:104A100024F4003444EA0242446D24F0700444F06B
:104A200060040ED006F58066B0420AD00F4F06F53E
:104A30008046B04218BFB84203D006F58066B04247
:104A400001D145F480354560446581650262426D5F
:104A500042F008024265426D22F004024265426D56
:104A600042651EE738B10B080000014000400140DC
:104A70008CFFFEFFFF8CFFFE0044014018681F4DB5
:104A8000046AA84224F480740462046A466824F428
:104A9000007444EA0222C46924F0730444F0600400
:104AA0001ED005F58065A8421AD0154F154DA842B5
:104AB00018BFB84203D005F58065A84201D146F47D
:104AC00040564660C461C1630262C26942F0080296
:104AD000C261C26922F00402C261C269C261E0E639
:104AE00022F4006242EA0C2222F48062E7E722F01C
:104AF000800242EA0C1222F040023CE70000014032
:104B0000004001400044014042685379032B0FD814
:104B1000DFE803F00B0805021068403070471068AA
:104B20003C30704710683830704710683430704738
:104B300000207047436801689A795B7912F0040F8E
:104B4000044A4868134493F8001101D06BF0A0B8F0
:104B50006BF0C2B838B10B08F0B54468364A246926
:104B6000C368C4F303245B6852F82460EFF3118434
:104B7000102585F312884568304F95F805E0D0F888
:104B80000CC002EB4E02D5F800E0128C02F4F05596
:104B9000DEF80C2022EA0502CEF80C2017F806E019
:104BA000DCF8102053F80E501F2A25F0010543F8B9
:104BB0000E5036D9203A2025DCF804C005FA02F25E
:104BC000CCF80C20E2B282F31188BA5D1C4C03EBE6
:104BD000020C46684569DCF804703C400C43CCF894
:104BE00004407179032924D8DFE801F01815120276
:104BF00031684031CCF80C500124CCF80810995899
:104C000041F0100199509958214399500474F0BD16
:104C100031683C31EEE731683831EBE731683431E7
:104C2000E8E72025DCF804C005FA02F2CCF80820F9
:104C3000C8E70021DEE700BF38B10B089CB20B08C3
:104C40000000FFFF03681A7E012A29D0002293F892
:104C50003010012904D1022142F4806283F830101F
:104C600093F84810012905D093F8601001290AD063
:104C700072B97047022142F4006283F8481093F839
:104C80006010012904D1022142F4805283F860109F
:104C90001B6800211B685962D9680A43DA607047B3
:104CA00002214FF400721976D1E700BF08B5204BFE
:104CB00098420ED003F5806398420AD01D4A03F54E
:104CC0008043984218BF904203D003F58063984216
:104CD0001BD1FCF765FD184B1849DA69DB69C2F393
:104CE0000222C3F302230A4492F8302002F01F028A
:104CF000D040114A1269C2F3C03243EAC2028B1893
:104D000093F8043103FB00F008BDFCF749FD0A4BA2
:104D10000A49DA69DB69C2F3021CC3F3021301EB2F
:104D20000C0292F8302002F01F02D040E1E700BFF1
:104D300000000140004001400044025838B10B0817
:104D4000D0E90030013904EE902A1A68006870B585
:104D500084B05C6815688EB2FFF7A8FF07EE900A72
:104D6000F8EE644A9FED5F7AF8EE677A87EEA40A60
:104D700030EE070A6FF0ECF923680138AB4280B2DD
:104D80007FD00023802194F83D20E660A360A161DC
:104D9000C4E90050C4E90433002A7BD00223211D5A
:104DA000284684F83D30FEF7FDF94F4B01229D4225
:104DB00084F83D2014D0B5F1804F11D0A3F57C4389
:104DC0009D420DD003F580639D4209D003F58063B9
:104DD0009D4266D003F578439D4262D004B070BD19
:104DE00094F83C3000224FF48051012BCDE90012A1
:104DF000CDE90222F2D0236802203C4984F83D002C
:104E0000986801400120996084F83D0084F83C20B6
:104E100094F83C10002201290292CDE90022DDD055
:104E2000314A0221934284F83D105868996834D081
:104E300002F58062934230D02D4A20F07000B3F129
:104E4000804F18BF934258602A480CBF01220022AD
:104E5000834208BF42F0010200F58060834208BF30
:104E600042F0010212B9244A934202D121F080019A
:104E700099600122002384F83D2084F83C3004B07E
:104E800070BD636883427FF47CAFE368B3427FF414
:104E900078AFA3E784F83C2080E7184A02405A60C4
:104EA000E4E794F83C3000214FF48052012BCDE927
:104EB0000021CDE9021191D02368022284F83D201F
:104EC0000A4A9868024001209A600D4A84F83C1012
:104ED000954284F83D009BD0A2F5784295427FF43C
:104EE0007DAF95E70AD7233C000001408800CEFF44
:104EF0000004004000080040001800408FFF0FFF32
:104F000000040140024B0348D3F81411FCF798B990
:104F1000602B002400000140034B4FF08040D3F889
:104F20001811FCF78DB900BF602B0024024B034819
:104F3000D3F81C11FCF784B9602B00240004004056
:104F4000024B0348D3F82011FCF77AB9602B0024F8
:104F500000080040024B0348D3F82411FCF770B955
:104F6000602B0024000C0040024B0348D3F83011A2
:104F7000FCF766B9602B002400040140024B034893
:104F8000D3F84011FCF75CB9602B002400180040F6
:104F9000024B0348D3F84C11FCF752B9602B0024A4
:104FA00000400140024B0348D3F85011FCF748B9C8
:104FB000602B002400440140024B0348D3F85411F5
:104FC000FCF73EB9602B00240048014010B5064CA8
:104FD0000648D4F83011FCF733F9D4F844110448EA
:104FE000BDE81040FCF72CB9602B00240004014000
:104FF000001C004010B5064C0648D4F83011FCF7F0
:105000001FF9D4F848110448BDE81040FCF718B95E
:10501000602B00240004014000200040BFF34F8FAC
:105020000549064BCA6802F4E0621343CB60BFF344
:105030004F8F00BFFDE700BF00ED00E00400FA0560
:105040000021012008B50EF0E9F972B6FFF7E6FF7E
:105050002DE9F043BDB0BFF35F8F8A4C0021626A37
:105060000B460D4622F4803262620A46C4F8941060
:10507000C4F898300133C4F89C20112BC4F8A02048
:10508000F6D10523C4F89430636A43F48033636235
:10509000BFF34F8FBFF36F8F7B487C4A7C49121A56
:1050A00071F044FED4F888207A4B012142F470025A
:1050B000C4F8882019601D611A6842F080021A60E5
:1050C0001A680A431A601A6842F480321A601A6831
:1050D00042F480521A609D61DD611D629D62DD6255
:1050E0001D635D639D63DD631D645D641A6822F466
:1050F00080221A601D664FF00063674AC2F80811EB
:10510000A3606BF02DFB654AD36813F0040FD368DE
:1051100040F0A380624B0021604A0391D96A21F0DC
:105120000101D962DB6A03F001030393936943F43D
:1051300040439361936903F440430393039B936952
:105140009E04FCD54C2200210DA8564C73F096FF0E
:10515000554A42F2030304F110011268B3EB124FF7
:105160004FF000024FF00C0318BF0C460792E268A4
:10517000A370002A4CD1494A494B916941F44041FE
:105180009161926902F440420792DA6A42F00102A8
:10519000DA62DB6A03F001030793079B3F4A9369D6
:1051A0009D04FCD53B4B4FF4403140480126D3F8D9
:1051B000E020002542F08002C3F8E020D3F8E03080
:1051C00003F0800306930323069A816108A90893DC
:1051D0000B93CDE90965FCF781F94FF48033082280
:1051E0000DA80E9302231D92E2790D961E95CDE92E
:1051F0001633A3781893A3881993A3791A93237A63
:10520000CDE91B23FBF782FA032838D0A0B1FEE7D3
:10521000234BD96A21F00101D962DB6A1F4903F0EF
:10522000010307938B6923F4404313438B618B691C
:1052300003F440430793B0E71D4B1A6812F00E0FBA
:105240003AD11A6822F00F0242F002021A601B687B
:1052500003F00F03022B2FD0FEE723F00703154CBA
:1052600043F00203D360216805E023685B1AB3F5BD
:105270007A7F3FF64FAF53689F04F6D54AE7FFF7B2
:10528000DFFE00BF00ED00E000000000B82E0000CF
:10529000E0C60C0800440258008000510048025843
:1052A00000040058A40300240010005C001C0258F5
:1052B00000200052602B00246B4A936903F07003B6
:1052C0003F2B05D8936923F0700343F040039361AB
:1052D000654AD36903F070033F2B05D8D36923F0E7
:1052E000700343F04003D3615F4AD36903F4E06382
:1052F000B3F5806F05D2D36923F4E06343F4806390
:10530000D361594A136A03F070033F2B05D8136A1F
:1053100023F0700343F040031362534B9A69140760
:1053200005D49A6922F00F0242F008029A614E4AAF
:10533000936923F470639361136898018CD51369A2
:1053400041F28830494C23F0070343F00303136113
:10535000216804E023685B1A834200F29D8113698F
:1053600003F03803182BF5D1936903F00F03082BD2
:1053700005D9936923F00F0343F0080393613C4A76
:10538000136803F00F03022B0BD9136823F00F03EC
:1053900043F002031360136803F00F03022B00D0E5
:1053A0005AE7314A936903F07003402B05D993699A
:1053B00023F0700343F0400393612B4AD36903F059
:1053C0007003402B05D9D36923F0700343F04003E9
:1053D000D361254AD36903F4E063B3F5806F05D93F
:1053E000D36923F4E06343F48063D3611E4A136AF4
:1053F00003F07003402B00F247811B4EFCF7AEF91F
:105400001C4BB2691C4DC2F30322134493F8303095
:1054100003F01F03D84028606868FBF7ADFF002841
:1054200040F03B811023149016900DA80D93FBF7CC
:105430006DF9002840F027813368104943F080035C
:105440003360D6F8F43043F00203C6F8F430D6F8EF
:10545000F43003F002030293029B0A6A084B42F005
:1054600001020A62216810E000440258602B002407
:105470000020005238B10B0800000024000400583E
:1054800080380100013B3FF4FAAE22689142F9D026
:10549000226823689B1A0A2BFBD94FF48023A24C65
:1054A0000DA84FF000080D934FF440130326022778
:1054B0002E936AF055FCD4F8EC300DA843F00203AB
:1054C000C4F8EC30D4F8EC3003F002030193019BF4
:1054D000D4F8943043F00203C4F89430D4F89430F4
:1054E00023F00203C4F89430904B1A6841F203038E
:1054F000B3EB124F8E4B8F4A38BF1A468E4B5A6011
:105500001A6822F47C5242F400521A601A6842F07F
:1055100060021A600D96CDE92A886AF021FC4FF4EA
:10552000E0430DA8CDF8E0800D93CDE924886AF022
:1055300017FC18230DA8CDF8B4800D93CDF8C880C2
:105540006AF00EFC4FF4803305210DA811960D93DF
:1055500020934FF4FA73CDF854801097CDE90E13D1
:105560000423CDE9138812936AF0FAFBD4F8E030F3
:1055700008A9724843F00103C4F8E030D4F8E030E1
:10558000099703F001030B96CDF828800593059B3E
:105590004FF48073CDF830800893FBF79FFF2369A9
:1055A00000F5006023F0FE7343F088732361D4F8A4
:1055B000E03043F00403C4F8E030D4F8E030099759
:1055C00003F004030B96CDF8288004934FF4007386
:1055D000049A0893CDF83080FBF780FF236923F00D
:1055E0007E4343F0FC432361FCF7B8F82860BFF327
:1055F0005F8F534D4646534C01276B6A23F480332B
:105600006B62C5F8948023E0002944D0D4F8009060
:10561000637A103414F8060C1B0643EA007343EA5D
:10562000410314F8051C43EA814314F8041C43EABF
:10563000414314F8031CC5F89860013643EA01435E
:10564000C5F89C90032E43F00103C5F8A03025D087
:105650006368217A002BD7D0D4F800900029D7D1E5
:1056600029F01F08A3EB0803202B38BF202318467E
:10567000984671F055FB431E07FA03F1884508BFB1
:105680000346D9B2C4E7FEE7136A23F0700343F080
:1056900040031362B1E6FEE7DEE5DDE50523C5F86C
:1056A00094306B6A43F480336B62BFF34F8FBFF368
:1056B0006F8FBFF34F8FBFF36F8F0022C5F850225B
:1056C000BFF34F8FBFF36F8F6B6943F400336B6190
:1056D000BFF34F8FBFF36F8FC5F88420BFF34F8F99
:1056E000D5F8805043F6E0761549C5F34E34C5F33E
:1056F000C905640104EA06002B4640EA8372013BB7
:10570000C1F86022F9D2203C14F1200FF2D1BFF38E
:105710004F8F4B6943F480334B61BFF34F8FBFF31F
:105720006F8F3DB0BDE8F083004402580010005C6C
:105730007FBB22307FBB2200008400400000025863
:1057400000ED00E0C4030024704700BF30B5012025
:1057500085B00DF05DFE01286DD03C494FF6FF008D
:105760003B4ACC683B4B04403B4D3C482243CA601B
:105770005A6FC5F8CC24D3F8F42042F00202C3F8E3
:10578000F420D3F8F42002F002020392039AD3F833
:10579000DC2042F00052C3F8DC20D3F8DC2002F019
:1057A00000520292029AD3F8DC2042F08042C3F801
:1057B000DC20D3F8DC2002F080420192019AD3F879
:1057C000DC2042F00042C3F8DC20D3F8DC20036880
:1057D00002F0004222480092009AD1F8FC40214A8F
:1057E00044F08074C1F8FC40A2FB03420024920CF8
:1057F000C5F8D0241C4AC0F8B02F1C4A4460A2FB54
:10580000032302689B0942F00102013B0260B3F1ED
:10581000807F08D24FF0E022F0205361072381F807
:105820002300946113614FF0E022136943F00403F5
:10583000136105B030BD00210DF0F0FD0C4B1A686E
:1058400082F308885B689847FEE700BF00ED00E040
:105850000003FA0500440258602B002400000024D5
:10586000001000E083DE1B4355CEACC5D34D621063
:105870000098F01F2DE9F041384E984606EB800362
:10588000D3F81441002C66D004F1CA0306F59A76C9
:105890000546B4F8CA02A36104F5E57366601746CD
:1058A000E3614FF48073261DE160C4E9043323688B
:1058B000C4F8C430A36300284AD194F8C9000DF09D
:1058C000DFFA18F0080F36D1BA0794F8C88023D44D
:1058D000FB0711D4052194F8CE0267F0BFFB94F8C2
:1058E000CE3201221E4903F01F005B09824041F8BD
:1058F00023203046BDE8F081013540460DF0C0FA66
:10590000EDB218B140F206630572C38094F8CC2260
:1059100002210DF08FFADDE76B1CDBB218B10372C8
:1059200040F20653C38094F8CD2202210DF082FA92
:10593000FB07CFD5E0E70135EDB218B140F20673B1
:105940000572C38094F8CD2202210DF073FAC1E7ED
:1059500067F08AF9B1E72646CBE700BF38B10B08FC
:1059600000E100E00148FBF7DBBA00BFF8030024C8
:105970000148FBF7D5BA00BFC80600240148FBF771
:10598000CFBA00BF980900240148FBF7C9BA00BF8D
:10599000680C00240148FBF7C3BA00BF380F00248D
:1059A0000148FBF7BDBA00BF081200240148FBF70D
:1059B000B7BA00BFD8140024426B2421002370B56D
:1059C000C0F8B41004461168806804F1340521F071
:1059D00001011160136053609360A179A063880294
:1059E000C4F8BC3084F8B03000F48050C4F8B4304F
:1059F000E364E0630803C4F8B83000F40050636562
:105A0000A36420640802637900F4806013F0010647
:105A1000606401D00420A06413F0020303D0A06CE2
:105A200040F00800A064C80709D5002E65D13BB33B
:105A3000E36D43F00103E3654FF400332366090788
:105A400020D52423D4F8B4102846C4F8B430136801
:105A500023F001031360FCF75DF8012833D0E36DF8
:105A6000002B56D1636B28465A6822F490425A6044
:105A70009A6822F022029A609A6842F008021BE0BB
:105A80000B07DED42423D4F8B4102846C4F8B4306D
:105A9000136823F001031360FCF73CF8012812D0CF
:105AA000E36D002B31D1636B28465A6822F4904293
:105AB0005A609A6822F02A029A601A6842F001023B
:105AC0001A606AF0B7F86279D5070DD5D4F8C030FE
:105AD000196841F480711960996841F00101996079
:105AE000196841F020011960900705D5D4F8C0204D
:105AF000136843F08003136070BDE06D40F0020056
:105B0000E0654FF48030606691E72846FBF72CF99A
:105B1000C9E72846FBF728F9A4E700BF81604BE7F7
:105B2000417149E70120704738B5134C41F20D131C
:105B3000124941F28832D4F81855D4F8D4042D040F
:105B40008560C56829400B430D21C360FDF7B6FB96
:105B500038B1D4F80825034600201343C4F80835AB
:105B600038BDD4F8D4345869C0F34320A0F1040000
:105B7000B0FA80F0400938BD602B0024C0E0FEFF81
:105B80002DE9F047B74C7C22002198B004F2D440B4
:105B900073F074FAD4F850154FF480524FF48043E8
:105BA00008684FF40031C4F8DC240122C4F8E03462
:105BB00094F80435C4F8D404C4F8E414C4F8E82410
:105BC000002B50D00322A84BA84984F80425426832
:105BD000134043F0FA034360036843F00303036098
:105BE000CB6CDE0340F1BC8008A8FBF717FE0A9AD5
:105BF0009F4BD4F8D404A3FB02135B09B2F5FA7FE0
:105C0000C0F0FD809B4A2168B2FBF3F202322368A8
:105C10005B1A9A42FBD80022974B98490292826005
:105C2000C2680D681340924AA2FB052541F28832F2
:105C300043F480536D0AC36002FB05F52B4603E075
:105C4000426B110600F1E180013BF9D24FF00043B5
:105C5000012084F80405D4F808251343C4F8083556
:105C600018B0BDE8F087864B98425DD0854B9842CE
:105C700000F0128194F85C050DF002F9824694F868
:105C80005E050DF0FDF8814694F854050DF0F8F826
:105C9000804694F856050DF0F3F8074694F8580539
:105CA0000DF0EEF8064694F85A050DF0E9F894F870
:105CB0005D2505460E2150460DF0BCF8484694F887
:105CC0005F250E210DF0B6F8404694F855250E21BB
:105CD0000DF0B0F894F8572538460E210DF0AAF8CB
:105CE00094F859250E2130460DF0A4F894F85B2560
:105CF0000E2128460DF09EF8D4F850350021B3F956
:105D0000040067F0ABF9D4F85035B3F90430002B38
:105D100007DB03F01F0001225B095B49824041F869
:105D20002320D4F8D4044DE7504BD3F8D42022F4E8
:105D30008032C3F8D420DA6F42F48032DA67DA6F47
:105D400022F48032DA67D3F8D42042F48032C3F8E8
:105D5000D420D3F8D43003F480330193019B89E736
:105D60008A6A8E6ACF6A16F47C7F4D6BC6F3051380
:105D700045D0C5F3CC0507F0010702F0030207FB8D
:105D800005F5012A07EE905AF8EEE76A05D0022AD7
:105D900000F0B484002A00F08C8407EE903A9FED66
:105DA0003B5AF8EEE77A0B6B85EE277ADFED385A2F
:105DB000C3F3080307EE903AB7EE006AF8EEE77A0D
:105DC000E6EEA57A77EE867A27EE277A2749F7EE70
:105DD000007A274B0A6B0A6B096BC2F3064206EE88
:105DE000902AF8EEE66A76EEA76AC7EE267AFCEE0F
:105DF000E77A17EE902AA3FB02135B09FEE62268FE
:105E000023689B1A022BFBD905E7224A4FF4D5736E
:105E10006E1E82638360184AC3681A4041F20813F9
:105E20001343C3604DB13346426B013B12F0450F43
:105E300001D0970450D55A1CF6D10023C4F8103570
:105E400083600D4BC268134043F48053C3602B46FC
:105E500003E0426B170600F1D383013BFFF4F6AE7B
:105E6000F7E700BF602B0024002CC0FF004402585D
:105E7000D34D621010210100C0E0FEFF000000249D
:105E8000007000520024024800E100E00024744A3F
:105E900000000039C5002000684BD3F8DC2022F454
:105EA0000072C3F8DC20D3F8842042F40072C3F8F7
:105EB0008420D3F8842022F40072C3F88420D3F81D
:105EC000DC2042F40072C3F8DC20D3F8DC3003F4A9
:105ED00000730093009BCDE6436B590700F11F84CC
:105EE000436BDA0700F11784436B5B0601D540234F
:105EF00083630123524A3721C4F81035002383609D
:105F0000C3681A4041F23713134341F28832C36029
:105F1000FDF7D4F998BB029A4FF6FE739A4200F24D
:105F20009580D4F8D404DFF81891464FDFF8188133
:105F300000233721836041F23713C26802EA090265
:105F4000134341F28832C360FDF7B8F903460028D5
:105F50007FF47EAED4F8D40441F229138760C2687E
:105F600002EA09021343C3604DB13346426B013B61
:105F700012F0450F01D0920404D5591CF6D14FF010
:105F8000805365E6436B5B0700F1B281C0F838804F
:105F90004269029B002A03F101030293029B03DB87
:105FA0004FF6FE718B42C3D902994FF6FE739942A8
:105FB00000F27B8357004FD50123C4F80C350368EA
:105FC000990700F09D8100231D4F836041F2023349
:105FD000C2683A401343C360FAF726FF034600281D
:105FE0007FF436AED4F8D404D4F80CC5426900F17D
:105FF0001801BCF1030FC4F840258269C4F8442598
:10600000C269C4F84825026AC4F84C2500F0A5838B
:10601000836041F20313C2683A401343C360002D0A
:106020003FF414AE436B013E13F0450F02D09F04C2
:1060300040F1F782731CF5D108E600BF0044025816
:10604000C0E0FEFF000010C1C5002000029A9A4285
:1060500000F22B83D4F8D40403689A0700F050812F
:10606000D4F80CC5BCF1030FADD1D4F8302500F144
:106070001801D4F834350968090DC4F81415910FC6
:106080008DF82010C2F383618DF82110C2F30161F5
:106090008DF82210C2F307418DF82310C2F30721B7
:1060A000D2B28DF824108DF825201A0DADF82620D7
:1060B000C3F303428DF82820C3F3C0328DF82920A2
:1060C000C3F380328DF82A20C3F340328DF82B20A1
:1060D000C3F300328DF82C2000228DF82D20BCF166
:1060E000000F40F0748240F6FC71D4F8382501EAC4
:1060F0008303C2F3C26143EA92730C93C2F3425327
:106100008DF83410C2F302618DF83510C2F382416C
:106110008DF83630C2F3C2338DF837108DF8383031
:106120000C9B9DF83810013301F00701023103FA8E
:1061300001F19DF8283003F00F050123C4F81C1568
:10614000AB40C4F820355B0A01FB03F34FF4007148
:10615000C4F82435C4F82815C2F38031D4F83C358E
:10616000D4F818558DF83910C2F3C61102F07F0229
:106170002D048DF83A10D90F8DF83B208DF83C1086
:10618000C3F34171C04E8DF83D10C3F382618DF8A9
:106190003E10C3F383518DF83F10C3F340518DF887
:1061A000401000218DF84110C3F300418DF84210DA
:1061B000C3F3C0318DF84310C3F380318DF8441020
:1061C000C3F340318DF84510C3F300318DF846100C
:1061D000C3F381218DF84710C3F30121C3F34603B4
:1061E0008DF8481001218DF8493041F207138DF8E0
:1061F0004A1007218560C2683240134341F2883259
:10620000C360FDF75BF8034600287FF421ADD4F8A6
:10621000D43425685A69900167D4402741F210129E
:1062200018469F60D96831400A431021DA6041F274
:106230008832FDF743F8002843D1D4F818353721C8
:10624000D4F8D4041B04836041F23713C26832408F
:10625000134341F28832C360FDF730F888BBD4F8AD
:10626000D4344FF0FF3241F20D115A629F62DA6A64
:1062700022F0FF0242F06302DA6298601846DA68A0
:10628000164041F288323143D9600D21FDF716F8EE
:10629000B8B9D4F8D43408A803E02268521B0132FC
:1062A0002BD05A6B12F4957F5A6B2CD11104F4D574
:1062B00000F12001D3F8802040F8042B8142F9D16D
:1062C000EBE7D4F80825D4F8D434C4F808256F4A8D
:1062D00001219A63D4F8082502430846C4F808252A
:1062E00084F8041518B0BDE8F0874FF40060EEE7BD
:1062F00004224FF080538263AAE44FF00040E6E7A7
:106300004FF08063A4E4120700F111825A6B9707E3
:1063100000F10F825A6B960608D50FE2D3F8802061
:1063200040F8042B2268521B0132E6D05E6B16F453
:106330008056F3D1564A9A6308980999DDE90A72A2
:1063400091FA81FC010A3D0C21F0FF015FFA82FE07
:1063500025F0FF0541EA106145EA0E05C0F3811EF4
:1063600089B2C0F340108DF80CE08DF80D00ADF847
:106370000E10F9B2CDF810C08DF81410C7F3072134
:10638000D4F80C058DF81510C7F3035101288DF8CA
:106390001610C2F38521ADF818508DF81A10C2F30B
:1063A00001218DF81B10C2F3031102F00F028DF8CA
:1063B0001C108DF81D209DF833208DF81E209DF8AF
:1063C0001C20D1B29DF81D20D2B270D00322D4F887
:1063D000E054C4F82C65904284F8042575D1D4F8B3
:1063E000082542F08052C4F80825D4F80825002A70
:1063F00079D1D4F8E864D4F8D824032ED4F8DC0496
:10640000D4F8E41409D8D4F82C75B7F5007F04D07B
:10641000B7F5807F0CBF02260426024358680A4362
:106420001C492A4301400A43012132435A6084F83F
:106430000415256803E023685B1B01335CD066F01C
:1064400065FC0428F7D100220120D4F80C35C4F8EB
:106450000825C4F8002584F80405FBB183427FF4C5
:10646000FFAB022384F860350B4CA4F134030FCB4F
:1064700084E80F00A4F1240310340FCB84E80F004C
:10648000002018B0BDE8F087C0E0FEFFFF0FE01F5E
:106490003A0F0018002CC0FFC4300024D4F8103587
:1064A000002BDFD0012BDDD018B0BDE8F0870A4308
:1064B000D4F8E0544FF0030114BF4FF400724FF4CE
:1064C000807284F80415C4F82C25B5F5004F86D0E9
:1064D000B5F5804F50D0CDB1D4F8082542F0006218
:1064E000C4F8082581E701229E491046996384F883
:1064F000042518B0BDE8F08701234FF0004218468C
:10650000C4F8082584F80435FFF7AABBCDE908557F
:106510005A69920158D408A866F01AFC20BB099B5E
:10652000DB0340F1F380D4F818353721D4F8D404D4
:106530001B048D4E836041F23713C268324013430F
:1065400041F28832C360FCF7B9FE68B9D4F8D404CC
:106550008560C26841F2061306213240134341F2BE
:106560008832C360FCF7AAFED4F8D434D4F80825E6
:106570001043C4F8080538E70022CDE908225A691B
:10658000900121D408A866F0E3FB0028ECD1099B18
:10659000590340F1BB80D4F818353721D4F8D4041E
:1065A0001B04714E836041F23713C26832401343BB
:1065B00041F28832C360FCF781FE0028D4D1D4F8C0
:1065C000D40402238360C4E74FF40060CEE7BCF13B
:1065D000010F18D11B04D4F838254FF4007103F4CF
:1065E0007C13C4F8201543EA1243C4F828150C9311
:1065F0000C9B01339B02C4F81C35C4F82435ABE571
:106600005A4B836387E4574A4FF0805301218263DA
:10661000D4F808251A43C4F8082584F80415FFF7B0
:1066200017BB436B5E0700F18F80436B13F00103D0
:1066300040F086800369DBB2032B7CD14B4B836334
:10664000436913F4604F0BD05D0400F1828013F4B2
:10665000004F14BF4FF480534FF48033FFF7F8BA64
:106660001B0C414941F209321D04C4F818358560FC
:10667000C36819400A43C260FAF7D6FB03460028F4
:106680007FF4E6AAD4F8D404D4F80CC5426900F12A
:106690001801C4F830258369C4F83435C569C4F8D5
:1066A0003855056AC4F83C55E5E44FF08073FFF7B0
:1066B000CFBA0A6807EE903A9506F8EEE77A32D537
:1066C0000D68F7EE005A0B6B294AC5F3C101C3F3FD
:1066D00008039FED285ACA4007EE103A06EE102A2A
:1066E000B8EEC77AB8EEC66AA6EE857AC6EE276A15
:1066F00037EE257A27EE267AFFF768BB07EE903A49
:106700009FED1D5AF8EEE77AFFF74DBBD4F8D4346D
:106710004FF080602AE701238363FFF78EBB0423D9
:106720008363FFF78ABB9FED155AFFF73CBB082038
:10673000CDE50220CBE50123FFF78ABA2020C6E58C
:1067400001228263FFF784BA042213468263FFF7B3
:106750007FBA4FF40053FFF77BBAD4F83025D4F852
:10676000343588E4FF0FE01FC0E0FEFFC5002000C5
:106770000090D0030000003920BCBE4B0024744CB4
:10678000C94BD3F86415D3F8682570B58C0FC2F3E4
:10679000072C100E83F89045C1F38364000183F841
:1067A0009145C1F3016483F89245C1F3074483F82E
:1067B0009345C1F30724C9B283F89445C2F3035447
:1067C00083F89515A3F89605C2F3C030B3F8961573
:1067D00089B22143C2F30344A3F89615C2F34031B2
:1067E00083F89845C2F3803483F89905002083F834
:1067F0009A4583F89B15C2F3003183F89C1593F8F2
:10680000601583F89D05012940F2F380022900F00C
:10681000C580D3F86C152A204FEA4C0C83F8A945A3
:10682000C1F3C01201F07F010CF07E0C83F8AAC501
:106830004FF0010C93F8AA451443D3F8702583F860
:10684000AA45D40F83F8AB15910D83F8AC45C2F37C
:10685000417401F00C01C2F3815583F8AD45C2F3D8
:10686000826483F8AE4583F8AF1593F8AF15D3F87B
:106870007445294383F8AF15C2F3405183F8B0152E
:10688000002183F8B115C2F3004183F8B215C2F3B9
:10689000C03183F8B315C2F3803183F8B415C2F365
:1068A000403183F8B515C2F3003183F8B615C2F351
:1068B000812183F8B715C2F30121C2F3460283F8A0
:1068C000B815C4F3074183F8B925220E090283F8ED
:1068D000BAC583F8BC25C4F30722A3F8BE15240665
:1068E000B3F8BE1589B21143A3F8BE15D3F87815D5
:1068F000C3F8C0450C0ED3F8C02542EA0442C3F8E1
:10690000C0250A0AD3F8C04502F47F422243C1F3EE
:106910000724C9B2C3F8C025D3F8C055D3F87C25E5
:106920002C43C3F8C04583F8C415110E83F8C51570
:10693000110C0906C3F8C8151102D3F8C8450A4658
:1069400001F47F01214392B2D3F88045C3F8C81502
:10695000D3F8C8150A43C3F8C825C4F30352D3F8C3
:10696000C81541EA1461C3F8C81593F8CC15114352
:10697000C4F3072283F8CC15210A01F47061A3F84F
:10698000CE15B3F8CE1589B21143C4F34602A3F86D
:10699000CE1583F8D02583F8D1C570BD1204D3F885
:1069A0006C1502F47C12C1F3072CC3F8A0250A0E63
:1069B000D3F8A04544EA0224C1F30742C3F8A04536
:1069C000D3F8A04522434FF40074C3F8A025D3F8B0
:1069D000A025C3F8E045013240F10004A40244EAD6
:1069E00092549202C3F8DC45C1F38034C3F8D82531
:1069F00012E74FEA8C2CD3F86C1592004FF0010E81
:106A00000CF44064C1F3C26502F47F72C1F3072C39
:106A1000C3F8A045D3F8A0452243CC0BC3F8A0256A
:106A200004F00602D3F8A04544EA9174C3F8A045E7
:106A3000C1F3026483F8A45583F8A545C1F3425419
:106A400083F8A645C1F3824483F8A745C1F3C03457
:106A500083F8A82593F8A825224383F8A825D3F81E
:106A6000A04593F8A82593F8985502320EFA05F53B
:106A70000EFA02F2C3F8E055D617A2FB052E05FB6D
:106A800006EE04FB0EEE0134A2FB0424A644520AD7
:106A9000C1F3803442EACE52C3F8D8254FEA5E22D1
:106AA000C3F8DC25B8E600BF602B002465F02ABFE0
:106AB00065F028BF704700BF704700BF014B1868E2
:106AC000704700BF60310024044B93F8A002A0F18E
:106AD0000300B0FA80F04009704700BF6031002425
:106AE000012380F849307047064BD3E9B602431EB4
:106AF0009042A3EB02038CBF0020012003EB003087
:106B0000704700BF6031002401F00F01D0F8D0229F
:106B1000C1EBC10102EB8102D0E9AE30D2F8142200
:106B200003F5037110B5C468D3F80402C3F80C224E
:106B3000A047002010BD00BFD0F8BC3283B110B513
:106B4000D0F8B84294F80002FF2807D09B6821468D
:106B500094F801229847FF2384F80032002010BDEA
:106B6000002070470346432201481A80704700BF47
:106B7000A41700240346432201481A80704700BF2F
:106B8000E81700240346432201481A80704700BFDB
:106B90002C18002403460A2201481A80704700BFBF
:106BA00070180024064B4FF0120C064A506803F18F
:106BB0001402A1F800C002280CBF18461046704706
:106BC0007C18002450400058042301480B80704773
:106BD000A4180024214BD3F80028D3F8080830B5B6
:106BE00012184FF01A040C8001D11D4830BD1C4909
:106BF0004FF0000ED3F804088C467546130FB2F11F
:106C0000204F0EF1020E8CF8035003F1300403F113
:106C100037034FEA02120CF1020C34BF8CF800402B
:106C20008CF80030BEF1100FE8D100221446030F9B
:106C3000B0F1204F02F10202CC7403F1300C03F1E9
:106C400037034FEA001001F1020134BF81F810C090
:106C50000B74082AEBD1024830BD00BF00E0F11FE1
:106C6000A818002400207047212810B505D022283C
:106C700030D0202814D0002010BD0029FBD0072AD6
:106C8000F9D11B4B93F82401D3F8204193F8252127
:106C900093F82631087100200C604A718B7110BD89
:106CA0000029E8D0072AE6D1114B0C79114A08686F
:106CB00083F82441D2F8E0224C798979C3F8200185
:106CC00083F8254183F82611002AD4D001460020FC
:106CD0009047D0E70029CED0022ACCD1054BD3F87B
:106CE000E432002BC7D0098800209847C3E700BFD3
:106CF000A417002460310024034B93F80C030038E0
:106D000018BF0120704700BF60310024034B93F887
:106D10000C03032894BF0020012070476031002439
:106D20000048704770340024174B002030B493F8AB
:106D30002A4014B1DD698D4205D001301033082896
:106D4000F5D130BC7047114BA2B1D3F8581301EB09
:106D500040218A4201D1022C05D093F8F82472B167
:106D6000012283F8412303EB0013012283F86A23F5
:106D700030BC704703EB001080F86A23E1E7012282
:106D800083F8F824ECE700BFA0340024603100242D
:106D9000002330B4194C04F5507084F8E43303E058
:106DA00001331030082B1CD0C5698D42F8D190F802
:106DB0002AC0BCF1030FF3D1AAB1D4F8581301EBE8
:106DC00043218A4208D094F8F82412B9012284F8A9
:106DD000F824012284F8412304EB0313012283F8F1
:106DE0006A2330BC7047D4F8E02304EB031304217A
:106DF000013283F86A13C4F8E023F2E7603100241B
:106E0000C0B1836823B10F4B072283F84223704738
:106E10000C4A042192F8400382F85433032882F884
:106E20004213C2E9D3330CBF80234FF48073C2E90D
:106E3000D1337047034B012283F8F82483F84123B0
:106E4000704700BF603100240346202201481A80A9
:106E5000704700BFCC1800240346202201481A8046
:106E6000704700BFEC1800240346202201481A8016
:106E7000704700BF0C19002403460A2201481A80FB
:106E8000704700BF2C19002410B50F4B0F4C03F5B1
:106E9000CA72D3F89431D4F88C18B4F89008C4F8B6
:106EA00028298861984702E01B69984720B9D4F8DF
:106EB0002839002BF8D1FEE7B4F890380020D4F838
:106EC0008C281B04936110BDA4170024603100249A
:106ED00038B5084BD3F8283953B1DB6914460D4651
:106EE00098474FF40073026800202A60238038BD61
:106EF0001B68FFDE6031002408B5074BD3F8283942
:106F000033B11B69984780F00100404240B208BD90
:106F10004FF0FF3008BD00BF6031002400207047F3
:106F20002DE9F041164C1646B4F89C28D4F8980880
:106F30001504856103B30F4603EB060806E0002342
:106F40004D68304639461A46A84738B9D4F828194A
:106F50000029F4D1FEE71B69984720B9D4F82839F5
:106F6000002BF8D1FEE7013607F50077B045EDD1EB
:106F7000D4F89808B4F89C2882610020BDE8F0811C
:106F8000603100242DE9F041194C1646B4F89C28D4
:106F9000D4F89808150485612BB30F4603EB060857
:106FA00001E00B699847D4F8281951B10023CD6846
:106FB000304639461A46A847D4F8281908B100299E
:106FC000EFD131B10B69984720B9D4F828190029BD
:106FD000F8D1FEE7013607F50077B045E3D1D4F8E4
:106FE0009808B4F89C2882610020BDE8F08100BFB9
:106FF0006031002400207047214938B50A68D1F873
:107000002C3953B1002AFCD0013A13F8014B0A6025
:10701000C1F82C3912B1204638BDFEE7D1F8BC02C8
:107020000028F8D00D7DD1F8D432D0F80402ADB9E3
:107030001A690121C3F830524FF40075012AA3F8F0
:107040001812C3F8240203F50671C3F82C5214D0A9
:107050001868D2B268F0D4FB204638BDC3F830229D
:1070600001211A694025A3F8181203F50671012AB7
:10707000C3F82402C3F82C52EAD1C3F82802E7E788
:1070800060310024D0F8B82270B5002A3CD001EB62
:10709000810300EB8303DC692CB900231C46C2F892
:1070A0001432204670BDD0F8D062C1EBC10506EBAA
:1070B00085056D6CB4FBF5FC05FB1C45002DECD182
:1070C000DD6101F07F0301F00F04012203EB830374
:1070D0001C2100EB830001FB0461C4EBC403C56108
:1070E0003C3106EB83039D6483F83C4083F83D20EC
:1070F000C3E914553269012AD2B208BFDD64306891
:107100002CB968F073FCCCE70224204670BD002443
:1071100068F076FBC5E700BF1D4B0A68C3F82C0971
:107120001A600AB100207047D3F8BC120029F9D0C8
:1071300010B5187DD3F8D432B0B14024D1F8040290
:107140000121C3F82402A3F8181203F50671C3E95C
:107150008B421A69012A08BFC3F828021868D2B204
:1071600068F04EFB002010BD4FF40072D1F80442CD
:107170000121C3F82442A3F8181203F50671C3E9EC
:107180008B201A69012AE9D1C3F82842E6E700BF3B
:107190006031002470B50022D0F8C84205461C4B6F
:1071A00084F838120D2684F8082204F50B70C4F810
:1071B0002C3204F50374D5F8D0322E631A6740F2EE
:1071C000011203F15801DE66A3F858201A695866C7
:1071D000012AD2B208BF9866186868F011FBD5F88A
:1071E000D0321F2000220121C3F82442C3E98B02C0
:1071F0001A69A3F818128A421868D2B203F5067108
:1072000008BFC3F82842BDE8704068F0F9BA00BF73
:10721000555342532DE9F047137882B09146044606
:107220008A465A2B5CD8DFE813F0E4005B005B0071
:107230007F005B005B005B005B005B005B005B0052
:107240005B005B005B005B005B005B005B00CA00F7
:107250005B005B005B005B005B005B005B00B00001
:1072600075005B005B0075005B005B005B005B0012
:10727000E0015B0006025B005B0064015B00F7005D
:107280005B005B005B005B0050015B005B005B0030
:107290005B005B005B005B005B005B005B005B0016
:1072A0005B005B005B005B005B005B005B005B0006
:1072B0005B005B005B005B005B005B005B005B00F6
:1072C0005B005B005B005B005B005B005B005B00E6
:1072D0005B005B005B005B005B005B005B00260209
:1072E000D0F8C822052400204FF0FF3592F85D3217
:1072F00002EBC3010133DBB281F83C4281F840026A
:10730000042B14BF82F85D3282F85D02284602B079
:10731000BDE8F0870023D0F8C8221D46A2F80A3243
:10732000284602B0BDE8F087D0F8C83270240020AB
:107330000C21186058601C70D97193F85D4293F865
:107340005C1298608C42D860188213D003EBC104A1
:10735000013194F83C52C9B29D70042994F841520D
:107360001D7394F8404218BF83F85C125C7308BF29
:1073700083F85C021221A3F80A1299F804208A42C9
:1073800018D80025A3F80A22C0E7D0F8C8020823BD
:107390000022D24DC11D4442A0F80A3200E0127A08
:1073A0000B46814203F8012904EB0302194615FA42
:1073B00082F2F4D10025284602B0BDE8F08799F8A2
:1073C0000130D0F8C802DB0740F16B810723811D33
:1073D0008322C24D4442A0F80A3200E0AA5C0B4668
:1073E000884203F8012904EB0302194692B2F5D151
:1073F000E0E7D0F8C862D6F81472002F40F05D8242
:10740000D0F8CC3208469B6898470546002840F0E3
:107410008C82A6F80A0279E7D0F8C86296F808824A
:10742000B8F1000F40F0718196F91832002BC0F2CC
:10743000D782D0F8CC3208469B6898470746002888
:1074400040F0A482D4F8CC325046DB689847054619
:10745000002840F00982D9F80210D4F8C80209BA0D
:10746000D0F86022C6F86412B9F807305BBA9BB254
:107470001944C6F86832914200F29D82B6F85E2245
:1074800002FB03F3D6F81422934240F091810121CC
:10749000B3F5007F86F8081228BF4FF40073D4F8C4
:1074A000D0020269C0F82C32012AC0F82462C0F868
:1074B0003052D2B2A0F8181200F5067108BFC0F819
:1074C0002862006868F09CF920E799F80130D0F84C
:1074D000C82213F0020340F07B81D2F86002D2E9A7
:1074E00099142144814200F20D821D46A2F80A320D
:1074F0000CE7D0F8C87297F80862002E40F00381BC
:1075000097F91832002B80F2EB81D0F8CC32084684
:107510009B6898470546002840F0E280D9F80200B1
:10752000D4F8C86200BAD6F86022C7F86402B9F885
:1075300007305BBA9BB21844C7F86832904200F239
:107540008181B7F85E2202FB03F3022287F808224A
:10755000D7F814229A4240F075814FF40073D4F8A2
:10756000CC2250463146A7F80A32B6F85E32D6F839
:107570006872156903FB07F7D6F86422B7F5007F38
:1075800028BF4FF40077B7FBF3F39BB2A84700285E
:10759000C0F27E81D4F8D03200222763186803F14C
:1075A00058015E66C3E91B7240F20112A3F858202D
:1075B0001A69012AD2B208BF9E6668F021F9B6F8AE
:1075C0005E02B7FBF0F0D6E999351A18D6F83432D6
:1075D0002D1ADB1BC6E99925C6F83432002D7FF43D
:1075E000E9AE032386F8083290E6D0F8C8520026A8
:1075F00008460DF102022E6001A96E60AE60D4F85B
:10760000CC325B689847002840F0098108200223AB
:10761000BDF802200C21E8702B8152BA019BA5F81D
:107620000A12013B6A81180EEB71190C1A0A2871B3
:107630006971AA71BEE6D0E9B26308465B6806F2DA
:107640005E2206F5187198470546002840F0D28062
:10765000D6F860320821B6F85E22013BA6F80A127D
:1076600052BAB080190EF370F2801A0C1B0A3170F6
:107670007270B3704AE6D0F8C80208230022174D92
:10768000C11D4442A0F80A3200E0127C0B46884239
:1076900003F8012904EB0302194615FA82F2F4D12A
:1076A00088E6D4F8CC4201EBC10199F80430E469D2
:1076B00004EB810422790532934228BF1346A0F8D7
:1076C0000A32002B3FF476AEE218034412F8011D93
:1076D000A24203F8011DF9D16CE600BFC0B20B084D
:1076E000D4F8C822022092F85D3202EBC3010133C4
:1076F000DBB281F83C0281F84062042B00F0838108
:1077000082F85D3256E63E4627E7B6F85E32084616
:10771000D6F868523146D4F8CC2203FB05F55769F8
:10772000B5F5007FD6F8642228BF4FF40075B5FB8D
:10773000F3F39BB2B8470028C0F21281B6F85E326C
:10774000D6F86422D6F86812B5FBF3F00244091AA1
:10775000C6F86422D6F83422C6F86812521BC6F85E
:10776000342221B920460D46FFF714FDCEE5D4F8AA
:10777000D00201FB03F301220021B3F5007FC0F822
:107780002462A0F818224FF00005026928BF4FF4C8
:107790000073C0F8301200F50671012AC0F82C32CF
:1077A000D2B208BFC0F82862006868F029F8ADE5D9
:1077B00090F85D3205215A1C00EBC303D2B283F866
:1077C0003C1283F84052042A74D080F85D22F1E51F
:1077D00092F85D3205240020591C02EBC303C9B2A4
:1077E00083F83C4283F84002042900F0CB8082F801
:1077F0005D12DFE5D4F8C8220021022492F85D3240
:1078000002EBC3000133DBB280F83C4280F8401247
:10781000042B7FF475AF0D4682F85D1276E5D4F83F
:10782000C822022092F85D3202EBC3010133DBB2C1
:1078300081F83C0281F84062042B7FF461AF82F84A
:107840005D62B7E596F85D3205211A460133DBB279
:1078500006EBC202042B82F83C1282F8405200F080
:10786000BC8086F85D32A5E5D4F8C822022092F8E3
:107870005D3202EBC3010133DBB281F83C0281F8D7
:107880004072042B7FF43CAF3D4682F85D723DE5CB
:10789000D4F8C8220424002192F85D3202EBC30020
:1078A0000133DBB280F83C4280F84012A3427FF4FF
:1078B00027AFB0E780F85D5228E596F85D320520E5
:1078C00000211A460133DBB206EBC202042B82F818
:1078D0003C0282F84012C4D10D4686F85D1215E5CF
:1078E00097F85D3205211A460133DBB207EBC2027D
:1078F000042B82F83C1282F8406200F0888087F8FE
:107900005D3257E592F85D12052408460131C9B28F
:1079100002EBC000042980F83C4280F840327FF43A
:1079200066AF1D4682F85D32F0E4D4F8C82202202A
:10793000002592F85D3219460133DBB202EBC1013A
:10794000042B81F8407281F83C0218BF82F85D3246
:107950004FF0050308BF82F85D7286F80832D5E45F
:10796000D4F8C8220424002092F85D32194601336D
:10797000DBB202EBC101A34281F83C4281F8400234
:107980007FF4BEAE054682F85D02BFE4D4F8C8229B
:10799000022092F85D3219460133DBB202EBC101DD
:1079A000042B81F83C0281F840827FF4A9AE454661
:1079B00082F85D82AAE490F85D3205211A4601330F
:1079C000DBB200EBC202042B82F83C1282F8405278
:1079D0003FF470AF80F85D32ECE486F85D5295E4D8
:1079E00096F85D3205211A460133DBB206EBC2027E
:1079F000042B82F83C1282F840827FF432AF454675
:107A000086F85D8282E4354682F85D627EE4354622
:107A100087F85D627AE400BFD0F8C81210B591F81B
:107A20000832022B07D0033B012B02D80021FFF7BD
:107A3000B1FB002010BD01F21B2291F8191204467F
:107A4000FFF7E8FB0028F4DA01212046FFF7A2FB4C
:107A5000EFE700BFF8B5037C0446002B4BD14FF491
:107A6000007302228121D0F8D00267F0D5FD0125F4
:107A70004FF4007329460222D4F8D0020127E562B0
:107A800067F0CAFD082303228221D4F8D002C4F88B
:107A90006C5167F0C1FD4FF40770276471F0DEFA96
:107AA0000546C4F8B802002846D0D4F8BC321B689A
:107AB00098470022267CC5F81422D4F8D032D5F895
:107AC0000402C5F8182206B3C3F8302240241A690C
:107AD00003F50671C3F824020026012AA3F81872E0
:107AE000D2B2C3F82C4208BFC3F82802186867F066
:107AF00087FE3046F8BD402302228121D0F8D00213
:107B000067F08AFD01254023B4E71A694FF4007439
:107B1000C3F8240203F50671BA42A3F81872D2B270
:107B2000C3F8306208BFC3F82802C3F82C421868B3
:107B300067F066FE3046F8BD3E46DAE738B5037CAE
:107B40000446002B55D14FF4007302220121D0F8D6
:107B5000D00267F061FD01254FF40073D4F8D00224
:107B600002228121C4F86C5167F056FD264B00209B
:107B7000D4F8CC1203F51462E562A3F8480BA3F81D
:107B80009C0B0B68C4F8C8229847D4F8D04294F8EC
:107B9000BC332068012B14D010221C4B026101E081
:107BA000013B02D00269D106FAD46022174B026170
:107BB00001E0013B02D002699206FAD4002384F866
:107BC000BC330022124B1F2504F50671C4F8302285
:107BD0000122C4F82C52A4F818222269C4F82432D5
:107BE000012AD2B208BFC4F8283267F009FE00208B
:107BF00038BD402302220121D0F8D00267F00CFDED
:107C000001254023AAE700BF60310024400D030096
:107C1000AC3C002470B5D0F8D05240F201120446BA
:107C200095F8BC33A5F85820012B09D0012228680B
:107C3000114685F8BC2367F0BFFF002385F8BC33ED
:107C4000D4F8D05200260121E66295F8BC33A5F89D
:107C500018128B4207D03246286885F8BC1367F0AB
:107C6000ABFF85F8BC63D4F8D05200264FF4817284
:107C7000C4F86C6195F8BC33A5F87420012B08D0CA
:107C800001220221286885F8BC2367F095FF85F85A
:107C9000BC630025D4F8B83225644BB1D4F8BC32AB
:107CA0005B689847D4F8B80271F0E0F9C4F8B852AC
:107CB000002070BD70B5D0F8D0520121044695F86F
:107CC000BC33A5F818128B4208D00022286885F82A
:107CD000BC1367F071FF002385F8BC33D4F8D05291
:107CE000002640F20112C4F86C6195F8BC33A5F887
:107CF0005820012B08D001222868114685F8BC23A2
:107D000067F05AFF85F8BC630025D4F8C802E56225
:107D100071F0ACF92846C4F8C85270BD2DE9F041A5
:107D20000B7882B000270D4613F060060446D0F8A9
:107D3000B8828DF80570ADF806702BD0202E2FD1AB
:107D4000CA88002A3BD01B067CD5D0F8BC324146FD
:107D500068789B6898470223EA884FF48071C4F8DA
:107D60009432D4F8D032C4E907221A651A69998787
:107D700003F13C01012AC3F848805F6501D1C3F8D3
:107D80004C8000261868D2B267F030FE304602B050
:107D9000BDE8F0814B780A2B2ED00B2B4DD0C3B110
:107DA0008021D4F8D00267F0D1FC0021D4F8D002B1
:107DB000022667F0CBFC304602B0BDE8F081D0F877
:107DC000BC32164648789B689847304602B0BDE8FA
:107DD000F08190F89C22032A50D0D4F8D002802160
:107DE000022667F0B3FCD4F8D002002167F0AEFCA5
:107DF000304602B0BDE8F08190F89C32032BECD104
:107E0000D0F8D03201220221C0E90722C0F8941232
:107E10004FF480711A650DF10502998703F13C0159
:107E20009A641A695E65012A02D10DF10500D864D1
:107E3000D2B2186867F0DAFDBDE790F89C32032BE8
:107E4000B9D0CAE74B7888F8012288F800320323BA
:107E5000C0F89432D0F8D032C0E95722C3F81022CB
:107E600003F5FE711A69C3F80882012AC3F8147277
:107E7000A3F8FC7108BFC3F80C8282E7D0F8D002E7
:107E800002220026C4F8942200F13C01C4E9072232
:107E900002654FF48074026943650DF10603012AFF
:107EA00084878364D2B208BFC364006867F09EFD14
:107EB00081E700BFF0B5002383B00E460446ADF85D
:107EC00006300B78D0F8C87213F060053DD0202D35
:107ED0002DD14A78FE2A24D0FF2A28D14A8832BBE5
:107EE000CA8822BB190622D44FF4807307F50370A9
:107EF00001210025A7F80832D4F8D0321F24C3E9A5
:107F00008B421A69C3F82402012AA3F81812D2B2CC
:107F100003F5067108BFC3F82802186867F070FC03
:107F200010E04D881DB9CE88012E00F0E58080213B
:107F3000D4F8D00267F00AFC0021D4F8D002022560
:107F400067F004FC284603B0F0BD4B780B2BEED84D
:107F500001A252F823F000BF997F04081980040899
:107F60002F7F04082F7F04082F7F04082F7F040829
:107F70002F7F04082F7F04082F7F04082F7F040819
:107F8000D97F0408897F040890F89C32032BCED156
:107F90008B78C7F80432D5E790F89C22032AC6D123
:107FA000D0F8D00202221D46C4F8942200F13C0110
:107FB000C4E9072202654FF48072002482870269B7
:107FC00044650DF10604012AD2B2846408BFC4647A
:107FD000006867F00BFDB5E790F89C32032BA6D143
:107FE000D0F8D0320122022107F50177C0F89412AF
:107FF00003F13C01C0E907221A65002218685A659E
:108000004FF480729F649A871A69012AD2B208BF1E
:10801000DF6467F0EBFC95E7D4F8D0728B8897F8B3
:10802000BC23D8B2012A00F0D7804FFA83FE012387
:10803000BEF1000F87F8BC33C0F28180102339688D
:108040000B61684B01E0013B02D00A69D206FAD409
:1080500000F00F000146002387F8BC33C0EBC003DB
:10806000BEF1000F4FEA83037DDBFA184FF0000CDE
:1080700003F5FE7382F8FDC182F8FC013B4497F8DA
:10808000BC23012A11D00122386887F8BC23197853
:108090005A7867F091FD002387F8BC3396F90430D5
:1080A000B188002B01F00F016ADB01EB8101002395
:1080B00004EB8101C1F85831237C002B73D14FF4BC
:1080C000007302220121D4F8D00267F0A5FA01233F
:1080D000C4F86C31D4F8C87297F80932022B72D008
:1080E0003279D2093FF42EAF012B3FF42BAF01219F
:1080F0002046FFF74FF825E718067FF518AFD4F8AC
:10810000CC3207F500779B69984702223860D4F893
:10811000D032C4F894224FF4807203F13C01186805
:10812000C4E907669A871A695D650025012A9F647C
:10813000D2B21E6508BFDF6467F058FC02E700F0AA
:108140000F00D7F800C0274B8201014642F0200201
:10815000CCF8102002E0013B3FF47DAFDCF81020AA
:108160009206F8D477E7FA184FF0010C3C3382F806
:108170003DC082F83C003B4497F8BC23624582D165
:1081800001EB8101002304EB81018B61237C93B916
:108190004FF4007302228121D4F8D00267F03CFA38
:1081A0000123E36296E7402302220121D4F8D002A2
:1081B00067F032FA8BE7402302228121D4F8D00203
:1081C00067F02AFAECE78121D4F8D00267F0BEFA12
:1081D000002387F80932B5E600F00F004FFA83FE5E
:1081E00001463BE7400D030038B5D0F8C8520446BD
:1081F00095F8183213B9D5F814324BB98121D4F857
:10820000D00267F0A3FA95F80932022B0AD038BDE4
:1082100095F80932002BF1D10121D0F8D00267F096
:1082200095FAEBE7D4F8D0321F20002205F503754C
:108230000121C3F82452A3F8181203F50671C3E90B
:108240008B021A691868012AD2B208BFC3F82852F3
:10825000BDE8384067F0D4BA70B5D0F8C8420546DA
:1082600094F808625EB1012E07D104F21B2294F843
:108270001912FEF7CFFF002834DB002070BDD4F8C0
:108280001032C4F83032D4F81432C4F83432D0F892
:10829000D032D3F830321F2B08D1364BD4F80C2211
:1082A0009A4203D194F81912012920D994F85D3229
:1082B0000021052004EBC3020133DBB282F83C024B
:1082C00082F840122846042B18BF84F85D324FF024
:1082D000020308BF84F85D1284F80932FFF784FFB7
:1082E000002070BD01212846FEF754FFC5E794F831
:1082F0001A32013B0F2BD9D804F21B22FEF78AFF5A
:10830000002894F808322BDB013B022BB5D9B4F8D6
:108310000A1259B3D5F8C832042283F80822D3F8D8
:10832000342283F83862521AC3F83422D3F8143254
:10833000994228BF1946D5F8D0321A692963012A13
:10834000D96640F20111D2B21868A3F8581003F1AF
:1083500058015C661E6708BF9C6667F051FA8CE79F
:10836000052BBFD02846FFF73FFF86E72846FEF7DC
:1083700011FF82E75553424308B520B9044863F022
:108380007FFF044808BD044863F07AFF014808BD38
:10839000D8500C080C3D0024FC500C08024808B5CD
:1083A00063F06EFF014808BD20510C080C3D00240D
:1083B000024808B563F064FF014808BD28510C0865
:1083C0000C3D0024024808B563F05AFF014808BD7F
:1083D00034510C080C3D0024304B002230481B68FF
:1083E000304910B5304C82B0C4F8BC2CC4F8B42C61
:1083F000A0FB032394F8E92CC4F8AC1C42F20F71E3
:10840000DB0CC4F8B81C013BC4F8B03C002A3FD0D8
:1084100002232649234884F8E93CFAF7C3FE244B9B
:1084200001220621372084F8E92CD3F8E82042F015
:108430002002C3F8E820D3F8E83003F020030193CA
:10844000019B64F00BFED4F8AC3C4FF400001949DA
:10845000194A4860D96841F00101D96099680A4019
:10846000062A06D0B2F5803F03D01A6842F0010216
:108470001A600020D4F8BC321049114AC3F8100227
:10848000C4F8E402C4F8E002C3E9812102B010BDDF
:1084900002F0FF0084F8E80CBAE700BF00000024F7
:1084A00083DE1B430014004060310024103E002492
:1084B0000044025800E100E0070001006852002477
:1084C000684200242DE9F047224E8846D6F8BC3297
:1084D000D3F81422002AFBD1B8F1000F37D000EBFB
:1084E0000809471EDFF870A009F1FF3917F8010FDE
:1084F000D6E9B6314A1C0AF80100C2F30B029A42CF
:10850000A3EB0203C6F8DC2234BF0021012103EBF8
:108510000133012B19D10CF01FFD04460D460CF060
:108520001BFD001B61EB0501B0F57A7F71F10003C3
:10853000F5D3D6E9B6329342A3EB02038CBF0021F8
:10854000012103EB0133012BE5D04F45CED140464D
:10855000BDE8F0876031002468520024F8B50C4E65
:1085600096F8A032032B00D0F8BD0D461446D6F87D
:10857000EC7C08E0FFF7A6FFD6F8EC3C241A054493
:10858000DB1B322BF0D8002C21462846F2DCF8BD4C
:1085900060310024F8B590F848305D1C0344EDB21A
:1085A00080F8485083F8341090F84930012B02D1FC
:1085B000132D00D8F8BD002380F84830002DF9D0E5
:1085C0000B4F97F8A032032BF4D1D7F8EC6C00F1E5
:1085D000340401E0002DEDD029462046FFF772FF5C
:1085E000D7F8EC3C2D1A04449B1B322BF2D9F8BD72
:1085F00060310024F8B5002390F84850A0F84830C6
:1086000005B9F8BD0B4F97F8A032032BF9D1D7F875
:10861000EC6C00F1340401E0002DF2D02946204634
:10862000FFF750FFD7F8EC3C2D1A04449B1B322B6C
:10863000F2D9F8BD6031002408B5FDF7A1FA58B1B0
:108640000E4A92F800330133DBB2072B82F8003375
:1086500003D9002382F80C3308BDD2F8383323B194
:108660001868998803691942F3D0D2F8EC1C0123E9
:10867000C2F8FC1282F80C3308BD00BF6031002440
:1086800010B50D4CD4F8383323B119689A880B69AA
:108690001A4202D0FDF774FA18B1002384F80C33A3
:1086A00010BDD4F8EC2C012384F80003C4F8FC229C
:1086B00084F80C3310BD00BF6031002438B5164C6F
:1086C0000021164D636C20681B04C5F80813144A7A
:1086D0000D218360C3681A4041F20D13134341F228
:1086E0008832C360FAF7EAFD58B1636B18436063E0
:1086F0000922D5F8EC3C002085F80C23C5F8FC32A3
:1087000038BD23685B69C3F34323042BF0D10220F7
:1087100085F80C3338BD00BF3430002460310024AC
:10872000C0E0FEFF70B50E4D04460E4695F80C33C2
:10873000042B0BD0082B07D1D5F8043383420CD07F
:10874000FFF7BCFF022801D0012070BD08230220E2
:10875000C5E9C14685F80C3370BD022070BD00BF6D
:10876000603100242DE9F04706460D4690461F462D
:108770005D4C94F80C1304290CD0082907D1D4F8C7
:108780000433B34206D0FFF799FF0228F1D001204D
:10879000BDE8F08706220123C4F8F48284F80C2394
:1087A000524A84F8F0325362EB06C4F8F872C4E916
:1087B000BA5646D1BFF34F8F4D4A05F500712B468F
:1087C000C2F8683220338B42FAD1BFF34F8FBFF328
:1087D0006F8F002D49D0474F97F83030012B30D1A3
:1087E000731C396D00228B427A6339D803233868B1
:1087F0004FF4007AFD6187F830304FF40073C262A5
:1088000010213B62DFF8F490BB6BC0F808A0C2688F
:10881000012B41F2101302EA090218BF760213433A
:1088200041F28832C360FAF749FD804618B33B68CD
:10883000314A9A630123786B40EA0800786387F82D
:108840003030FFF7F9FED4F8F452002D49D0012062
:10885000D4F8F8320022D4F8EC12A847032097E7A6
:108860007B6B43F000737B63EBE7224A536B43F06F
:1088700000635363E5E738684FF0FF321821426226
:10888000C0F828A0C26A22F0FF0242F09002C26241
:10889000C26842F04002C2609022856501250565EC
:1088A000FA628660C26802EA090941F2181249EACE
:1088B0000202C26041F28832FAF700FD50B13B6813
:1088C0000D4A9A637B6B1843786387F83050C7F87A
:1088D0002C80B6E73A68D36B43F48D73D363BDE85D
:1088E000F087032054E700BF60310024C430002427
:1088F00000ED00E034300024FF0FE01FC0E0FEFF79
:108900002DE9F04F634D1F4683B0064695F80C33B2
:108910000C469046042B09D0082B03D0002003B04E
:10892000BDE8F08FFFF7CAFE0228F7D114F01F024E
:1089300047D101235849C5F8F04CC5F8F83C0B6203
:108940004FF40073C5F8F43C002C48D0DFF854A174
:108950009AF83010012934D1701CDAF85010CAF896
:108960003420884243D8DAF80000CAE909430323D7
:108970008AF83030DAF83830C262012B35D0730211
:1089800001934FF40079454B41F21012C0F8089062
:10899000C16819400A431021C26041F28832FAF7D7
:1089A0008DFC3E4B834648B3DAF800303C4A9A636C
:1089B0000123DAF8340040EA0B00CAF834008AF8E0
:1089C0003030FFF739FED5F8F442002CA6D0002253
:1089D000D5F8F832D5F8EC121046A0479EE7314A98
:1089E000536B43F000635363EBE70196C9E7DAF892
:1089F000343043F00073CAF83430E2E7DAF80000AC
:108A00004FF0FF3211214262C0F828904FF0010967
:108A1000C26A22F0FF0242F09202C262C26842F0D1
:108A20004002C26081228465C0F85090CAF82C20B0
:108A3000019A8260C268134041F211121A43C26067
:108A400041F28832FAF73AFC68B1DAF80030144A99
:108A50009A63DAF834301843CAF834008AF8309050
:108A6000CAF82CB0ADE7DAF8002005234846C5F86F
:108A7000F48285F80C33D36BC5F8F87243F4957320
:108A8000D363D5F8EC3CC5E9BA46C5F8FC3203B06F
:108A9000BDE8F08F60310024C4300024C0E0FEFF48
:108AA000FF0FE01F343000242DE9F0417F4C0226F7
:108AB0007F4F804D94F80C03431E082B45D8DFE808
:108AC00003F052547544C72E16440500FDF72CF8E8
:108AD000002840F0DF80D4F8FC32D4F8EC2CFA33D4
:108AE00093422FD2FFF7A8FD94F80C03E4E7FDF7BB
:108AF0001BF80028EFD0D4F808330022012B84F8AB
:108B0000002340F2CC80D4F80423013B0821013239
:108B1000C4F8083384F80C13C4F8042321E0654B2F
:108B20005B6AEBB90722D4F8EC3CD4F8F45284F831
:108B30000C23C4F8FC329DB1D4F8F8320120D4E9FA
:108B4000BA21A84794F80C03431EDBB2022B70D85D
:108B5000D4F8EC3CD4F8FC229B1AC82B00F2958088
:108B60000020BDE8F08184F80C6364F0CFF804289D
:108B7000E8D1FDF705FE0028E4D13B78002BA3F1F6
:108B80000203B3FA83F314BF022201225B0984F8C3
:108B9000012384F80233FDF7F3FD0028A2D1464BF0
:108BA00003229B6C84F80C23C4F81033FDF7E8FD16
:108BB0000028C7D1404BC4F80803042093F82C10B8
:108BC000DA8D84F81613A4F81423196B1A6B090EA6
:108BD00084F80C03120C84F8171384F818231A6B0A
:108BE000196B120A84F81A1393F8341084F81923B5
:108BF00084F81B1393F8351093F83520C14002F028
:108C00000F0284F8201384F821239A6BDD8FC4F8B7
:108C10001C23DA8FD98FC2F30B1301F00F0243EA42
:108C2000152384F8242303F00F0303F5FA63A4F853
:108C30002233082818BF04280CBF01200020BDE8FB
:108C4000F081D4F8FC32D4F8EC2C6433934287D210
:108C5000D5F82080B8F1000FF3D1FCF765FF0028AC
:108C60003FF428AF0423D4F8F45284F8008384F846
:108C70000C33002D3FF475AFD4F8F8324046D4F8E9
:108C8000E822D4F8EC12A8475CE7FFF7D5FC94F88B
:108C90000C03CEE70423012084F80C3361E7F9D1FB
:108CA000FFF70CFD94F80C03431E4EE760310024DF
:108CB000C0300024C4300024F03000242DE9F843F3
:108CC000354E307A0AF0DCF80546B07A0AF0D8F86A
:108CD000044630780AF0D4F88146B0780AF0D0F82B
:108CE000804630790AF0CCF80746B0790AF0C8F827
:108CF00006461DB10D23EB8000232B721CB10D2302
:108D0000E38000232372B9F1000F05D00D23A9F8E9
:108D10000630002389F80830B8F1000F05D00D2384
:108D2000A8F80630002388F808301FB10D23FB8017
:108D300000233B721EB10D23F3800023337248469B
:108D40000AF04CF8012148460AF04EF840460AF075
:108D500045F838460AF042F830460AF03FF84046F7
:108D600001210AF041F8384601210AF03DF80121BD
:108D700030460AF039F828460AF030F820460AF062
:108D80002DF8284601210AF02FF820460121BDE8E0
:108D9000F8430AF029B800BFB430002410B51C20F5
:108DA0000AF06EF8044611210AF01EF81CB1A388DF
:108DB00022681B049361C8200CF0FCF82046BDE833
:108DC00010400AF00BB800BF2DE9F04F844D87B07A
:108DD000D5F8FC4C636913F0010A02D007B0BDE876
:108DE000F08F6269A3691A42F8D06369A2691340DF
:108DF0009E0703D5636903F0020363616369A26997
:108E000000941340D80612D5A36923F01003A36180
:108E1000236AC3F3434203F00F06022A00F075836E
:108E2000062A00F0DD82A36943F01003A3616369A1
:108E3000A269134019037ED46369A26913405903E0
:108E400000F1B9806269A3691A4257D46369A269C3
:108E500013401F0509D5009BD3F80838DE0700F141
:108E60008C83636903F4006363616369A2691340DF
:108E7000180111D5636903F000636361594B93F8DE
:108E8000F020002A40F03A82012283F8F020626D3F
:108E9000C2F38302C3F8F4206369A2691340D904C2
:108EA00000F1B3816369A26913409B0400F14C8116
:108EB0006369A26913401F0700F114826369A26904
:108EC0001340DE0200F109826369A269134098022F
:108ED00000F1FE816369A2691340590000F1F3813A
:108EE0006369A26913405A077FF578AF6668730714
:108EF00000F1358363681E4366606FE7009B03F5EE
:108F00000062D3F8043823F001035360354B93F823
:108F1000F020012A00F00C82D3F8003193F89C2253
:108F2000042A03D193F89D2283F89C22636903F0FD
:108F3000004363618AE7D4F81868D4F81C381E40EF
:108F4000360C3FF479AFDFF8A09004F530674FF0AE
:108F5000000BCDF804A008E076080BF1010B07F137
:108F6000200709F11C0900F05082F207F4D504F53E
:108F700030625FFA8BFA02EB4A118968D4F8143830
:108F800001EA030818F0010F40F0428218F0080FC0
:108F900040F05A8218F0100F01D01023BB6018F077
:108FA000200F01D02023BB6018F4005FD4D04FF411
:108FB0000053BB60D0E7D4F81838D4F81C2803EA73
:108FC00002081FFA88F8B8F1000F3FF43BAF009B8E
:108FD000054E03F510690023CDF804A09B460FE071
:108FE00060310024604100245C3E00245FEA5808A0
:108FF0000BF1010B06F11C0609F1200900F0828239
:1090000018F0010FF2D05FFA8BFAD4F81028D4F8D8
:10901000347804F510630AF00F0103EB4A13CF40D4
:109020009B68FF01FFB217431F40FA0726D500993E
:109030000BF00F0301229A40D1F8343823EA0203DF
:10904000C1F834380123D5F80C1DC9F8083099420D
:1090500000F09E82B84BD3F80031BAF1000F00F057
:10906000BD82D3F8B422526942B193F89C1203290D
:1090700004D1184651469047D5F8FC4C3B0702D521
:109080000823C9F80830F80602D51023C9F80830BB
:10909000790602D54023C9F80830BA0702D5022361
:1090A000C9F808303B06A1D5D6E9140181429DD804
:1090B000421A736C04EB4B17934207F5106728BFF5
:1090C0001346BA69033392B2B2EB930F2ED30AF16F
:1090D000010A04EB0A3A81422BD2421A736C95F8CA
:1090E0000CED9A4228BF1A46B36C02F1030C4FEA0A
:1090F0009C0CBEF1000F11D11FFA82FE0EF1030E7F
:109100005FEA9E0E0AD003EB8E0053F8041B8342E5
:10911000CAF80010F9D1B36CD6E914011344114414
:10912000B364BB6971659BB29C45D4D98142FFF49D
:109130005DAF0BF00F0301229A40D4F8343823EAD4
:109140000203C4F8343851E7D4F800197B4A0A40C6
:10915000C4F80029D4F8042842F48072C4F8042822
:10916000D4F8083813F0060240F0D280C5F8082D74
:10917000F8F716FBD5F8083DDAB2022A00F0E480D1
:10918000E268B3F1000822F4705218BF4FF00108F2
:10919000E260E36843F41053E360DFF89C914023FE
:1091A00000220126D9F800411F461146D4F8D0020A
:1091B00066F032FA3B4600228021D4F8D002C4F88F
:1091C0005861C4F8647166F027FA00236762C4F836
:1091D00094326360C4F8A432D4F8C832A66184F82B
:1091E0009C62002B00F00B82D4F8B43220460021A0
:1091F0005B689847D9F80031D5F8FC4C83F81080AB
:10920000636903F40053636152E6009B03F5006059
:10921000436823F0010343604FF484632361484BA8
:1092200001E0013B02D022699206FAD4D5F8006D24
:109230001EB3009B4FF67F3103F5106399600AF16E
:10924000010A1A682033B24522F4001243F8202C98
:1092500053F8202C42F0006243F8202CC3F8E811A8
:10926000D3F8E02122F40012C3F8E021D3F8E02182
:1092700042F00062C3F8E021E0D1C36943F001137A
:10928000C361D5F82C3D002B48D0D0F8843043F092
:109290000B03C0F88430436C43F00B034364009924
:1092A0002046284AD1F8003823F4FE63C1F800387C
:1092B00095F80C1D66F020FAD5F8FC4C636903F4B0
:1092C00080536361EEE5636903F08043636107E601
:1092D000636903F400136361FCE5636903F48013BD
:1092E0006361F1E5144BD3F8000190F89C32032B35
:1092F0006DD0636903F008036361DFE5D3F80031E3
:10930000042193F89C2283F89C1283F89D22C3E5E4
:1093100013F0020F14BF02220F2227E7426942F224
:109320002B0313434361036943F00B030361B6E767
:10933000002283F8F020F9E56041002400F8FFFFE7
:10934000400D030020420024BC4BBD4A034493421D
:1093500040F24C82BB4BBC4A0344934240F29182A0
:10936000BA4BBB4A0344934240F27184B94BBA4AA8
:1093700003449342C0F09084B84BB94A03449342EB
:1093800040F2FC84B74BB84A03449342C0F01285C4
:10939000B64BB74A03449342C0F0B385B54BB64AC7
:1093A00003449342C0F0A985B44BB54903448B42B2
:1093B00034BF4FF4E0514FF4C051E2684FF0010860
:1093C00022F47052E260E3680B43E360E5E6D0F814
:1093D000B432DB69002B8CD09847D5F8FC4C88E779
:1093E00004F58051C6EBC602A648C3F30A130E6803
:1093F00005EB8202C0F8C0600968C0F8C410D2F85A
:10940000101F0B44C2F8103F0DE5DDF804A013E572
:10941000012302EB4B11BB60D5F80C3DD4F840C0E2
:10942000012B886800F0DD80974B9C4500F0D581CA
:10943000D5F80C3F5BEA030300F0F183504666F079
:1094400057FBD5F8FC4CA1E50822904804EB4B13E0
:10945000BA60226C03F53063114602929A68814229
:1094600004D9110402D54FF400429A60854AD2F81B
:10947000004192F8C0E004F52A7184F8A8E292F85D
:10948000C1C084F8A9C292F8C33092F8C2A00AEB16
:10949000032A1FFA8AFAA4F8AAA292F8C53092F811
:1094A000C40000EB0320134680B2A4F8AC0292F88B
:1094B000C72093F8C63003EB02230122C4F894229C
:1094C0000EF01F029BB2012AA4F8AE32C4F8983203
:1094D00000F0A080022A00F0F680002A00F0D88078
:1094E0000EF08001D4F8D00266F030F9029B674A92
:1094F000934204D9D5F80C1D012900F0BC81D5F8A0
:10950000FC4C47E5DDF804A09CE447F6F0721342FA
:109510003FF489ACC3F30A13C6EBC6024FEAC60C8C
:10952000D91C05EB82028908D2F804EF09D00EEBB2
:10953000810004F580577246396842F8041B824264
:10954000FAD1ACEB06020EEB030105EB8202C2F886
:10955000041FD2F8101F0B44C2F8103F63E4494BBC
:109560000122D3F80001D0F8B43280F89C220179AE
:109570005B689847D5F8FC4CBCE4424B0421D3F817
:10958000003193F89C2283F89C1283F89D2268E4B2
:10959000D6E911231344B364BBF1000F7FF45AAD35
:1095A000D5F84C3D002B00F03583364BD5F8440DF3
:1095B000D3F80031D3F89422022A00F0D38032F09D
:1095C000040200F0508193F8A022012A7FF454ADE8
:1095D0000022D5F8FC4C83F8A0224FE5D5F8440DC5
:1095E000E8E7030740F10581284B9C457FF6CEACA8
:1095F00002047FF5CBAC4FF400438B60C6E4D4F893
:10960000B832002B7FF4F0ADD4F8C032002B7FF4D9
:10961000EBADEFE50EF06003402B00F0F0801EF0A4
:10962000400F00F0EC80D4F8D002802166F08EF874
:10963000D4F8D002002166F089F857E7405327FF9D
:10964000FF340C00401E1BFF3F420F0000DC0BFFED
:109650007F4F1200808CF9FE20D6130060B6E5FE25
:109660005FE3160000D3CEFE40771B00C05BB3FE65
:10967000C091210000CA91FE20753800E05459FEC7
:10968000E09C4100604100240A31544F0A30544F9D
:109690000EF0600EBEF1200F00F0DF80BEF1400F33
:1096A00000F0DB80BEF1000F00F01181D4F8D00291
:1096B0008021039266F04AF8039AD4F8D00211464A
:1096C00066F044F812E70EF06002202A00F0C58030
:1096D000402A00F0C280002AA5D1BCF1010FC1B21E
:1096E00000F0F182BCF1030F00F0DA82BCF1000F50
:1096F000DCD194F89C32022B00F04483032B92D1EE
:10970000000600F18C8301F00F02142303FB0242D8
:10971000D2F858A1BAF1000F00F0588301F07F028F
:1097200003FB024303F5AA73002A40F01C840022C5
:109730001A60D4F8D0020222C4F8942200F13C014D
:10974000C4E9072202650022836442654FF48072F7
:1097500082870269012A08BFC364D2B2006866F03A
:1097600045F9C3E6D3E90812914200F22382D86991
:10977000B0FBF2F102FB110111B9824240F26B829F
:10978000D3F8B422D2683AB193F89C12032903D1DA
:10979000184602939047029BD3F8D002802102938F
:1097A00065F0D4FF029B05220024D3F8D002C3F851
:1097B0009422026900F5FE71C0F80842012AA0F85F
:1097C000FC41D2B2029308BFC0F80C42C0E9844405
:1097D000006866F00BF9029BF5E603043FF50BAF5A
:1097E00080067FF52BAE20238B6027E64FF4705167
:1097F000E3E5830648D520238B60FFF7C7BB94F8C9
:109800009C32013B022B3FF60EAFC0B203283FF65D
:109810000AAFD4F8B43220469B689847B4F8AE3209
:10982000002B7FF463AE00287FF460AED4F8D03212
:10983000E0610422C4F894229864C3E914004FF450
:10984000807203F13C019A871A69012A08BFD86423
:10985000D2B2186866F0CAF848E6D4F8B4322046A6
:109860009B68984742E6D3F8D0028021029365F0C6
:109870006DFF029BA7E6C84AD5F8FC0C65F03CFFDB
:109880003DE64FF4605198E510F0280F7FF47EAB71
:10989000C24B9C4502D902043FF5ADAE0B69D9F825
:1098A0000422C3F31203D31AC9F81432D9F80832C8
:1098B0001344C9F80832D5F80C3F5BEA03037FF480
:1098C000BDAD2046B44A012165F016FFB6E5BCF1F6
:1098D000090F3FF6A8AE01A252F82CF0919A0408A5
:1098E0005B9A0408279604087D9A040827960408C2
:1098F000D19904089B990408279604084B990408F9
:10990000059904085FFA8AF2DFF894A2012A8AF81E
:109910000C203FF688AE94F89C32022B00F0BD82FA
:10992000032B00F09D82D4F8D002802165F00EFF59
:10993000D4F8D002002165F009FFD4F8B4329AF8C7
:109940000C1020465B689847D0E5012B7FF46BAE86
:1099500094F89C22022A00F24582002A3FF463AE6A
:10996000D4F8D002224600214FF0020C42F8081F22
:10997000C4F894C2C4E90733C0E914314FF48073CA
:1099800000F13C01826483870369012B08BFC26434
:10999000DAB2006866F02AF8A8E54FEA1A23002236
:1099A000013BADF81620062B3FF63DAE01A252F862
:1099B00023F000BFA59B04087F9B0408639B040859
:1099C00027960408279604084D9B0408DF9A04088C
:1099D00003437FF428AEBAF17F0F3FF624AE94F82C
:1099E0009C32032B3FF41FAE5FFA8AF2D4F8D032D8
:1099F00084F89E2293F8BC13012911D083F83820F3
:109A000000201A68D2F8001821F4FE61C2F800188C
:109A1000D2F8001841EA0A11C2F8001883F8BC0312
:109A20000422002003F13C01C4F894224FF4807218
:109A3000E0619A871A699864012AD2B208BFD86493
:109A4000C3E91400186865F0D1FFBAF1000F00F007
:109A50008582022384F89C3248E594F89C32013BCD
:109A6000022B3FF6E0ADBAF1010F7FF43FAD0020CD
:109A7000D4F8D032C4F8A402E061DAE6BAF1010FFA
:109A80007FF434ADC4F8A4A2D4F8D0320020CFE6DD
:109A900094F89C22013A022A3FF6C5AD022B7FF4CE
:109AA000C2AD0123E360D4F8A4320BB10323E36019
:109AB000D4F8D0320222C4F8942203F13C01C4E964
:109AC00007221A6500220C345A654FF480729C6498
:109AD0009A871A69012A7FF4BBAEDC64B8E6237C5E
:109AE000002B7FF4A0ADD4F8B4320DF116001B6B3F
:109AF000984707234370BDF816200AB3B4F8AE3276
:109B0000002BC1D09A424FF0020128BF1A46D4F868
:109B1000D032C4F89412ADF8162003F13C01C4E928
:109B200007221A65002298645A654FF480729A875A
:109B30001A69012AD2B208BFD864186865F056FFC6
:109B4000B4F8AE32002B7FF4D1AC9DE7237C002B20
:109B50007FF469ADD4F8B4320DF116005B6B984711
:109B6000C9E75FFA8AFABAF1050F3FF65CADDFE8A4
:109B70001AF0ED01E501DD01CC0102022501237C93
:109B8000002B40F00B82D4F8B4320DF116009B6A22
:109B9000984702234370AEE7204200240A30544F16
:109BA00058420024D4F8B0320DF11601207C1B6815
:109BB0009847A0E78A1AD3F8D04202931A6292B269
:109BC00004F13C01DA6122650022A06462654FF471
:109BD0008072A2872269012AD2B208BFE06420689D
:109BE00065F004FF029B0021D3F8D0020269C0F89F
:109BF0000812012AA0F8FC11D2B208BFC0F80C125A
:109C0000C0E9841100F5FE710068029365F0EEFE74
:109C1000029BD8E42046C34A65F06EFDC5E4236C80
:109C2000C1498B4203D91368002BFFF607AC002310
:109C30001361136943F400231361136943F018039C
:109C40001361136943F0C0431361FFF7F7BB4FF48F
:109C50005051FFF7B2BBD3F898229042BFF490ADB9
:109C6000D3F8D00200244FF480720293DC6100F13B
:109C70003C01828702698464012AD2B2C0E914449B
:109C800008BFC464006865F0B1FE029B0021D3F8F0
:109C9000D002C3F89812A9E74FF44051FFF78DBBEB
:109CA00094F89C0202285BD003287FF4FFAC5AEAA8
:109CB00003037FF4E9AE4A063FF4E6AED4F8D002DF
:109CC00065F044FDE0E694F89C32022B48D0032B6B
:109CD0007FF4ECACBAF1000F7FF408AC4B063FF414
:109CE000D3AED4F8D02201F00F01536899423FF669
:109CF000CBAE10F0800F4FF01C0040F0478100FB0E
:109D000001234FF0000C03F5FE7383F801C01970B6
:109D10000021997092F8BC1301293FF4B5AE0121DE
:109D200082F8BC1393F801C01878D978BCF1010F00
:109D30001368A1F102010CBF03F5106303F5306352
:109D4000012903EB4013186820F40010186003D8B1
:109D5000196841F080511960002382F8BC3393E602
:109D600011F07F0AD4F8D00232D065F0EFFCD4F8BD
:109D7000D002802165F0EAFCFFF7B8BB4FF4305108
:109D8000FFF71BBB4A067FF44EAC03064FF00202FE
:109D9000D4F8D0324FF000014CBF04F1140004F5A8
:109DA000AA700160C4F89422C4E90722C3E914210F
:109DB000986444E54FF42051FFF7FFBAD4F8B0326D
:109DC000D3F818A0BAF1000F40F0A780D4F8D00261
:109DD000802165F0BBFC5146D4F8D00265F0B6FC9A
:109DE000FFF784BB032A7FF41EACD4F8D002022212
:109DF00004F1040CC4F8942200F13C010269C4E9A6
:109E0000073303650023012AC0F848C043654FF4B7
:109E1000807383877FF4A1ACC0F84CC09DE401F04F
:109E20000F03142202FB0343D3F818A0BAF1000F6A
:109E3000CCD001F07F014B1C03EB830304EB8303C5
:109E400000293FF474ACD4F8D0221C2000FB01227E
:109E500092F83E20002A00F0968001221A6068E401
:109E60003AB3616801293FF40FAED4F8B432C9B2F5
:109E700020465B6898479AF80C10D4F8B4326160B9
:109E8000002B3FF4D0AB1B682046984700287FF496
:109E9000CAABD4F8D032E061CBE4B2B103230121E4
:109EA00084F89C32D4F8B4326160002BEBD1FFF718
:109EB000BABBD4F8B43202216260204684F89C1206
:109EC00011465B6803929847039AD4F8D032042174
:109ED000E261C4F894124FF4807118699A64012801
:109EE000998703F13C0108BFDA64C3E91422C2B2C6
:109EF000186865F07BFDFFF7F9BA4FF40051FFF7E2
:109F00005CBA4FF41051FFF758BAD4F8B032D3F816
:109F100010A0BAF1000F3FF459AF0DF11601207CEB
:109F2000D047E8E5204200240A30544FD4F8B0323C
:109F3000D3F80CA0BAF1000FEFD147E7D4F8B03254
:109F4000D3F808A0BAF1000FE7D13FE7D4F8B03258
:109F5000D3F804A0BAF1000FDFD137E7012384F86A
:109F60009C32FFF7C3BAD4F8D0221C2000FB012298
:109F700092F8FE216EE7D4F8B032D3F814A0BAF10B
:109F8000000FCAD122E71A60FFF7D3BB00FB012301
:109F90004FF0010C3C3383F801C0B8E6D4F8B4327A
:109FA0000DF11600DB6A984702234370A3E500BF5A
:109FB000F8B55B4CD4F8AC3C1A69960702D5DA6860
:109FC000950748D41A69500702D5DA6851073AD480
:109FD0001A69120702D5DA6817072CD41A69D6064F
:109FE00002D5DA68D5061ED41A69D00702D5DA6818
:109FF000D10738D41A69120602D5DA6817066FD469
:10A000001A69D60502D5DA68150670D41A6954069D
:10A0100002D5DA68500671D41A69910602D5DA6859
:10A02000920672D4F8BD6FF0100100221961D9694F
:10A0300084F8C82CD8E76FF0080100221961D969AB
:10A0400084F8C82CCAE76FF00401002219619969ED
:10A0500084F8C82CBCE76FF00201002219619969ED
:10A0600084F8C82CAEE72F4A6FF0010193421961C2
:10A07000C0D1D4E9B625AA42BCD02B498CBFC2F5C9
:10A080008055AD1A0A44D4F8BC12A8B2D1F81462B3
:10A09000C1F80822C1F81002002EABD1D4F8D43296
:10A0A00001276063C1F8147240F20111D866186983
:10A0B0005A66B842A3F858101E6703F1580108BF4A
:10A0C0009A66C2B2186865F09BFBD4F8D81229448E
:10A0D000B1F5805FC4F8D8121BD0D4F8AC3C89E746
:10A0E0006FF080021A611A69D6058FD58BE76FF47D
:10A0F00080721A611A6954068ED58AE76FF04002A1
:10A100001A611A6991068DD589E76FF020021A61EC
:10A11000F8BD0022D4F8AC3CC4F8D8226AE700BFEE
:10A120006031002400140040685200240378022BA0
:10A1300012D00F4943680269D1F85C05023A184011
:10A1400010B4400AD1F85445D1F8501504FB020070
:10A150005DF8044B08447047054B4268D3F8481536
:10A16000D3F8440500EB410000EB5220704700BFDC
:10A17000603100242DE9F84F9B4602F0020708B930
:10A18000002F52D1844DD5F84C45002C58D14FF0BA
:10A19000FF3E824C4FF0000CF146F046F246E66975
:10A1A000B04200F0D08094F82A60002E61D0012ED9
:10A1B00010D105EB0C1696F86B63F3070AD416F072
:10A1C0007E0F07D1F30940F0AC80666A564501D294
:10A1D000B246E1460CF1010C1034BCF1080FDED19F
:10A1E000BEF1FF3F04D1B8F1FF3F00F0A780C646A3
:10A1F000D5F8DC430EF1020605EB0E18013405EB31
:10A20000061CC5F8DC43CCF84443C8E9D704002455
:10A21000CCF8484305EB061494F84A43042C05D8BF
:10A22000DFE804F02F4988495F005B4D95F8F8346A
:10A23000DBB10123022485F841332046BDE8F88FC5
:10A24000D5F85465D5F8503506FB0434A0429ED3AA
:10A2500095F8F83413B9012385F8F8340123002464
:10A2600085F841332046BDE8F88F012385F8F8349E
:10A27000DFE7E6460CF1010C1034BCF1080F8ED17B
:10A28000AEE712F0010C72D105EB0610BBF1030F23
:10A290004FEAE20890F84B9368F3C71980F84B93A4
:10A2A00063D94FF6FF705B46834528BF034605EB35
:10A2B0000610A0F84833042C13D097B1D5F8E0036A
:10A2C000D5F8DC3301300133C5F8E00305EB0E109F
:10A2D000C5F8DC33C0F8603305EB0613042083F8BF
:10A2E0004A03500707D505EB061090F84B3343F0AF
:10A2F000010380F84B33D3060AD505EB061696F812
:10A300004B33C3F34502013262F3460386F84B3305
:10A31000D5F85833012403EB4E2320460B60BDE8EB
:10A32000F88FE0460CF1010C1034BCF1080F7FF4FB
:10A3300036AF55E700242046BDE8F88FB9F1FF3F5E
:10A34000F8D0CE4654E70CF10206E64605EB0618B7
:10A3500098F84A43002C3FF44BAFD5F8DC43013466
:10A36000C8F84443C5F8DC4354E763469FE7D5F893
:10A370002839002BDED0D5F858135F68002301EB95
:10A380004E21074AB8470028D4D005EB0615022312
:10A3900085F84A3351E700BF60310024A03400241F
:10A3A000296D040870B5114D82B00E4695F8403302
:10A3B000022B16D1020AC4B2D5F84405002301A924
:10A3C00010440322FFF7D6FE012808D195F8403348
:10A3D000022B019B0CBF23F8146043F8246002B0E9
:10A3E00070BDC0F3D41200F07F04E5E760310024B3
:10A3F0002DE9F04F424C012883B00D4694F840738C
:10A400008CBF4FF0000B4FF0010B1646032F0B686B
:10A4100035D0022F59D14FEA13284FF48079DFB29B
:10A420000138012819D84FF0010A9E4264D9D4F8A6
:10A43000BC241AB1D4F8D814994249D0D4F84405B0
:10A440000023092201A94044FFF794FE01281FD0F0
:10A45000022810D060B12B68E7E7BFB194F8F83458
:10A4600013B9012384F8F8340123022084F841331E
:10A4700003B0BDE8F08F022003B0BDE8F08F4FF0CD
:10A480008009C3F3D41803F07F07C9E7CA46CCE7B5
:10A4900094F840230199022A14D0032AEBD151F8F1
:10A4A000273023F07043B3FA83F357445B095B45CD
:10A4B0002B681FD053444F452B60ECD308F10108A3
:10A4C0000027B2E731F81730EDE74FF48079D8E78D
:10A4D000D4F85415013A02EB41224902B2FBF1F2E1
:10A4E0001344B3FBFAF20AFB12320AB153449B1A2B
:10A4F0002B609AE7B342BBD303202E60B8E700BFBE
:10A50000603100242DE9F04FDFF858B18946174635
:10A5100083B09BF84013D9F80020022940F08680D0
:10A52000D6B2DBF844554FF48073A6EB020805EB76
:10A530001225B8449844BA4208F1FF38B8FBF3F842
:10A5400047D200F0010AA844032907EB0604A8EB50
:10A550000503A4EB02040CBF80224FF480729442E6
:10A5600028BF14460EB9944237D20B2201A92846BF
:10A57000FFF700FE012802D003B0BDE8F08F9BF882
:10A580004013D9F80020022902F1010327D0B44278
:10A5900010D96FF040420198324400EB8202043837
:10A5A00000EB840042F8043F824203F10103F9D139
:10A5B000D9F80020A61B32449742C9F8002002D1E6
:10A5C000BAF1000F43D1974205F101054FF00006A3
:10A5D000BAD8012003B0BDE8F08F0A22C6E7B44222
:10A5E00010D96FF0004CDDF804E0B4440EEB4C0CD5
:10A5F000AEF1020E0EEB440E2CF8023FE64503F1DD
:10A600000103F9D1921B22449742C9F80020DAD104
:10A61000BAF1000FD7D06FF00043019A4FF6FF71E7
:10A62000234422F8131003B0BDE8F08F02F07F0638
:10A63000DBF844350329C2F3D415A6EB02081D4408
:10A6400018BF4FF48073B84408BF802372E76FF0DF
:10A650004043019A4FF0FF30234442F82300D9F8D9
:10A660000020B0E76031002430B50446C06983B0F3
:10A6700010B9012003B030BD0D460023032201A90B
:10A68000FFF778FD0128F5D1B4F92030002B0ADA64
:10A69000144B93F8F8240AB983F8F8040122022035
:10A6A00083F84123E6E7019A012D4FEA431102EBBB
:10A6B000431303D0022D11D1E5255554A268DA6168
:10A6C0002278032A04D100221A775A779A77DA7708
:10A6D000626A110C5A83998203B030BDE268DA6174
:10A6E000EEE700BF60310024F0B5002990F83C305F
:10A6F00083B0044614BF02210021042B72D8DFE886
:10A7000003F0030C3A456100FFF7AEFF012867D163
:10A71000626B002A6CD184F83C003B4D4FF6F77613
:10A720003A4F16E0B2424AD861F07EFD01284FF060
:10A7300000011ED1206BFFF735FE012819D1019AC7
:10A74000D5F85815531E22638B4228BF0B46C5F817
:10A75000583595F8402301A9236B032A18469AB26D
:10A76000E0D1BB422BD861F05FFD01284FF0000122
:10A77000E0D003B0F0BD426B04F130010020FFF7E0
:10A78000C1FE01282CD1032384F83C301E48E26A24
:10A79000D0F8D83400F2B440D0F8A0109B1A42622E
:10A7A000C26801FB03F3816801EB4325002102EB42
:10A7B00043238560C360FFF757FF012810D10423AE
:10A7C00084F83C3094F82830042B02D1002384F81C
:10A7D0002830A36B83B120469847012003B0F0BD19
:10A7E0000228C6D194F82830042B08D00220C0E7F4
:10A7F000022384F83C30BFE7012003B0F0BD002302
:10A80000022084F82830B4E760310024F7FFFF0FFE
:10A8100038B590F834300446052B40D8DFE803F013
:10A820001E03390F1863006B4FF0FF31FFF7BAFDBD
:10A83000012834D1E06AA0BB032384F8343000211E
:10A840002046FFF711FF012829D1042384F8343072
:10A8500094F82830082B28D0012038BD234D00F172
:10A8600030010120D5F84C250232FFF7C1FD012847
:10A8700028D00238C0B2012811D8052384F834301A
:10A8800094F82830082B15D00123022085F8F934DC
:10A8900038BDC06A216BFFF785FD0128CCD00020B0
:10A8A00038BD022384F83430F4E70023012084F813
:10A8B000283038BD0023022084F82830012385F891
:10A8C000F934E5E7D5F85425E368206B03EB422320
:10A8D000E26AC5F85805C4E9033002B96062012391
:10A8E00084F83430A0E7014DCAE700BF603100248E
:10A8F00038B590F838300446032B4CD8DFE803F025
:10A90000022E37422A4BE56893F84003D3F85415DA
:10A910000328D3F8BC04D3F8D8240CBF4FF0800C24
:10A920004FF4807C226101FB0CF1A0EB412005EB90
:10A930004125E560C3F8BC04D3F8C004A0EB412175
:10A94000E06AC3F8C01402EB0C01C3F8D814C4E9E0
:10A950000C2148BB6262012384F83830002115487D
:10A96000FFF782FE012811D1022384F83830626B90
:10A9700004F130010120FFF7C5FD012806D10323B2
:10A9800084F8383000212046FFF76EFE431EDBB20C
:10A99000012B01D938BD022094F82830062BF9D1BB
:10A9A000002384F8283038BDA2EB0C022263D2E7E2
:10A9B00060310024143600244368C3F308020A44BB
:10A9C000B2F5007F2DE9F043044683B00D4605D271
:10A9D0002B440120636003B0BDE8F08390F91A10A6
:10A9E000481C0AD0484A02EB011292F86B136FF32D
:10A9F000000182F86B13FF22A27694F91B20511CF0
:10AA000016D0414E023206EB021191F84B13C1F3FE
:10AA1000450101292ED9013901F03F0106EB02124F
:10AA2000FF2692F84B0361F3460082F84B03E6766B
:10AA300094F800C0BCF1020FCAD0334ED6F85425AA
:10AA4000B5EB422F4FEA422910DCD6F85C2503EA29
:10AA50000208C8F10002AA4208DC05EB08024A45D8
:10AA60000AD2206900283FD10120B4E7002003B0BA
:10AA7000BDE8F0830021D1E7227E206912F00807AB
:10AA800027D0D6F8D824411C8A4214D300D1002103
:10AA90004B44A5EB0905BCF1020F6061A3EB080371
:10AAA0004544084621616360DCD1D6F86425B3EBE8
:10AAB000422F8DD3D8E796F8F82422B9012386F8DF
:10AAC000F83463682069012286F8412394F800C0B5
:10AAD000DEE701A961F0A8FB0128C7D101996368ED
:10AAE00094F800C02069D3E796F84023032A06D0E3
:10AAF00080B24FF6F77290427FF66AAFB4E7034A2E
:10AB000090427FF665AFAFE760310024F7FFFF0F9B
:10AB10002DE9F04390F8384083B00546032C00F24D
:10AB2000A680DFE804F002186E0BFFF771FE012823
:10AB30000FD0022809D1032385F8383000202B6C70
:10AB4000022485F8280003B19847204603B0BDE8E9
:10AB5000F08385F838002B78022B5ED0454A6B686D
:10AB6000D2F85C2503EA0209C9F34F292846414F70
:10AB7000FFF7DCFA0646A9EB000901A902223046DC
:10AB80000023FFF7F7FA09EB060801284FF40072DB
:10AB90001FFA88F84FF00001044606F10106D4D1EF
:10ABA00001986EF06BFAEB694FF4007128460BB117
:10ABB0006B68C3B3D7F854355A1E90450CD2FFF7D3
:10ABC000FBFE01230028D8D197F8F8240AB987F8AA
:10ABD000F83487F84133D0E7C3EBC3532846590212
:10ABE00001F50071FFF7E8FE40B997F8F83413B9A2
:10ABF000012387F8F834012387F84133022385F8CD
:10AC0000383000222B6C85F8282053B101242846C7
:10AC10009847204603B0BDE8F0836B68C3F34F2923
:10AC2000A4E7012491E7019B4FF020324FF0100E72
:10AC30004FF02E0C1A605A6083F800C0C3F807204A
:10AC40006C6A1A625A6283F80BE0C3F8272083F813
:10AC500020C083F821C0EA6B5C8324FA0EF45A8783
:10AC600022FA0EF29C8283F82BE09A86A2E7002457
:10AC70006BE700BF60310024B1F904300F2B2DE9E0
:10AC8000F0410D4682B0044616463AD02046FFF702
:10AC90004DFA94F91B80B8F1FF3F43D05F4F07EBAB
:10ACA0000813D3F85C33984215D097F8F834002B8A
:10ACB00000F08480012387F841332278022A00F0D3
:10ACC00081802369002B66D101230022184632605F
:10ACD00002B0BDE8F081D7F8581301EB48210029F4
:10ACE00079D0AB88204601331BB201EB4311AB8016
:10ACF0003160FFF71BFA01232860184602B0BDE857
:10AD0000F0814FF40071FFF757FE002851D04FF645
:10AD1000FF732046AB80FFF709FA94F91B80B8F166
:10AD2000FF3FBBD12278022A57D02369002BC5D020
:10AD30003A4F97F84013032968D09BB24FF6F7714A
:10AD40008B4294BF00230123002BB7D130B997F871
:10AD5000F834002B4ED0012387F841330023112211
:10AD600001A9FFF707FA012835D10199D7F858331F
:10AD7000CB1A48BF03F2FF13B3F5805F4FEA63229B
:10AD800033D397F8F83413B9012387F8F834012343
:10AD900087F841332BE0214A92F84023032A2DD033
:10ADA0009BB24FF6F772934294BF00230123002B0E
:10ADB0008AD10023184602B0BDE8F081012387F84C
:10ADC000F83477E7154F6368D7F86425B3EB422F63
:10ADD000BFF47AAFEDE7227870E7104F6368D7F8D9
:10ADE0006425B3EB422FB1D3EEE74FFA82F884F833
:10ADF0001B8074E7012387F8F834ACE7084A9342D4
:10AE000094BF00230123002BD3D05DE704498B427C
:10AE100094BF00230123002B98D04FE7603100241A
:10AE2000F7FFFF0F2DE9F04F90F8303087B0044660
:10AE3000042B53D8DFE813F005000E005500F60090
:10AE40004E00CC4862F0B4FB4FF6FF72012322841F
:10AE500084F83030C84D04F11C0801AE04F131090A
:10AE600005F2FC47324641463846FFF705FF012808
:10AE700000F0FF80022831D195F916355A1C0AD00E
:10AE800005EB0313FF2193F86B2385F816156FF379
:10AE9000000283F86B2395F917355F1C17D0023336
:10AEA00005EB031292F84B23C2F34502012A40F24C
:10AEB0005F81013A02F03F0205EB031393F84B1355
:10AEC00062F34601FF2283F84B1385F8172504230C
:10AED00084F830300020E36A2070984707B0BDE85E
:10AEE000F08FA54D95F82435002BF7D104F11C09FE
:10AEF000A04F01AE4FF00908324649463846FFF7E9
:10AF0000BBFE012840F023810198002800F0FD805D
:10AF10000378E52B01D0002BEED1D5F85833C31AB6
:10AF200048BF03F2FF13B3F5805F4FEA632280F05E
:10AF30005B811201914B13449A7B042A0CD0D5F803
:10AF4000DC230132C5F8DC235A6004229A73D5F859
:10AF5000E0330133C5F8E03395F916355E1C0AD0AD
:10AF600005EB031393F86B236FF3000283F86B2355
:10AF7000FF2385F8163595F917355A1C17D002337B
:10AF800005EB031292F84B23C2F34502012A40F26B
:10AF90007581013A02F03F0205EB0313FF2185F8AA
:10AFA000171593F84B1362F3460183F84B132022D5
:10AFB00000216EF063F8D4F83110D4F8352003A8DE
:10AFC000019B19605A6094F83B20B4F839109A72CA
:10AFD0001981019B627EDA7203F0E4FA002800F026
:10AFE000E5809DF80E509DF80F10BDF80C0041EA69
:10AFF0004511019BA0F2BC709DF8102041EA402150
:10B00000D2028DB219829DF8111042EA41129DF8C8
:10B01000121042EA510291B2DA8103221D83D982D1
:10B0200084F83020237E980608D50023112202A937
:10B03000E069FFF79FF801287FF450AF204662F0E7
:10B04000B7FA2369002B00F08680237E03F0F70215
:10B0500013F00403227640F09380122A00F0B280AD
:10B060000022E36A204684F82820984707B0BDE80C
:10B07000F08FDDF804A0BAF1000F00F0C1809AF85B
:10B080000030002B00F0BC809AF80BB01BF0080FCA
:10B090007FF4E8AE0B22494650466DF081FF002850
:10B0A0007FF4E0AE637E8BEA0303DB0640F1EA80C7
:10B0B00095F916355F1C0AD005EB0313FF2193F8B1
:10B0C0006B2385F8161560F3000283F86B2395F95E
:10B0D0001725561C3FF4FBAE023205EB021393F822
:10B0E0004B33C3F34503012B40F21181013B03F0C5
:10B0F0003F0305EB021292F84B1363F34601FF2363
:10B1000082F84B1385F81735E1E695F8FC34022BED
:10B110003FF4DDAE95F82435002B7FF4D8AE85F8EA
:10B1200034353846C5F83835C5F83C3585F83035FE
:10B13000D5F8103585F82485C5F82835D5F8583563
:10B14000C5F82C35FFF7E4FC01283FF4D5AE022802
:10B150003FF4BDAEC2E6237E190781D5064B93F8B6
:10B16000DC24002A7FF4BAAE072283F8DC2477E7D8
:10B170000022A1E65C36002460310024BC340024A7
:10B18000A56800232046E66A294684F82830FFF7A0
:10B1900013FC00286CD194F82830002B7FF49EAE6D
:10B1A0000223C4E90B6584F8283097E6019B6FF011
:10B1B0007E01472244F281751974014698735A74CE
:10B1C000D8732AE7E06A0421626AA063204684F803
:10B1D0003C3084F8281063636362C4E90B22C4E93D
:10B1E000023362F0E5F979E695F8F83413B90123F2
:10B1F00085F8F83401236FF00F0285F8413399E6A2
:10B2000095F91635581C0AD005EB0313FF2193F866
:10B210006B2385F816156FF3000283F86B2395F9FD
:10B220001735591C16D0023305EB031292F84B2345
:10B23000C2F34502012A23D9013A02F03F0205EB8D
:10B24000031393F84B1362F34601FF2283F84B1369
:10B2500085F81725237EDA067FF539AE2E4862F091
:10B26000A7F94FF6FF720223228484F8303039E6C2
:10B27000002E3FF433AE2046B0472FE600228BE687
:10B280000022DCE7BAF81420BAF81A3043EA024385
:10B29000D5F8542563625202DAF81C30B3FBF2F1A0
:10B2A00002FB1131A36009B113445B1AE36084F817
:10B2B00019B095F91635581C0AD005EB0313FF2178
:10B2C00093F86B2385F816156FF3000283F86B2350
:10B2D00095F91725511C16D0023205EB021393F88D
:10B2E0004B33C3F34503012B13D9013B03F03F0359
:10B2F00005EB021292F84B1363F34601FF2382F829
:10B300004B1385F81735032384F830308AE6002381
:10B31000EFE60023ECE700BF5C36002410B50378AD
:10B32000044690F818C0023B012B02D91CF0060F0E
:10B330006ED11CF0200F44D194F91A20511C0AD070
:10B340003A4BFF2103EB021393F86B236FF30002D8
:10B3500083F86B23A17694F91B20531C16D0334934
:10B36000023201EB021393F84B33C3F34503012B75
:10B370004BD9013B03F03F0001EB0213FF2193F88F
:10B380004B2360F3460283F84B23E1761CF0080F51
:10B390000ED0264991F8DC34072B06D091F8F8340A
:10B3A000002B3FD0012381F84133002381F8DC34A6
:10B3B0000023E26A237084F8283042B3BDE81040CD
:10B3C00010471B4A0023E069D1691032884206D039
:10B3D0000133082BB0D0D16910328842F8D113491B
:10B3E000023301EB031292F84B23C2F34502012A08
:10B3F00016D9013A02F03F0201EB031393F84B1305
:10B4000062F3460183F84B1396E70020B4E710BDC2
:10B410000121FFF729F90128F9D194F818C088E72C
:10B420000022E9E7012381F8F834BBE7603100240A
:10B43000A0340024324A4FF0FF30F8B5A2F5507C1A
:10B440000023044603E001331032082B14D092F895
:10B450002A100429F7D10CEB031191F86B13CE07D6
:10B46000F1D4651C116A01D08142ECD21C46013333
:10B4700008461032082BEAD1631C01D10120F8BD27
:10B48000204DA61C05EB0613B3F8481399B9D5F85F
:10B490005813D5F8283901EB4421B3B105EB041456
:10B4A000DF68194A0023D4F85C03B84768B1022862
:10B4B0001AD00020F8BDD5F8283933B105EB0412B5
:10B4C0009B68D2F85C039847E1E7D5F8E03305EBD9
:10B4D000061603210122013B002086F84A13C5F815
:10B4E000E03385F8E423F8BDD5F8E03305EB061624
:10B4F00001220020013B86F84A23C5F8E033F8BD5D
:10B50000A034002460310024916D04082DE9F0433B
:10B5100090F8283083B00446013B082B0BD8DFE8B5
:10B5200003F0383C1F2305290A2E33000121FFF7C1
:10B53000DBF8012802D003B0BDE8F08300222378B5
:10B5400084F82820002BF6D0226C0321D4E90103D3
:10B5500084F828108342E26238BF03462046A36085
:10B5600003B0BDE8F043D9E6002103B0BDE8F043E5
:10B57000FFF7BAB803B0BDE8F043FFF7B9B903B0BD
:10B58000BDE8F043FFF744B903B0BDE8F043FFF76F
:10B59000BFBA03B0BDE8F04344E4DFF84C91436820
:10B5A000D9F85C55026B9C461D40D9F85415A81873
:10B5B0004E02B0EB412FC0F0918094F800E04FF6BE
:10B5C000F777DFF82081BEF1020F14D02069002840
:10B5D00053D1D4F804C0A3680021E26A634584F81B
:10B5E000281038BF6346A360002AA4D0204603B0C9
:10B5F000BDE8F0431047D4F804C0D9F86415BCEB9B
:10B60000412FE8D22069217E090728D5D9F8D8141E
:10B6100000F1010C61451ED299F8F81421B90123FB
:10B6200089F8F8346368226B012189F8411394F892
:10B6300000E0921B33442A445B1B00259642636062
:10B640002263C4E904C09C46BDD9BEF1020F39D0C3
:10B650002069F8B9BFE7ECD14FF0000CE9E701A988
:10B6600060F0E2FD01287FF466AF2069DDF804C0D8
:10B6700094F800E06368226BDBE799F84013032934
:10B6800019D081B2B94294BF002101210029BAD05A
:10B69000D4F804C099F84033032B19D080B24FF688
:10B6A000F773984294BF00200120002893D194445E
:10B6B000C4F804C08FE7404594BF00210121002950
:10B6C000A1D0E5E7D9F86415B3EB412FEFD382E7BA
:10B6D000044B984294BF00200120E6E794F800E074
:10B6E000B3E700BFF7FFFF0F6031002438B5194CF6
:10B6F0004422002104F2FC4528466DF0BFFC94F87A
:10B7000040334FF6FF71D4F86025022B2846A4F889
:10B7100016154FF003014FF01005C4F8202518BF8F
:10B720000B4684F814150021C4F80C2584F8FC3469
:10B7300084F81555FFF740F948B994F8243533B922
:10B740000222C4F82835C4F82C3584F824250120B9
:10B7500038BD00BF60310024704700BF024A136843
:10B7600023EA00001060704780620024704700BF29
:10B7700090F83C20034602F0FF0012B1002283F84B
:10B780003C207047007970470079C0F34010704743
:10B7900000794009704700BF704700BF03685A1C1A
:10B7A00002601970704700BF03685A1C026019706C
:10B7B000704700BF024B586803681B68184700BFFA
:10B7C00080620024F0B53B4E082241F2210033781C
:10B7D000934002E0013A8BB209D013F4004F4FEAD4
:10B7E0004301F7D080EA4303013A9BB2F5D1B6F8A2
:10B7F000011000295BD0DFF8CCE02F4DAE4554D2CC
:10B80000AEF1060E0EEB0104AC4234BF0027012757
:10B81000052998BF47F00107002F46D141F2210CBE
:10B82000744514D00EF1FF3E601E1EF8011F082261
:10B8300083EA012313F4004F4FEA43018CEA4303E8
:10B840000CBF8BB29BB2013AF4D17045EDD1228886
:10B8500052B1A11DA94226D2A118A646A94222D2C0
:10B86000052A20D90C46DBE7A71C254641F221001A
:10B8700015F8011B082283EA012313F4004F4FEA55
:10B88000430180EA43030CBF8BB29BB2013AF4D16F
:10B89000AF42EDD167880434FF1AA61B074BB7FAF5
:10B8A00087F71E817F093846F0BD1746FBE7044F36
:10B8B000BC1EDAE7000002080000040880620024D1
:10B8C00003000208070002084FF480538381704789
:10B8D0004FF40063838170474FF4006383817047A6
:10B8E0004FF40063838170474FF400638381704796
:10B8F000074B10B403F11001002453F8042B8242CB
:10B9000008BF43F8044C8B42F7D15DF8044B7047F5
:10B910008C62002470B5374C638DA08BB4F9345021
:10B92000C01A238DB4F922C000FB03F3B4F932002E
:10B93000266C05EBE335C00290FBF5F000EBE3303D
:10B94000A0F57A6EA0630EFB0EF30EFB0CFC1D132C
:10B95000B4F92E304FEAEC2C05FB03F30CEBE32C8F
:10B96000B4F92C3005FB03F3B4F924501B140EFB7F
:10B9700005FEB4F9205003EB6E330CEB850CB4F9E3
:10B980003C500233E48C0CFA05FC9B100CF1020CC9
:10B9900003F50043A6EBAC0C04FB03F34CF250346C
:10B9A0002C41DB0B04FB0CF4002C1EDB6400B4FB0D
:10B9B000F3F389B11C1240F6DE3504FB04F405FBF9
:10B9C00004F40D4D241403FB05F504EB254404F6A3
:10B9D000CF6403EB24130B602AB100EB800040001E
:10B9E000083000111060012070BDB4FBF3F35B0060
:10B9F000DFE700BF8062002443E3FFFF01207047C0
:10BA0000012070472DE9F84F6E4F0E4615467C6CAD
:10BA1000B7F84800B7F95290C0EB2413B7F84E803E
:10BA200040004FEAE97BC0EBE40003FB03F4B7F905
:10BA30004C30241303FB04F4B7F94A30A41303FB7E
:10BA400000F0B7F9503004EBE0240020A4F5FA31FF
:10BA50003C6683FB013281FB01EC12034FEA033A9F
:10BA600042EA135209FB0CF30EFB0B3BA9FB0E3908
:10BA7000D9441B0A43EA096313EB0A0342EB292268
:10BA8000A3FB083902F5004208FB02984FEAE8736D
:10BA90004FEA680253EA680800F08780B7F95880D7
:10BAA00008FB0CF9B7F956C04FEAE87A8CFB011C89
:10BAB0000EFB0A994FEA4C4CA8FB0E8E4CEAD13C87
:10BAC000CE44490411EB08014EEB0C0C4018796E82
:10BAD000C1F58018B7F954100CEBC10108F0004C07
:10BAE0004CEA580C4FEAC878B8EB00006CEB010147
:10BAF00010EB000841EB010E18EB000841EB0E0EB5
:10BB00004FEA881C4FEA8E1918EB0C0C49EA986929
:10BB10004EEB090E4FEA8E0E4EEA9C7E4FEA8C0CDD
:10BB20001CEB000C41EB0E0E4FEA8E0E4EEA9C7E93
:10BB30004FEA8C0C1CEB000041EB0E0165F042FF5C
:10BB4000B7F95E204FEA6138B7F95CE0430BB7F90B
:10BB50005A7002FB08FC4FEAE27943EAC14303FB57
:10BB600009C9A2FB032CCC4402FB08F803FB0C8898
:10BB7000A2FB032C4FEAEE73C444520E42EACC12ED
:10BB8000121841EB6C6C0EFB01F103FB0011AEFBD4
:10BB900000300144DB0C43EA4133D0184CEBE14167
:10BBA000000A40EA016000EB07100EB1000A3060A5
:10BBB00025B104EB8404803424122C600120BDE8FC
:10BBC000F88F00BF8062002431B10A4BD3ED207A98
:10BBD000FDEEE77AC1ED007A52B1064B9FED067A91
:10BBE000D3ED217A67EE877AFDEEE77AC2ED007A2F
:10BBF00001207047806200240000C8422DE9F04F08
:10BC0000604D85B0B5F89630D5F888001B02B5F8C0
:10BC10009480B5F89260B5F89840CDE90112C21A47
:10BC2000B5F89000B5F88E3067EB07074FEA004E85
:10BC3000A8FB020CD90308FB07CCC00940EA4C6002
:10BC40004FEAEC1C10EB0E00A6FB023E06FB07EED3
:10BC50004FEA13234CF1000C43EA0E634FEA2E2EF9
:10BC60005B18A4FB021604FB07644FEAD1514EF1A6
:10BC7000000E41EA4421E41511F5FA6844F100068A
:10BC8000B8F5FA6F039676F1000630DAA1FB01B63B
:10BC900001FB04FA06EB4A0A4FEA8B064FEA8A09CF
:10BCA00016EB0B0649EA9B794FEA560B4AEB09095A
:10BCB000B6084BEAC97B46EA8976B0EB0B006CEB21
:10BCC000690C9B1B304E6EEBA90E4FF0FF39B0454F
:10BCD000039E76EB090626DB02FB07F7A2FB022197
:10BCE00001EB4707D20F42EA4702B8EB0208019C7A
:10BCF0008CB1D5F89C10A1FB033201FB0E2E5B0D1D
:10BD000043EACE234FEA6E5E1B1A6EEB0C0CDB0B84
:10BD100043EA4C432360029B0BB1C3F8008001202F
:10BD200005B0BDE8F08F40F6AC56891944F1000427
:10BD300001FB04F4A1FB019101EB44044FEAC901AA
:10BD4000E600B9EB010146EA597664EB06060818ED
:10BD50004CEB060C19EB090644EB040A16EB09063A
:10BD600044EB0A0A4FEA8A0A4AEA967AB600B6EB28
:10BD700009016AEB0404490841EAC4715B1A6EEBDD
:10BD8000640EA9E78062002424FAFFFF01207047B7
:10BD9000124B10B4124C1B68D4F8A0001B1AFA2BDB
:10BDA0000FD811B1D4F8AC300B6032B1D4F8B03048
:10BDB00001205DF8044B1360704701205DF8044BCF
:10BDC0007047D4F8A430002223F00403104684F80E
:10BDD000A820C4F8A4305DF8044B70474C3E002402
:10BDE0008062002438B51446002944D0344B0D46F7
:10BDF0009FED344AD3ED2D7AB3F9CC20B8EEE76A43
:10BE0000D3ED347A04EE902AB3F9C820F8EEE77A3D
:10BE100093ED307AC6EE046A05EE902AB3F9CA2093
:10BE200093ED2F0A05EE102AB3F9C620B3F9C430FA
:10BE3000F8EEE44A06EE102AF8EEE55AC7EE843A28
:10BE400007EE903AB8EEC55AB8EEC77AB8EEC66AB1
:10BE5000B8EEC00AE6EEA45AA6EE856AF8EEE77AD6
:10BE6000A6EEA57AE6EE867AA6EE870AA3EEA70AE4
:10BE700068F06EF928600CB3114BF6EE005A9FED96
:10BE8000115A93ED346AB3F9BA20B8EEC66AB3F921
:10BE9000B83007EE902A9FED0C0A07EE103AF8EE44
:10BEA000E76AC6EE057AB8EEC77A67EEA67AE7EEDD
:10BEB000257A27EE800A68F04BF92060012038BD12
:10BEC000806200240000F04A0000C8422DE9F843D7
:10BED0000446D0E900301344834221D88E18676BA2
:10BEE0008E421AD00D464FF0000904F1100801E00F
:10BEF000AE4212D0236B5A1C23442263202A15F829
:10BF0000011B1974F4D14146204617B9F7F78AFA94
:10BF10000746AE42C4E90C97ECD13846BDE8F88339
:10BF20004FF0FF37F9E700BF2DE9F04F54220446E8
:10BF300000218DB0A3486DF0A1F8A34A611EE01C5A
:10BF4000144611F8013F5D1E052D88BF002388426D
:10BF500044F8043BF5D102F11003114651F8040BEB
:10BF6000012800F024818B42F8D1114651F8040BCE
:10BF7000022800F012819942F8D1114651F8040BC1
:10BF8000032800F000819942F8D152F8041B0429DB
:10BF900000F0EF809342F8D105204FF01A080026F8
:10BFA000884CDFF84892FFF7A3FC884F0620FFF784
:10BFB0009FFC257B002D41D0284694F90DA006F06A
:10BFC0005FFF8346E0B10523026800258049837145
:10BFD000804B0572134480F807809B0A31F81300E8
:10BFE00060F042FEBBF80430DBF8000007A90793BD
:10BFF00003230B950893CDE90955F5F76FFA257BD7
:10C000000023302204E001331C2B36D019F83320F2
:10C010009542F8D109EBC3035B68F4200122236148
:10C02000062100FB0A7A16446275DAF8F0308AF8C5
:10C03000EC209A18A1752375CAF8F02008F10108C0
:10C040000C345FFA88F8B8F1200FB2D196B1DFF85E
:10C050007C814FF00009DFF898B1C2469AF8EC30C5
:10C060006BB909F101090AF1F40A0BF58C7BB9F1FE
:10C07000030FF3D10DB0BDE8F08F0023CDE7BAF880
:10C0800006004FF4403660F0EFFDBAF8040060F0AF
:10C09000EBFDDAF8F030F421DAF80020012BCAF8D1
:10C0A000283001FB09814FF0030CD4BF002301238A
:10C0B000CAF81020CAF81C300023CAF838308AF8B1
:10C0C0002C30CAF83030CAF820308AF824308AF888
:10C0D000483004930823CAE9056301238AF8253010
:10C0E0004FF48063CAF834304FF48053CAE90FC369
:10C0F0004B6E002B00F0B98193689D0003D59168C9
:10C10000354B0B4093609368DC0013D4334B90683D
:10C110001968334B034043F080539360314BB1FBBC
:10C12000F3F30493049B2BB1049B013B0493049B06
:10C13000002BF9D19368D80019D4F423012403FB10
:10C140000983596E41F010015966996E2143996631
:10C15000936859074ED5F42303FB09835B6EF423E0
:10C1600003FB09835A6E42F010025A6679E70024F5
:10C17000EEE71D4B342193F8282183F80411013296
:10C1800083F8282108E71849352491F8280181F817
:10C19000F840013081F82801F7E61349312491F87D
:10C1A000280181F8EC40013081F82801E5E60E49CC
:10C1B000302491F8280181F8E040013081F828010D
:10C1C000D3E600BF546300248C6200245819002475
:10C1D00024B20B080000FEA7C0FFFF5F0000002490
:10C1E000C0FFFF6F400D030080620024E8B20B081F
:10C1F00000000030F42303FB0983596EC906AED456
:10C20000596E21F4817141F0020159669368DB0790
:10C2100013D49F4B9A4200F0E98303F580739A424E
:10C2200000F0E4839B4B9B68DE0706D49A498B6839
:10C2300023F47C1343F440338B60984B98491B687C
:10C24000D368194043F208030B43D36090689368A6
:10C2500000F0040003F00803184300F04283DAF80A
:10C260001030DAF81C20012A00F08D841A6B22F0BD
:10C270000F021A63F42202FB0982536E23F00303B8
:10C2800043F001035366002C7FF4EBAE9AF8603064
:10C290000594012B3FF4E5AE0121DAF810308AF85D
:10C2A000601099688D0740F1E9829A68F4207D4911
:10C2B0007D4A00FB09807D4D466E314041F0020110
:10C2C000416699680A4042F000429A609A68002AE2
:10C2D000C0F2F282F42000234FF480654FF4006135
:10C2E00000FB09804FF0030C714E426E22F00302F6
:10C2F00042F0010242664FF400528AF86030CAF8F8
:10C300009830CAF89CC0CAE91F33CAE92833DAF862
:10C310000C30CAF878304FF48073CAE923234FF405
:10C320000033DAF80820CAF8943003F18043103360
:10C33000CAE921519A425546316845F8742F00F0F8
:10C34000988018339A4200F094805A4B5A4FBA4260
:10C3500018BF9A4207F118070CBF01230023BA4205
:10C3600008BF43F001031837BA4208BF43F0010386
:10C370001837BA4208BF43F001031837BA4208BF62
:10C3800043F0010307F55677BA4208BF43F00103B3
:10C390001837BA4208BF43F001031837BA4208BF42
:10C3A00043F001031837BA4208BF43F001031837BE
:10C3B000BA4208BF43F001031837BA4208BF43F03E
:10C3C00001031837BA4208BF43F00103002B50D1D4
:10C3D0003A4B9A424DD03A4B3A498A4218BF9A4258
:10C3E00001F114010CBF012300238A4208BF43F06E
:10C3F000010314318A4208BF43F0010314318A4219
:10C4000008BF43F0010314318A4208BF43F001031F
:10C4100014318A4208BF43F001031BB92A4B9A42E8
:10C4200040F0DA850020F421284B8AF8A800022089
:10C4300001FB0981134481F8A9001421B3FBF1F336
:10C44000116883402248084042F2A0510143284627
:10C450001160CAF8D030F4F7C5FFDAF8D03003F035
:10C460001F0201239340436050E08B668AF86030DE
:10C4700042E60020F4238AF8A800022003FB098387
:10C4800083F8A900136823F00103136027E000BFBD
:10C490000020024000600258006302580010005C57
:10C4A00003C0F0FFFDEEFFFFC0FFFE3F00F8C32515
:10C4B000602B00244000024058000240B8040240B3
:10C4C000085402581C54025894540258F8ABFDA763
:10C4D0000F00FEFF33685B1A052B00F247821368DA
:10C4E000DB07F7D4136828467E4919407E4B0B437F
:10C4F0001360536923F007035361F4F773FFDAF80D
:10C50000D03003F01F023F2393408360DAF8742099
:10C51000764B77498A4218BF9A4201F118010CBF45
:10C52000012300238A4208BF43F0010318318A42E5
:10C5300008BF43F0010318318A4208BF43F00103EA
:10C5400018318A4208BF43F0010318318A4208BFFC
:10C5500043F0010318318A4208BF43F0010301F59B
:10C5600056718A4208BF43F0010318318A4208BF5E
:10C5700043F0010318318A4208BF43F00103183128
:10C580008A4208BF43F0010318318A4208BF43F0D2
:10C59000010318318A4208BF43F0010318318A426F
:10C5A00008BF43F001035349511A484248415249D8
:10C5B0008A4208BF43F00103504900900343501AD8
:10C5C0001431D0F1000CA2EB010701F114014CEB86
:10C5D000000CD7F1000EA2EB01004CEA03034EEB76
:10C5E000070E41424EEA0303414145480B43019186
:10C5F0004449571A794279410B430291111A484232
:10C6000048414149571A0343794279413F4FBA4261
:10C61000039114BF002701270B4301D1002F4FD0F6
:10C62000009B019943EA0C034EEA030319430B46AE
:10C6300002991943D3B20843039901430F4300F011
:10C6400061841422083BB3FBF2F3314A1A4403F02D
:10C650001F039200CAF8D420012202FA03F3CAF899
:10C66000DC302C4BCAF8D830DAF87C30802B00F064
:10C670008881DAF87820DAF8D430D1B2013ADAE9F0
:10C68000360C072A1960C0F804C000F283814A1EE4
:10C69000072A0ED8002F00F0A6841F4B0B449B00E6
:10C6A000CAF8E0301D4BCAF8E43001239340CAF8C1
:10C6B000E830DAF8E03000221A60DAE939325A60FC
:10C6C000F4230122002103FB09839646C3F8C81016
:10C6D00083F8A9200AF11003CAF85C50CAF8AC30FC
:10C6E0000F4B26E03F8010FE002D0200100002409C
:10C6F0002800024008540258B80402401C54025852
:10C700006C54025858540258805402589454025899
:10C7100000960016805802583F960016405902585D
:10C72000546300240EF1010E0C33BEF1070F00F02C
:10C730007B815A7D002AF5D093F90D004FFA89F2DA
:10C740009042EFD1AE4A611C9AF8600002EB84047B
:10C7500000220128C9B2D4F8E0509C7D06920094D2
:10C760001A693FF47EACDAF810400120A7688AF815
:10C7700060007F0700F1F981C2F313070197002FD2
:10C7800040F06D82C2F38467B840970ED4F81CC0A5
:10C7900007F01F0730344CEA00004FEA951C05F003
:10C7A0001F0544F8140C0CF00C0C1F20AF4000FACD
:10C7B00005F55CF8040020EA05053D434CF80450FB
:10C7C000DAF810008568846805F0040504F00804B0
:10C7D0002C4341D1C2F30454009FD50D143007FA05
:10C7E00004FC072705F00405A7402C5824EA070499
:10C7F00044EA0C042C508348006800F07040B0F10B
:10C80000805FDAF81000C46800D0C468046E950632
:10C8100004F0F844B4EB826F03D1046E24F00044BA
:10C820000466446E04F0F844A54203D1446E24F03B
:10C8300000444466846E04F0F844A54203D1846E3B
:10C8400024F000448466C46E04F0F844A54203D189
:10C85000C46E24F00044C4668468E40709D4D0F8A8
:10C86000C040002A019D24EA0504C0F8C040C0F27F
:10C87000398200220C468AF8602053E79968C8077D
:10C880007FF514AD996801F00D01012900F0888051
:10C89000536E43F010035366936E43F001039366A7
:10C8A000F423002103FB09835A6E42F010025A66FA
:10C8B0008AF86010FFF7D5BB059A01320592059AF8
:10C8C000AA42FFF403ADF422002102FB0982536E59
:10C8D00023F0120343F0100353668AF86010FFF749
:10C8E000C0BBD168484B0B40DAF8441043F0030357
:10C8F000D360136923F001031361136923F07043BC
:10C900000B431361414B9A4268D003F580739A42FE
:10C9100064D03F4B9B6813F4403F14BF01230023B6
:10C92000002B00F03A81F4F73BFFDAF81430B3F54E
:10C93000003F00F00782B3F5403F00F0B281B3F54D
:10C94000803F00F0FF812F4B1A6841F20303B3EBE5
:10C95000124FC0F079812F4B984240F29A81DAF859
:10C9600010309A6842F480729A607AE4F4232022AC
:10C9700003FB0983C3F8C820032283F8A920FFF72B
:10C9800070BB0023DAF8D420CAF878301360DAE9F3
:10C9900036325A600023CAE93833CAF8E8308FE6E5
:10C9A00099681D4A1D4E0A4042F002029A60032215
:10C9B0001A6031689A68D0077FF578AC3268521AED
:10C9C000022AF7D9F42303FB09835A6E42F01002BE
:10C9D0005A669A6E42F001029A6661E7104B9B68B4
:10C9E00013F4403F14BF0123002399E7074B0D497F
:10C9F0009B6889680B43DF073FF51FAC084916E4C5
:10CA0000E8B20B080010005CFCBFFFFF00200240F2
:10CA100000630258002D3101C0FFFF7F602B00240E
:10CA20000023024000210240DAF810009E4B984299
:10CA300000F0A78003F58073984200F0A2809B4924
:10CA40008B68826852073FF50CAB9AF86020012A88
:10CA50003FF407AB03F01F030122DAF8F050092B73
:10CA60008AF8602000F2888040F22122DA40D7075D
:10CA700040F182808268D40723D484688C4A1442AF
:10CA800040F0758184688B4A224042F00102826046
:10CA900034688A68D10602D0874A904211D085490D
:10CAA0000CE08268D20704D482680A4042F0010296
:10CAB00082603268121B022A00F259810268D7078D
:10CAC000EFD5F4217D4A7C4C01FB0981A0424E6EDA
:10CAD00002EA060242F480724A6600D133B9F423B6
:10CAE00003FB09835A6E22F480125A66F42303FB77
:10CAF00009835A6E12F4805200F037819A6E22F048
:10CB000006029A66DAF85C1000246D4BCB636D4B1D
:10CB10000B646D4BCB641C23036043688AF8604050
:10CB200043F010034360C268DAF83C3022F003029D
:10CB30001343C36091F83430012B0CD0012381F8EA
:10CB4000343091F83530012B00F037814FF4006319
:10CB500081F834404B65DAF81020564B91680B4051
:10CB600043F004039360FFF77CBAF42303FB0983CB
:10CB70005A6E42F020025A6600238AF86030FFF7AE
:10CB800070BA52495CE7196BDAF8282021F00F01DE
:10CB9000013A0A431A63FFF76DBB4D4A936D03F4E4
:10CBA0004033B3F5803F00F00181B3F5003F00F062
:10CBB000EF80002B00F0E780DAF81430B3F5101F97
:10CBC00000F09E810AD8B3F5E01F00F0D88122D989
:10CBD000B3F5001F7FF4B7AE4009B4E6B3F5201FEC
:10CBE00000F0F681B3F5301F7FF4ADAE394B1A6813
:10CBF00041F20303B3EB124F4BD2374BB3EB102F81
:10CC000025D2DAF810309A6822F4407242F4807229
:10CC10009A60FFF726BBB3F5801F07D00BD9B3F599
:10CC2000A01F03D0B3F5C01F7FF48DAE9B0C5B003B
:10CC3000B0FBF3F087E6B3F5002FF7D023F4002222
:10CC4000B2F5802FF2D07EE6234B984210D8DAF866
:10CC500010309A6822F440729A60FFF702BB92FA91
:10CC6000A2F7B7FA87F707F01F07B840970E8DE5D0
:10CC70001A4B9842C5D91A4B9842DAF810309A6884
:10CC800000F25A8122F4407242F400729A60FFF777
:10CC9000E8BADAF810309A6822F480729A60FFF7E6
:10CCA000E0BA80084FE600BF00200240006302584F
:10CCB0003F000080C0FFFF7F00210240FEF0FFFF29
:10CCC000010004085500040859000408002302402C
:10CCD000004402580010005C21BCBE0041787D0178
:10CCE00081F0FA02A74CA04230D004F58074A04233
:10CCF0002CD0A54CA54DA54FAD68A46805F0E07CEF
:10CD0000E44304F00104002C3FF42FAFA04CA242F6
:10CD100000F017819F4CA24200F06F819E4CA2420E
:10CD20007FF4A7AD6C023FF5A4AD974A90427FF423
:10CD3000A0ADBA6822F0E07242EA0C0242F480022E
:10CD4000BA6096E51B0CB0FBF3F0FCE5934C944FF6
:10CD5000A568A4F54074A46805F0E07CBF683C4376
:10CD60008E4FE44304F00104CDE79A66CAE6F4234B
:10CD700003FB09835A6E42F010025A669A6E42F023
:10CD800001029A66F8E607A8F4F748FD079813E74A
:10CD9000D36C13F040530ED0B3F1805F00F01A81D2
:10CDA000804AB3F1005F08BF104605E707A8F4F713
:10CDB000F3FD099800E77C48FEE60B684FF0140C81
:10CDC0007A4A40307A4E0CFB05FC0225794FB3427B
:10CDD00018BF934206F1300681F835500CBF01228E
:10CDE00000224C65B34208BF42F001021836724C73
:10CDF000B34208BF42F001021836B34208BF42F006
:10CE000001021836B34208BF42F0010206F5567619
:10CE1000B34208BF42F001021836B34208BF42F0E5
:10CE200001021836B34208BF42F001021836B3427D
:10CE300008BF42F001021836B34208BF42F00102B7
:10CE40001836B34208BF42F001021836B34208BF99
:10CE500042F00102A34208BF42F00102A4F595642A
:10CE6000BB4218BFA3420CBF0127002702D0002AF3
:10CE700000F0D7801C6824F001041C608C6D0094C5
:10CE8000002F00F0FA80D1E919466660CE6E16B127
:10CE9000D1E91C456560CC6D009D04F01F0E3F2458
:10CEA00004FA0EF4AC601C6824F480241C608C68C6
:10CEB000C3F804C0402C00F0B0809860C3F80CB0F8
:10CEC00017B9002A00F0F380186820F01E0040F027
:10CED00016001860186840F008001860096E0868AD
:10CEE000C40303D5086840F4807008601EB131683F
:10CEF00041F4807131601A6842F001021A602AE63A
:10CF0000800920E52D49103B11441822A829B3FBC4
:10CF1000F2F300D808332A4A1A4403F01F039200A0
:10CF2000CAF8D420012202FA03F3CAF8DC30254BF8
:10CF3000CAF8D830FFF798BB42F440729A60FFF706
:10CF400090B92A023FF595AC0F4A90427FF491AC1C
:10CF50001D4A1068BA6822F0E07242EA0C0242F4FC
:10CF60000002BA60194AB0FBF2F25200069202E0E7
:10CF7000069A013A0692069A002AF9D179E4000944
:10CF8000E1E400BF00200240006002580063025844
:10CF9000000084CB000052C70000B8CF002302403D
:10CFA0000021024040787D010090D00358000240EB
:10CFB0004000024028000240B8040240F0FBFDBFE0
:10CFC000008200108008024000000024400D030091
:10CFD000C009B8E45348EFE54023C0F8C83080F8F2
:10CFE000A9C0FFF73EB8504B0B449B00CAF8E03095
:10CFF0004E4BCAF8E430FFF758BBED013FF539ACB2
:10D000004B4A90427FF435ACBA6822F0E07242EAB3
:10D010000C0242F08072BA602BE4C3F808B0D8600A
:10D020004EE7444C444DAB4218BFA34205F12805DE
:10D030000CBF01240024AB4208BF44F001041435A6
:10D04000AB4208BF44F001041435AB4208BF44F0C2
:10D0500001041435AB4208BF44F001041D6825F0FB
:10D0600001051D60354DAB4208BF44F001048D6DD4
:10D07000009514B9324CA34219D1D1E91946666022
:10D08000CE6E16B1D1E91C456560002A7FF403AF6E
:10D09000CC6D009D04F01F060124B4406C608C68C8
:10D0A000C3F804C0402C38D09860C3F80CB02148B5
:10D0B000214CA34218BF834204F128040CBF012075
:10D0C0000020A34208BF40F001001434A34208BF6F
:10D0D00040F001001C6824F00E0444F00A041C60B7
:10D0E000184CA34208BF40F001001434A34208BF0B
:10D0F00040F001001434A34208BF40F001001C6856
:10D1000044F004041C600E4CA34208BF40F0010030
:10D1100000283FF4F0AECE6EE0E6C3F808B0D86069
:10D12000C5E700BF00093D003F82001040090240F2
:10D13000006002581C540258085402588054025887
:10D140009454025858540258DFED0A7AB7EE007A28
:10D150000023C0ED020A20EE270A0360C7EE007A22
:10D1600030EEA77AC0ED017AC0EE877AC0ED037A7F
:10D17000704700BFDB0FC9400369426830B5484DB6
:10D1800083B00BB9002A65D0C46A0133D0ED067AAA
:10D190000361631C77EE807A012BC362C0ED067ACF
:10D1A00048D0D0ED075A07EE903A90ED097A30EE6C
:10D1B000656A2968F8EEE76A8A1A8168C6EE267AF7
:10D1C0008A4277EEA57A30EE670AC0ED087AC0EDA4
:10D1D000077AF0EE477AE6EE007AC0ED0A7AC0ED03
:10D1E000097A01D803B030BD012B4BDD07EE104AA0
:10D1F000B8EEC77A87EE870AB5EEC00AF1EE10FAEC
:10D2000043DBB5EE400AF1EE10FA41D4F1EEC07AFC
:10D21000F4EE677AF1EE10FA37D690ED057AB4EEB7
:10D22000E77AF1EE10FA18D5037B23B303230370DA
:10D2300003B030BD2B6881689A1ADFED1A7A80ED51
:10D24000080A8A4280ED070AC0ED097ACAD9B0EE11
:10D25000670ADBE72A68426096E7D0ED047A02238A
:10D26000D0ED066AF8EE677A037086EEA77A80ED55
:10D27000067A03B030BD296800220361C3624160B1
:10D280008261AFE79FED070AC0E7DFED067AC4E7EA
:10D29000019067F045F80198F0EE407AB8E700BFDA
:10D2A0004C3E00240000000070B50346044600F127
:10D2B000480500262DED028B82B0DA6AB1EC017AC6
:10D2C000D3ED067A013277EE877A012ADA62C3ED6E
:10D2D000067A74D093ED075A07EE902A93ED096A07
:10D2E00077EE455AF8EEE77AC5EEA76A76EE857ACC
:10D2F00037EE677AC3ED087AC3ED077AF0EE467A27
:10D30000E5EE877AC3ED0A7AC3ED097A1833AB42AA
:10D31000D3D102693D4E01324168336802615B1A24
:10D320008268934247D900259FED398AE36A012B31
:10D330004BDD013B94ED0A7A07EE903AF8EEE77A7E
:10D3400087EE270AB5EEC00AF1EE10FA53DBB5EE10
:10D35000400AF1EE10FA51D4F1EEC07AF4EE677A99
:10D36000F1EE10FA47D690ED057A01351834B4EE97
:10D37000E77AF1EE10FA2BD4022DD7DDB4EEE77A7E
:10D38000F1EE10FA24D4D0ED047A0223D0ED066A2F
:10D39000F8EE677A90ED0C7AD0ED125A037086EEB3
:10D3A000A76AC7EE276A85EEA77A80ED066AC0ED08
:10D3B0000C6A80ED127A02B0BDEC028B70BD83ED79
:10D3C000087A83ED077A5E62A0E7B0EE480AC3E709
:10D3D000037B2BB10323037002B0BDEC028B70BD45
:10D3E000002231680361C362416082610263436469
:10D3F0008264C365DFE7F0EE487AB4E7019066F037
:10D400008FFF0198F0EE407AA8E700BF4C3E002461
:10D4100000000000F0EEC07AB0EEE07AB4EEE77AF9
:10D42000F1EE10FA77FE275AF5EE405AF1EE10FAB7
:10D430004CD0B4EEE77A9FED273A9FED272AB7EE5E
:10D44000005A9FED264AF1EE10FADFED254ADFED96
:10D45000252ADFED253A54BFF0EE671AF0EE471AA1
:10D460009FED226AC1EEA56AF0EE435AE6EE825ABB
:10D47000E6EEA23AA6EEA54AF0EE455AB0EE645AA0
:10D48000E6EEA35AA6EE845AA6EE856AB1EE466A87
:10D49000C6EE256AB4EEE77AF1EE10FA03D5DFEDB9
:10D4A000147A77EEE66AF5EEC00AF1EE10FA03D5CB
:10D4B000DFED107A77EEE66AB5EEC00AF1EE10FA0B
:10D4C00048BFF1EE666AB0EE660A7047DFED0A6AA1
:10D4D000E0E700BFE3B59EBE39094E3D88FA16BEAF
:10D4E00045FE7FBF99FB243F69A2163EA7DFA8B483
:10D4F000DB0FC93FDB0F4940A7DFA834D1ED007A2D
:10D50000F7EE002A90ED043AD0ED053AA7EEA73ADF
:10D5100090ED064AD0ED074A90ED085A90ED096A61
:10D52000D0ED0A6A90ED0B7A80ED043A91ED003A65
:10D53000D1ED015AD0ED0C7AE3EE253AC0ED053A73
:10D54000D1ED003AD1ED025AA3EEA54A80ED064A8C
:10D55000D1ED005A74EEA54AC0ED074AD1ED014A5B
:10D56000D1ED005AA4EEA55A80ED085A91ED015A6A
:10D57000A5EE056A80ED096AD1ED015A91ED026AC6
:10D58000E5EE866AC0ED0A6AD1ED016A37EE267AC9
:10D5900080ED0B7AD1ED026A91ED007AE6EE877AA2
:10D5A000C0ED0C7A91ED027AD1ED017A90ED0D3A51
:10D5B000D0ED0E3AA7EE273A90ED0F4AD0ED104A83
:10D5C00090ED115AD0ED127AD0ED135A90ED006A19
:10D5D00080ED0D3A75EEA25A91ED023AD0ED016A56
:10D5E000E3EE033A90ED027AC0ED0E3AD1ED023A45
:10D5F00034EE234A80ED0F4A91ED004A74EE844ADE
:10D60000C0ED104AD1ED014A35EE245A80ED115A91
:10D6100091ED025AC0ED135A77EE857AC0ED127A79
:10D62000D1ED017AD1ED005A67EEA77A91ED025A59
:10D63000E5EEA57AE5EE057AA5EEA76A80ED006A2B
:10D6400091ED016AE6EE276AC0ED016AD1ED026A4A
:10D65000A6EEA77A80ED027A90ED037A77EE277A2C
:10D66000C0ED037A704700BF2DE9F04F00F1100ABA
:10D6700089B0834600F1300807460546D64656462F
:10D6800084460024CDF80CA0CDE90112624628465C
:10D690007CB1D2ED007A01463B468946F3EC016A43
:10D6A000103199ED007A6345E6EEC77AC2ED007A53
:10D6B000F3D1043204307245EAD1032C04F1010A9B
:10D6C0002ED062463046ABEB050994B1D2ED047A18
:10D6D00009EB0003294600940C46F3EC016A103173
:10D6E00094ED007A8342E6EEC77AC2ED047AF3D174
:10D6F000009CD2ED046A103216ED047A10304245D7
:10D70000C6EE877AC2ED007ADFD10CF1140C08F175
:10D710000408043514360EF1100E10375446B5E7E0
:10D720000025002305A80BF1140401350593069389
:10D730000793042DDDE9022A52F8043B049316D026
:10D74000F2EC017A04A95346C0ED007AB1EC017AFB
:10D75000F3EC016AE6EEC77AA342C0ED007AF5D198
:10D7600001350AF1100A04301434042DE8D1019A6D
:10D7700008AE02250BF14004103276ED017A022D3D
:10D780002046A2F1040142ED017A1FD02346F3ECBA
:10D79000016AB2EC017A9842E6EEC77AC1ED007AEE
:10D7A000F5D154ED016A6B1C87EEA67A81ED007A03
:10D7B00013D0013D0A4676ED017A143C022DA0F10A
:10D7C0001000A2F1040142ED017ADFD154ED016AAB
:10D7D00087EEA67A02ED017AEBE709B0BDE8F08F9B
:10D7E00010B584B00C46B6EE006A024669461030A9
:10D7F000FFF73AFFDDED007A9DED017A67EE867A5C
:10D80000DDED026A27EE067A66EE866AF4EE677A46
:10D81000C4ED007A84ED017AC4ED026AF1EE10FAEB
:10D820000CD6B4EE477AF1EE10FA12D6F4EE666A30
:10D83000F1EE10FA17D6012004B010BDF0EEE77A31
:10D840009FED0F6AF4EE467AF1EE10FAE9DD002062
:10D85000F2E7B0EEC77ADFED0A7AB4EE677AF1EE5E
:10D8600010FAE3DDF3E7F0EEE66ADFED057AF4EEB9
:10D87000676AF1EE10FAD4BF01200020DCE700BF98
:10D88000FFFF7F7F60EEA00AE0EE000AF5EEC00A1F
:10D89000F1EE10FA0CDBF5EE400AF1EE10FA0AD4C4
:10D8A000B1EEE00AB4EE400AF1EE10FA00D670478D
:10D8B0009FED070A7047B0EE600A08B566F030FDCC
:10D8C000B4EE400AF1EE10FA68BF9FED010A08BD00
:10D8D0000000000060EEA00AE0EE000AE1EE010A9E
:10D8E000F5EEC00AF1EE10FA0CDBF5EE400AF1EEAF
:10D8F00010FA0AD4B1EEE00AB4EE400AF1EE10FAE2
:10D9000000D670479FED070A7047B0EE600A08B571
:10D9100066F006FDB4EE400AF1EE10FA68BF9FED26
:10D92000010A08BD00000000DFED257AB4EEE70A29
:10D93000F1EE10FA08DD9FED237A30EE470AB4EEDF
:10D94000E70AF1EE10FAF8DCDFED1F7AB4EEE70A31
:10D95000F1EE10FA08D59FED1B7A30EE070AB4EE0F
:10D96000E70AF1EE10FAF8D4DFED187AB4EEE70A20
:10D97000F1EE10FA18DD30EE670A37EEC00A60EEFD
:10D98000007ADFED135A9FED136ADFED136AA7EEFD
:10D99000A56A9FED127A60EE275AE7EE866AA7EE37
:10D9A000A67AA5EE870A70479FED0D7AB4EEC70AF6
:10D9B000F1EE10FAE3D530EE270A37EE400ADEE743
:10D9C000DB0F4940DB0FC940DB0F49C0DB0FC93F0C
:10D9D0009A7C2E36FAAF4FB93587083CA4AA2ABEE6
:10D9E000DB0FC9BF10B53E4CB4FBF2F4A1420DD31E
:10D9F00000234FF07E52436083600260C360036186
:10DA00000023836143610362C36110BD07EE902A66
:10DA1000DFED345AB7EE006ADFED336AB8EE677AAD
:10DA200007EE901AB0EE405AF8EE677A27EE257AA4
:10DA300067EEA67AC6EE076AC7EEA64AFDEEE47A5E
:10DA400017EE902A2032402A47D8B0EE640AFFF73A
:10DA50006BFFB0EE404A9FED250A34EE800AFDEEE2
:10DA6000C07A17EE902A2032402A31D8FFF75CFFA7
:10DA7000F8EE006A60EE266A012B24D0F7EE007AF9
:10DA8000F6EE005A37EEC00A60EE255A35EE055A1A
:10DA9000B7EE007A84EE056A76EE077A37EE467ABC
:10DAA00080EE275A85EEA76AC6EEA75AC7EE276A08
:10DAB00080ED015A80ED006A80ED026AC0ED035AE4
:10DAC000C0ED046A9CE7F7EE005AB0EE660ADDE7A7
:10DAD000DFED076A9FED070ACEE79FED064ABAE73A
:10DAE00020A10700BD378635DB0FC940DB0FC93FDA
:10DAF0000000008000000000DFED077A30EE270A0A
:10DB0000FDEEC07A17EE903A2033402B00D80BE799
:10DB10009FED020A704700BFDB0FC93F0000000005
:10DB20009FED530A91ED005A35EE000A08B5FDEE5F
:10DB3000C07A17EE903A2033402B7DD8FFF7F4FEE1
:10DB4000FDEEC57AB0EE403A17EE903A2033402B06
:10DB50007BD8B0EE450AFFF7E7FEB0EE405AF1EE93
:10DB6000402A91ED014A9FED420A34EE000AFDEE93
:10DB7000C07A17EE903A2033402B74D8FFF7D4FECA
:10DB8000F0EE404AB1EE402AFDEEC47A17EE903A2C
:10DB90002033402B64D8B0EE440AFFF7C5FEB0EE48
:10DBA000404AD1ED021A9FED320A31EE800AFDEEB5
:10DBB000C07A17EE903A2033402B4ED8FFF7B4FED0
:10DBC000F0EE403AFDEEE17A17EE903A2033402B2A
:10DBD00040D8B0EE610AFFF7A7FE63EE836A80EDDE
:10DBE000024A20EE037A63EE857AB0EE666A20EE92
:10DBF000055AF0EE475A63EEA43AA5EE446AE7EE02
:10DC0000845AA6EEC45AC0ED003AE7EE047A62EEFA
:10DC1000A42A22EE000A64EE834A80ED046AC0ED75
:10DC2000052A80ED010AC0ED084AC0ED035A80EDD7
:10DC3000065AC0ED077A08BDFDEEC57A9FED0D3A94
:10DC400017EE903A2033402B83D9DFED0B2A9FED5E
:10DC5000095A86E79FED070ABFE7DFED063AB1E70D
:10DC60009FED044A9DE79FED042ADFED024A8BE712
:10DC7000DB0FC93F00000000000000802DE9F04FDD
:10DC800083B0054688469DF830400D9E002C0192D9
:10DC900014BF4FF030094FF020091C1E48DB16F866
:10DCA000010B014600286CD0002C65D04FF0000A13
:10DCB000324601E0002C34D012F8013B2746013CEB
:10DCC000002BF7D1BAF1000F3AD1023F002C67D0F8
:10DCD000BA4645450AF1FF3A4946284601D2019B1A
:10DCE0009847BAF1FF3FF4D10D9A23463C1B1078B8
:10DCF000014600283ED04FF0000A01339F1B4545E6
:10DD000006EB070B284601D2019B984716F8011B2A
:10DD10000029F4D1BAF1000F16D1584603B0BDE87E
:10DD2000F08FBAF1000F33D0014678B32346E4E711
:10DD300016F8010B634278B31C464FF0010AB7E7AF
:10DD400001460028D9D18346002C04F1FF36E4DDDA
:10DD50003446454506F1FF364946284601D2019B27
:10DD60009847731CF5D10BF1010BA344584603B03F
:10DD7000BDE8F08F9B46D0E723464FF0FF349A462C
:10DD8000BBE7671E002CA3D1A346C6E78346C4E7C2
:10DD900023464FF0FF34ABE7E64383463446D8E7EB
:10DDA00023463C46A4E700BF0FB430B583B00B4C0C
:10DDB00006AB53F8042BD4E94B01019362F0F8FC55
:10DDC0000546606803685B6998470028F9D02846D3
:10DDD00003B0BDE8304004B0704700BF806200244B
:10DDE0000EB410B583B00446084905AB01A853F83A
:10DDF000042BCDE9003462F0DBFC019B00221A7099
:10DE000003B0BDE8104003B0704700BFA9B70408D5
:10DE10000CB4F0B53C4CADF5277DD4F83431002B73
:10DE20004CD094F83C31994240D8384B4FF47A7139
:10DE3000374A1B68A2FB030206A8920901FB1233B2
:10DE40003449FFF7CDFF06ABAC9A0646034432498E
:10DE500001A80193ADAB009362F0AAFC019B0246BE
:10DE60000A2000215D1C01951870019BD4F83451E3
:10DE7000581C0190197035B32B681B6A1BB12846DA
:10DE80009847D4F834519DF8181049B10DF1190490
:10DE90002B6828461B68984714F8011B0029F7D106
:10DEA0000DF5277DBDE8F04002B070470123D4F89E
:10DEB000402103FA00F01042B7D1F1E7D4F838312D
:10DEC000002BAED1ECE7D4F83871002FE8D09019D0
:10DED00026ABFD2206A9841C1846CDE90455ADF8F1
:10DEE0001020224668F022FF02220346044402A9C1
:10DEF0003846CDE902342FF0A1FF0DF5277DBDE8AE
:10DF0000F04002B0704700BF806200244C3E002405
:10DF1000D34D621044510C089DB7040830B54FF43E
:10DF2000004087B02EF0A0F958B14FF400410446EC
:10DF30002EF0C0F9022806D1226848F201039A4265
:10DF400025D007B030BD94F9040000234FF46121BF
:10DF500002241A460293CDE900144FF400412EF03A
:10DF6000B3F91D4BC3F834010028EAD01B4A1C4BFF
:10DF70001C481D491D4CCDE90332CDE901101C4B55
:10DF800002211C4A00200094FFF742FFD9E7124CFF
:10DF900000254FF4004084F8D8535DF063F9002861
:10DFA000CFD0D4F8443183420AD0D4F8203283420F
:10DFB0000BD0D4F8FC3298420AD0C4F83851C0E7EC
:10DFC00004F5A273C4F83831D0E704F50873F9E713
:10DFD00004F53F73F6E700BF8062002468510C0827
:10DFE00074510C0880510C088C510C0894510C0889
:10DFF00020510C0850510C0838B5184C0330D4F897
:10E00000DC5305EB9003B3F5007F18D804EB8101D6
:10E0100020F00302C4F8DC3304F57874D1F8E00B87
:10E02000C3F5007304EB850510449B000C4AC1F84E
:10E03000E00B04210020FFF7EBFE284638BD00214D
:10E04000084A08460D46FFF7E3FED4F8683C284628
:10E0500043F00073C4F8683C38BD00BF8062002400
:10E06000A8510C08CC510C0838B505680446EB697A
:10E07000F3B1987800B938BDB3F90A20012007EE52
:10E08000902AF8EEE77AC4ED057AB3F90C2007EE92
:10E09000902AF8EEE77AF1EE677AC4ED047AB3F9E4
:10E0A0000E3007EE903AF8EEE77AC4ED067A38BD06
:10E0B00009211420FFF7A0FF0346E861D9E700BF5C
:10E0C00038B505680446EB69E3B1987800B938BD06
:10E0D000B3F90420012007EE902AF8EEE77AC4EDA8
:10E0E000047AB3F9062007EE902AF8EEE77AC4ED39
:10E0F000057AB3F9083007EE903AF8EEE77AC4ED06
:10E10000067A38BD09211420FFF776FF0346E8613F
:10E11000DBE700BF38B505680446EB69E3B19878E2
:10E1200000B938BD9A880120D2BA07EE902AF8EEDD
:10E13000E77AC4ED047ADA88D2BA07EE902AF8EECC
:10E14000E77AC4ED057A1B89DBBA07EE903AF8EE60
:10E15000E77AC4ED067A38BD09211420FFF74CFF99
:10E160000346E861DBE700BF38B505680C46EB699C
:10E170007BB1987800B938BD5B890120084ADBBAC9
:10E1800082FB0312DB17C3EB221303F26D13238010
:10E1900038BD09211420FFF72FFF0346E861E8E7A7
:10E1A00079787878944603EB43032DE9F0411CF825
:10E1B000068B86B0144602EB430315464FFA88F6E9
:10E1C000821B9CF80070002AA0EB070EB8BF5242D9
:10E1D000BEF1000FB8BFCEF1000E964501DA6546DC
:10E1E0007EB20CF1060C6345EAD19F1F6B8803E0F9
:10E1F000A74218D014F8068FB0459C46F8D1CA1A29
:10E20000B4F80280002AA1EB080EB8BF5242BEF15A
:10E21000000FB8BFCEF1000E7245E9DDA7424346BC
:10E220002546C446E6D16C790346CDF808C02A7865
:10E230000494287901920390012000910321034A5C
:10E24000FFF7E6FD284606B0BDE8F081DC510C087A
:10E2500003681A46591C016012F8021B02605878C4
:10E2600041EA0020704700BF02681146531C03605A
:10E27000D31C11F802CB01605178036093781B0422
:10E2800043EA0123111D43EA0C030160D07843EAFD
:10E290000060704712B370B50446864604E0981BD0
:10E2A00017D114EB0C0C15D01EF8013BA3F1410063
:10E2B000A2EB0E0C192811F8010BA0F1410598BF33
:10E2C000203300F12006192DE9D91B1A04D10028AA
:10E2D000E7D170BD604670BD184670BD10467047EE
:10E2E000028840F2B55CA2F5FA6210B54FEA920ED0
:10E2F000817802F00302C3780139124C02EB42022A
:10E30000013B01EB82020CFB0E33017904EB42026C
:10E310008479B2F8202113444279008903EB430346
:10E3200001EBC3030021C3EB031302EB8303064A93
:10E33000C3EB0313224402EB83024FF47A73C2FB54
:10E34000030110BDE8B20B0880436D382DE9F041A0
:10E3500017461E4605464FF47A720023384631466A
:10E36000454C63F02FFB4549454A0144454882FB33
:10E3700001C34FEAE17C0B44CCEB631382FB03C285
:10E380004FEAE37C1A44CCEB621284FB02C44FEAEE
:10E39000E27CCCEBA40C80FB0C404FEAEC74C4EBA9
:10E3A000E010C3EB0314A1EB8401A971C2EB0211CD
:10E3B000A3EB81036B710CEB4C03A2EBC30240F2A5
:10E3C000B55303FB10CC80002A71BCF5896F45DA88
:10E3D00040F2DA239C4548DCBCF5B77F2A4BB4BF3A
:10E3E0000022012202EB42014FEA420803EBC10383
:10E3F00091B2B3F8363108EB020E244C04EBCE0494
:10E400004FF00B0E163401E034F8023D634520DD79
:10E41000BEF1010EF8D11C4B42444FF0010E03EB4C
:10E42000C202B2F8203100F5FA600CF1010C4FF491
:10E430007A7285F802E00844ACEB030C3146002305
:10E440002880384685F803C063F0BCFA2A81BDE80D
:10E45000F0810EF1010E5FFA8EFEE4E7032140F237
:10E4600096534FF006080A46C5E7022140F22943B9
:10E470004FF004080A46BEE7ABAAAA2A80BC92C79E
:10E480008988888873B06D16E8B20B0808B40B0849
:10E4900070B42D4D8DB006468C466C460FCD0FC422
:10E4A0000FCD0FC495E80F0084E80F00B3070DD11E
:10E4B000264B274A06FB03F3B2EBB30F42D3254AA0
:10E4C000B2EB331F2CBF1D241C2400E01C24731E40
:10E4D00040F26D120194002B194606FB02F2B8BF00
:10E4E000B11C1D4E02EBA1021C4981FB0301DB178D
:10E4F000ADF1040000EB8C05A3EB6110C3EBE1135D
:10E5000001A902441A44253286FB0230D317104475
:10E51000C3EBA000C0EBC000101A01E051F8044F9B
:10E5200003198D4286FB03024FEAE3701A44C0EBE5
:10E53000A200C0EBC000A3EB0000EFD1201A0DB089
:10E5400070BC70471D24C2E768B40B08295C8FC2F9
:10E55000285C8F020AD7A300932449921F85EB51B0
:10E5600008B50E4BD3F8702CD3F8743C52EA030C68
:10E570000AD10146002340F2011218460B804A805E
:10E580008B808B710B8108BD054909688A1843F19E
:10E590000003FFF7DBFE012008BD00BF80620024FE
:10E5A0004C3E002430B5144D83B00446D5F8702C91
:10E5B000D5F8743C52EA03010AD1002340F201125B
:10E5C000184623806280A380A371238103B030BDED
:10E5D0000A4909688A1843F10003FFF7B7FEB5F846
:10E5E000783C20460DF106022146ADF806305DF07C
:10E5F00065FD012003B030BD806200244C3E002444
:10E600008842F0B54FF0010439D301FB04F4B0FBAC
:10E61000F4FC8C45F9D26CB30025BCF1000F04FB6F
:10E620001C00B4FBF1F7D4BF0026012665B95EB922
:10E63000A142354618D99E460CF1300C0EF801CB9C
:10E6400000238EF80030F0BDBCF1090F10DD002A68
:10E6500014BF372657269E46B444A14205F1010552
:10E660000EF801CB7346EBD83C46B0FBF7FCD4E781
:10E670003026F0E79E4600238EF80030F0BD844639
:10E68000CAE700BF90420B462DE9F041B0FBF2F61D
:10E690000446154608D2124A05FB16441846135D77
:10E6A00000F8013BBDE8F0819642B6FBF2F706D2D6
:10E6B0000B4A05FB1767D15D03F8011BECE7BA4273
:10E6C000B7FBF2F807D905FB1878054A12F80810CD
:10E6D00003F8011BEDE74046FFF7D4FF0346F2E7DE
:10E6E00018520C08B5EEC00ADFED357A0023F1EEC2
:10E6F00010FA70B5C8BF30EE270A86B0D8BF30EE2A
:10E70000670ADFED307A054603A902936E4620EED4
:10E71000270ACDE90033FDEEC07A17EE904A84EA6D
:10E72000E470A0EBE4705EF0C9FC002C03A8ACBF61
:10E7300020232D238DF8003062F07CFA012829D0A7
:10E74000022833D003281DD003A930466BF0E6FB26
:10E75000304662F06FFA044631462846033CE4B284
:10E76000224668F0E3FA002328462B5562F062FA4D
:10E770002E22431C31192A54E8186BF0EBFB284673
:10E7800006B070BD302303A930468DF801306BF020
:10E79000C5FBDDE7302303A930468DF801308DF845
:10E7A00002308DF803306BF0B9FBD1E7302303A9B9
:10E7B00030468DF801308DF802306BF0AFFBC7E7C3
:10E7C0006F12033A00007A440378092B01D0202B02
:10E7D00005D110F8013F202BFBD0092BF9D02D2BB0
:10E7E00063D02B2BB7EE000A08BF01300278A2F1EC
:10E7F0003003D9B2092961D8F2EE046ADFED4D7A0F
:10E8000007EE103A10F8012FB8EEC77AA2F13003E4
:10E81000D9B2A7EEA67A0929F0EE477AF0D92E2AC6
:10E8200050D0037803F0DF03452B3BD110B442787E
:10E830002D2A73D02B2A62D0A2F130030130092B8C
:10E8400063D80024002303EB830302EB430310F897
:10E85000012FA2F13001303B0929F4D9B3F59A7F99
:10E860001A46B7EE007A28BF4FF49A72072B09D9DF
:10E870001346DFED316A083B27EE267A072BFAD8DC
:10E8800002F007022AB1F2EE046A013A27EE267A74
:10E89000FBD1002C3BD0C7EE877A5DF8044B20EE0D
:10E8A000270A704720EE270A704742780130BFEEF2
:10E8B000000AA2F13003D9B209299DD92E2ADFED31
:10E8C0001D7AAED143780130A3F13002D1B20929CB
:10E8D000A8D8B2EE047AF0EE475A06EE902A10F865
:10E8E000013FB8EEE66AA3F13002D1B2C6EE076A84
:10E8F000092927EE257A77EEA67AEED992E7827873
:10E900000230A2F13003092B9BD9B7EE007A67EEF3
:10E91000877A5DF8044B20EE270A70478278023030
:10E92000A2F13003092B01D801248BE7B7EE007A5E
:10E93000B1E700BF0000000020BCBE4C00B503786A
:10E94000202B03D110F8013F202BFBD0092BF9D04D
:10E950002D2B14D04FF0010E411E002311F8012F72
:10E96000303A5FFA82FCBCF1090F03D90EFB03F0C9
:10E970005DF804FB03EB830302EB4303EEE7013096
:10E980004FF0FF3EE8E700BFA94B0022A9492DE95F
:10E99000F04F591A99B091460192CDE902313422D3
:10E9A00000210BA86AF06AFBA24AA34B0892039AC3
:10E9B0000A92029A0992DA68D60707D59F4A5A60E6
:10E9C00002F188325A60DB68DC070DD49A4BD3F829
:10E9D0000C21D50708D5994AC3F8042102F18832E1
:10E9E000C3F80421D3F80C3101227E2305A908A81D
:10E9F000CDF854908DF858208DF81430FDF766FA54
:10EA00000028C0F2AB809DF81430082241F22101A9
:10EA10001B0203E05B00013A9BB206D01804F9D553
:10EA200081EA4303013A9BB2F8D1854E06AFADF8B7
:10EA30001630844B9E4256D241F2210472883388AC
:10EA4000C2F30B058DF81D90C3F30B011B0B8DF862
:10EA50001C30AB1DADF81A10ADF81830130400F1DE
:10EA60008F800622394608A8FDF730FA002875DBAA
:10EA7000BDF8163039460DF11E0011F8012B83EA5E
:10EA80000223082213F4004F14BF84EA43035B00FF
:10EA9000013A9BB2F6D18842EFD12A46716808A8A4
:10EAA000ADF81630FDF712FA002857DB7168BDF893
:10EAB00016304819814210D00139013811F8012F60
:10EAC00083EA022308221D044CBF84EA43035B004F
:10EAD000013A9BB2F7D18842F0D1ADF81630143626
:10EAE000584B9E42AAD30222394608A8ADF8189086
:10EAF000FDF7ECF9002831DBBDF816300DF11A01F5
:10EB000041F2210217F8010B082483EA00231804BC
:10EB10004CBF82EA43035B00013C9BB2F7D1B94290
:10EB2000F0D102220DF1160108A8ADF81630FDF75C
:10EB3000CDF9002812DB1498002840F08580159844
:10EB400000280BDB9DF85830002B40F09280002805
:10EB50000DBF012200220123002301E00123002236
:10EB6000019901310229019102DC002B7FF417AFDA
:10EB70001AB1304B1B787E2B53D0052006F0D0FE07
:10EB80004FF00008C2460AF1010A0622394608A8D9
:10EB90005FFA8AFA8DF81DA0FDF798F90028DDDBF1
:10EBA000BDF8163039460DF11E0011F8012B83EA2D
:10EBB0000223082213F4004F14BF84EA43035B00CE
:10EBC000013A9BB2F6D18842EFD171682A4608A873
:10EBD000ADF8163001EB080B5946FDF777F9002820
:10EBE000BCDB0BEB0500BDF81630834512D00BF1F2
:10EBF000FF31013811F8012F83EA0223082213F4B0
:10EC0000004F14BF84EA43035B00013A9BB2F6D184
:10EC10008842EFD1BAF1030FA844ADF81630B2D153
:10EC20005DE7FCF7CFFD0028A7D019B0BDE8F08F55
:10EC3000000004080000020800200052230167457C
:10EC400098F50C0898FA0C08089B099A034493421B
:10EC500084D80CABC0F12002214618446AF00EFAA9
:10EC6000159818B90CA908A8F4F7DCFBCDE91490A5
:10EC700066E7094BDA6842F00102DA60DA68D10728
:10EC80007FF565AFD3F80C2142F00102C3F80C21E7
:10EC9000D3F80C315BE700BF0020005270B5458807
:10ECA0000B4604460021C5F30B0518462A466AF0B8
:10ECB000E5F92169084A0346914202D3074A914285
:10ECC00005D319B11846BDE87040084770BD2A4603
:10ECD000BDE8704068F02AB898FA0C0847FF0C08A5
:10ECE00010B50446C06900B110BD09211420FFF71A
:10ECF00083F9E06110BD00BF10B5164C04EB800035
:10ED0000C06820B300EB400004EB800292F9D5C04C
:10ED1000BCF1FF3F1CD092F8DD00C0B164448C20F0
:10ED200092F8DC10002394F828E1142200FB0CFC7C
:10ED3000094C0CEB0100013A714434F8100013FA4D
:10ED400080F3F6D10548A0FB0330C0F30F1010BDCF
:10ED5000002010BD8062002400000030CDCCCCCC5F
:10ED6000036810B51A790446022A03D000232360F1
:10ED7000237110BD987A04F083F80028F6D040F68D
:10ED80001A610022C1802021027204F02DF80023B4
:10ED90002360237110BD00BF2DE9F84FB84CB94D69
:10EDA000AC4250D29B4602E00C34AC424BD294F8B9
:10EDB00005C08C45F8D194F804C0844501D00028E2
:10EDC000F2D194F807C09445EED12568002D3BD0D0
:10EDD00000222C606A60AA60EA602A616A61AA6106
:10EDE000EA61217929710129A679AE60207AE8606B
:10EDF00032D0022927D1E07A04F042F894F9097060
:10EE0000A861A07A2F7404F03BF86861F8B19E4CB9
:10EE100007EB47094FEA470854F8392004EBC909C2
:10EE2000AAB199F8162002B30E21002280F806B08C
:10EE3000C17102720D2103F0D7FF6B6923B11A680B
:10EE40009B88936100E000252846BDE8F88F28469E
:10EE50000025FFF785FFF7E7E07A04F011F8627A02
:10EE6000A37AA8612A746B74EEE7B9F808005DF024
:10EE7000FBFEB9F808000122410900F01F00023929
:10EE80008240092912D8DFE811F00D0111001501A7
:10EE9000F200EA00E200DC00D400CC000A007B486B
:10EEA000D0F89C1021EA0202C0F89C2008EB07026F
:10EEB00007F1010904EBC2025FFA89F9507903F006
:10EEC000DFFF824620B140F60A3280F80890C28007
:10EED00008EB070204EBC202D07903F0D1FF20B1A6
:10EEE00040F60A5280F80890C28008EB070204EB53
:10EEF000C202907903F0C4FF20B140F60A4280F8C4
:10EF00000890C28008EB0702504608EB070A16F08B
:10EF1000040604EBC20204EBCA0A14BF4E212E21E0
:10EF2000927A03F087FF9AF8070003F0A9FF9AF896
:10EF30000B202E2103F07EFF9AF8060003F0A0FFBD
:10EF40009AF80C200E2103F075FF9AF804000028AF
:10EF500040F0EB8008EB07024D4B54F8322011686B
:10EF60009A4221F00101116000F0F98049498A427A
:10EF700000F0BC8001F580618A4240F0A6804349E0
:10EF8000D1F890C04CF4004CC1F890C0D1F890C0BA
:10EF90002CF4004CC1F890C0002E40F093804FF04C
:10EFA00000764FF08071D2F80CC04CF0004CC2F8E3
:10EFB0000CC0D2F808C02CF4F07CC2F808C013686A
:10EFC000DB0721D49368DFF8D8E003EA0E0E324B5A
:10EFD0004EEA03039360D368DB0005D4D2F800C087
:10EFE0004CF4805CC2F800C0D36831432B4E1E4005
:10EFF000314341F08861D160116821F400611160F2
:10F00000116D21F001011165002840F09F804744F7
:10F010000122686904EBC704A27500283FF40AAF17
:10F0200002E71A48D0F8881021EA0202C0F88820C6
:10F030003CE71648D0F88C1021EA0202C0F88C2078
:10F0400034E71248C16F21EA0202C2672EE70F4877
:10F05000D0F8941021EA0202C0F8942026E70B4869
:10F06000D0F8901021EA0202C0F890201EE707486D
:10F07000D0F8841021EA0202C0F8842016E700BF0D
:10F0800058040008200600082C02002400440258FE
:10F09000003001400038004007000020FFFF39D851
:10F0A000E0FFBF8F3D48D0F8981021EA0202C0F877
:10F0B0009820FBE63948D0F8801021EA0202C0F817
:10F0C0008020F3E6002631466DE735498A4254D167
:10F0D0003249D1F898C04CF4005CC1F898C0D1F81E
:10F0E00098C02CF4005CC1F898C055E72B49D1F8C2
:10F0F00090C04CF4804CC1F890C0D1F890C02CF472
:10F10000804CC1F890C027498A427FF445AF23491B
:10F11000D1F89CC04CF0200CC1F89CC0D1F89CC028
:10F120002CF0200CC1F89CC036E703F0A9FE20B1FA
:10F1300040F60A6280F80890C2800D2103F054FE68
:10F1400008EB070204EBC202107903E703F098FE14
:10F1500000283FF45CAF02688188916157E70F494E
:10F16000D1F898C04CF4805CC1F898C0D1F898C030
:10F170002CF4805CC1F898C0C5E70B498A42C2D123
:10F180000649D1F898C04CF4801CC1F898C0D1F859
:10F1900098C02CF4801CC1F898C0FDE600440258C9
:10F1A000003401400014005800500140104B70B56D
:10F1B000104CA34203D318E00C33A34215D293F8AA
:10F1C00005C08C45F8D193F804C008B18445F3D14B
:10F1D00093F807E09645EFD11D6895F804E0E64501
:10F1E000EAD12E689E42E7D100E00025284670BD96
:10F1F00058040008200600080379022B00D070474D
:10F2000010B590F9102082B008314FF0030E0020A5
:10F210004FF0010C694402EB42021C4C8DF80000D7
:10F2200054F832208DF801C08DF802308DF803E0DB
:10F2300011F808EC16498A4223D0A1F578418A4298
:10F2400021D001F580618A4205D0124B9A4214BF49
:10F250004FF0FF330323116803EB430321F0010157
:10F2600004EBC30311601969936851F82E1023F061
:10F27000E0430B439360136843F00103136002B053
:10F2800010BD0346E7E76346E5E700BF2C02002414
:10F29000003001400034014090F91030F0B503EB2C
:10F2A00043032A4E154683B056F8336004468368FC
:10F2B0009A071ED5FF2701230DF106028DF80610CF
:10F2C00030460DF107018DF80770F5F707F90123B6
:10F2D0000DF106020DF1070130468DF806508DF84C
:10F2E0000770F5F7FBF8A3689B0716D5012003B05C
:10F2F000F0BD43691BB19A88186812048261144BEF
:10F30000144A1868144BC0005768A3FB00308009EA
:10F310005368DB1B9842FBD2CCE70D4A4FF4FA70DE
:10F320000D4B12680B4900FB02F24868A3FB023246
:10F3300092094B681B1A9A42FBD26369002BD5D005
:10F340001A6801209B88936103B0F0BD2C02002451
:10F3500030300024001000E0D34D621010B5037966
:10F3600084B084468E46012B0DD0022B08D18368D1
:10F37000DB0758BF01F07F0104B0BDE810408BE708
:10F38000002004B010BD81680DF10F0014467246D4
:10F3900001F001018DF80F40CDE900019CF811103A
:10F3A0009CF91000F4F71CFB04B010BD2DE9F041EE
:10F3B000816B10236B4F064604684FF064086A4A5D
:10F3C00090F83500B7FBF1F189B2FEF7EBFE438808
:10F3D000002105462046B7FBF3F73764FFF70CFF23
:10F3E00080226B212046FFF7B9FF05F0B5FD0646E8
:10F3F0000F4605F0B1FD831B61EB0701B3F57A7F82
:10F4000071F10003F5D3B8F10108EED14FF06408B3
:10F41000072268212046FFF7A1FF05F09DFD064663
:10F420000F4605F099FD831B61EB0701B3F57A7F69
:10F4300071F10003F5D3B8F10108EED142464FF067
:10F4400064086B212046FFF789FF05F085FD06461D
:10F450000F4605F081FD831B61EB0701B3F57A7F51
:10F4600071F10003F5D3B8F10108EED14FF00F08A8
:10F4700001226B212046FFF771FF05F06DFD064666
:10F480000F4605F069FD831B61EB0701B3F57A7F39
:10F4900071F10003F5D3B8F10108EED14FF00F0878
:10F4A00018221B212046FFF759FF05F055FD06469F
:10F4B0000F4605F051FD831B61EB0701B3F57A7F21
:10F4C00071F10003F5D3B8F10108EED14FF00F0848
:10F4D00018221C212046FFF741FF05F03DFD06469E
:10F4E0000F4605F039FD831B61EB0701B3F57A7F09
:10F4F00071F10003F5D3B8F10108EED14FF00F0818
:10F500002A791A212046FFF729FF05F025FD064636
:10F510000F4605F021FD831B61EB0701B3F57A7FF0
:10F5200071F10003F5D3B8F10108EED16A79192120
:10F5300020466426FFF712FF05F00EFD05460F4634
:10F5400005F00AFD431B61EB0702B3F57A7F72F108
:10F550000003F5D3013EEFD120460321BDE8F04181
:10F560004AE600BF40420F0098B40B081EE700BFF8
:10F570002DE9F0410468054682B0B6227E2120467E
:10F580004FF06408FFF7EAFE05F0E6FC06460F467A
:10F5900005F0E2FC831B61EB0701B3F57A7F71F1A3
:10F5A0000003F5D3B8F10108EED102212046FFF7A0
:10F5B00023FE63691BB19A88196812048A6105F0F9
:10F5C000CBFC06460F4605F0C7FC831B61EB070228
:10F5D000B3F57A7F72F10003F5D3636913B11A684A
:10F5E0009B8893614FF00A0805F0B6FC06460F466B
:10F5F00005F0B2FC831B61EB0701B3F57A7F71F173
:10F600000003F5D3B8F10108EED142467C21204633
:10F61000FFF7A4FE05F0A0FC06460F4605F09CFC93
:10F62000831B61EB0702B3F57A7F72F10003F5D318
:10F63000002259212046FFF791FE05F08DFC064679
:10F640000F4605F089FC831B61EB0702B3F57A7F57
:10F6500072F10003F5D394F910305E218D4A03EB6B
:10F6600043038DF8071052F83360A3689A0740F1FE
:10F67000E48001230DF1070200213046F4F72EFF4C
:10F680004FF4A473844A30460021F4F727FFA3689F
:10F690009B0740F1E6804FF00A0805F05DFC064646
:10F6A0000F4605F059FC831B61EB0701B3F57A7F28
:10F6B00071F10003F5D3B8F10108EED1012259210F
:10F6C0002046FFF74BFE05F047FC06460F4605F0C7
:10F6D00043FC831B61EB0702B3F57A7F72F10003F1
:10F6E000F5D38C2240212046FFF738FE05F034FC8C
:10F6F00006460F4605F030FC831B61EB0702B3F5AD
:10F700007A7F72F10003F5D3032241212046FFF7EF
:10F7100025FE05F021FC06460F4605F01DFC831B67
:10F7200061EB0702B3F57A7F72F10003F5D3AA6BA0
:10F7300009235A4E95F83500B6FBF2F291B2584AB9
:10F74000FEF730FD43884221B6FBF3F62E640279C2
:10F75000204642F0C002FFF701FE05F0FDFB054622
:10F760000E4605F0F9FB431B61EB0602B3F57A7F09
:10F7700072F10003F5D3082243212046FFF7EEFD86
:10F7800005F0EAFB05460E4605F0E6FB431B61EB80
:10F790000602B3F57A7F72F10003F5D304225821F3
:10F7A0002046FFF7DBFD05F0D7FB05460E4605F0CA
:10F7B000D3FB431B61EB0602B3F57A7F72F10003C2
:10F7C000F5D30A2253212046FFF7C8FD05F0C4FBFC
:10F7D00005460E4605F0C0FB431B61EB0602B3F580
:10F7E0007A7F72F10003F5D300227C212046FFF7D7
:10F7F000B5FD05F0B1FB05460E4605F0ADFB431B1C
:10F8000061EB0602B3F57A7F72F10003F5D30622AD
:10F810007D212046FFF7A2FD05F09EFB04460D4624
:10F8200005F09AFB031B61EB0502B3F57A7F72F1D9
:10F830000003F5D302B0BDE8F08163691BB11A681B
:10F840009B881B049361174B17491A68174BD2000A
:10F850004868A3FB023292094B681B1A9A42FBD2FA
:10F8600007E7104A4FF4FA70104B12680E4900FB7C
:10F8700002F24868A3FB023292094B681B1A9A42B3
:10F88000FBD26369002B3FF406AF1A689B88936133
:10F8900001E700BF2C020024F8B40B0840420F001F
:10F8A00040B60B0830300024001000E0D34D621049
:10F8B00010B5046884B02379012B0FD0022B0AD134
:10F8C000A368F0222046DB074CBFFF217F2104B054
:10F8D000BDE81040E0E4002004B010BDA268617CE7
:10F8E00094F9100002F001020DF10F040192FF22C1
:10F8F0000094F0248DF80F40F4F772F804B010BDB6
:10F9000030B50468CA4385B0237941EA0211012B5E
:10F91000CAB20ED0022B09D1A3682046DB074CBF28
:10F92000D221522105B0BDE83040B5E4002005B039
:10F9300030BD8DF80F200DF10F05A268617C94F9A0
:10F94000100002F00104D22200950194F4F748F867
:10F9500005B030BD10B5046884B02379012B0FD0F9
:10F96000022B0AD1A368B4222046DB074CBFFF213B
:10F970007F2104B0BDE810408EE4002004B010BD2B
:10F98000A268617C94F9100002F001020DF10F04ED
:10F990000192FF220094B4248DF80F40F4F720F870
:10F9A00004B010BD30B5046885B02379012B0FD0A9
:10F9B000022B0AD1A3680A462046DB074CBFA521CB
:10F9C000252105B0BDE8304066E4002005B030BD1B
:10F9D000A2680DF10F0594F910008DF80F10617CED
:10F9E00002F00104A52200950194F3F7F9FF05B098
:10F9F00030BD00BF10B5046884B02379012B0FD04F
:10FA0000022B0AD1A36896222046DB074CBFFF21B8
:10FA10007F2104B0BDE810403EE4002004B010BDDA
:10FA2000A268617C94F9100002F001020DF10F044C
:10FA30000192FF22009496248DF80F40F3F7D0FF37
:10FA400004B010BD30B5046885B02379012B0FD008
:10FA5000022B0AD1A3680A462046DB074CBF872148
:10FA6000072105B0BDE8304016E4002005B030BDE8
:10FA7000A2680DF10F0594F910008DF80F10617C4C
:10FA800002F00104872200950194F3F7A9FF05B065
:10FA900030BD00BF30B50468C90185B02379CAB252
:10FAA000012B0BD0022B06D17821204605B0BDE8F2
:10FAB0003040FFF7F1BB002005B030BD8DF80F20BE
:10FAC0000DF10F05A268617C94F9100002F00104A9
:10FAD000782200950194F3F783FF05B030BD00BF95
:10FAE00010B5046884B02379012B10D0022B0BD100
:10FAF000A36855222046DB074CBFA521252104B071
:10FB0000BDE81040FFF7C8BB002004B010BDA268DC
:10FB1000617C94F9100002F001020DF10F040192D2
:10FB2000A522009455248DF80F40F3F759FF04B037
:10FB300010BD00BF10B5046884B02379012B10D02C
:10FB4000022B0BD1A3682E222046DB074CBFF421E9
:10FB5000742104B0BDE81040FFF79EBB002004B044
:10FB600010BDA268617C94F9100002F001020DF151
:10FB70000F040192F42200942E248DF80F40F3F725
:10FB80002FFF04B010BD00BF154B30B59A8F85B064
:10FB90000468920123793432012BD2B20FD0022BA8
:10FBA0000AD1A3682046DB074CBFF421742105B0BD
:10FBB000BDE83040FFF770BB002005B030BD8DF8C8
:10FBC0000F200DF10F05A268617C94F9100002F07E
:10FBD0000104F42200950194F3F702FF05B030BD53
:10FBE0008062002410B5046884B02379012B0DD005
:10FBF000022B08D1A36831222046DB074CBFF42139
:10FC00007421FFF749FB012004B010BDA268617C9C
:10FC100094F910000DF10F0402F001020094312458
:10FC20000192F4228DF80F40F3F7DAFE012004B0C0
:10FC300010BD00BF10B5046884B02379012B0CD02F
:10FC4000022B07D101225821204604B0BDE8104004
:10FC5000FFF722BB002004B010BDA268617C02F057
:10FC6000010294F910000DF10F048DF80F3001928C
:10FC700058220094F3F7B4FE04B010BD10B5046828
:10FC800084B02379012B0CD0022B07D1012248210B
:10FC9000204604B0BDE81040FFF7FEBA002004B0D3
:10FCA00010BDA268617C02F0010294F910000DF110
:10FCB0000F048DF80F30019248220094F3F790FE64
:10FCC00004B010BD10B5046884B02379012B0CD0AA
:10FCD000022B07D11A460821204604B0BDE8104087
:10FCE000FFF7DABA002004B010BDA268617C94F975
:10FCF000100002F001020DF10F040192082200949D
:10FD000002248DF80F40F3F76BFE04B010BD00BF66
:10FD100010B5046884B02379012B0CD0022B07D1D5
:10FD200001220821204604B0BDE81040FFF7B4BA14
:10FD3000002004B010BDA268617C02F0010294F9B9
:10FD400010000DF10F048DF80F300192082200947D
:10FD5000F3F746FE04B010BD2DE9F04105461F46FD
:10FD60002A48164695F9103082B003EB430350F849
:10FD70003380AB689A0719D5FF230DF106028DF881
:10FD8000061040460DF107018DF807300123F4F706
:10FD9000A5FB3B46324600214046F4F79FFBAB688B
:10FDA0009B0718D5012002B0BDE8F0816B691BB13B
:10FDB0009A88186812048261154B1868154BC000A8
:10FDC000A3FB0030144B80095A685C68A4EB020C5A
:10FDD0006045FAD2D0E70E4A4FF4FA700D4B126824
:10FDE0000D4900FB02F24868A3FB023292094B68FE
:10FDF0001B1A9A42FBD26B69002BD3D01A680120E0
:10FE00009B88936102B0BDE8F08100BF2C02002402
:10FE100030300024D34D6210001000E030B5057979
:10FE200083B084468E46012D0DD0022D08D1846802
:10FE3000E40758BF41F0800103B0BDE830408BE7D4
:10FE4000002003B030BD806814460A46009400F0DC
:10FE500001049CF811109CF910000194F3F7C0FD07
:10FE600003B030BD2DE9F04105461F462A4816462D
:10FE700095F9103082B003EB430350F83380AB6840
:10FE80009A0719D5FF230DF106028DF8061040469A
:10FE90000DF107018DF807300123F4F71FFB3B46F6
:10FEA000002231464046F4F719FBAB689B0718D592
:10FEB000012002B0BDE8F0816B691BB19A88186817
:10FEC00012048261154B1868154BC000A3FB00306B
:10FED000144B80095A685C68A4EB020C6045FAD2A6
:10FEE000D0E70E4A4FF4FA700D4B12680D4900FB33
:10FEF00002F24868A3FB023292094B681B1A9A422D
:10FF0000FBD26B69002BD3D01A6801209B889361C8
:10FF100002B0BDE8F08100BF2C0200243030002484
:10FF2000D34D6210001000E030B5057983B08446EF
:10FF30008E46012D0DD0022D08D18468E40758BFEC
:10FF400041F0800103B0BDE830408BE7002003B0F2
:10FF500030BD806814460A46009400F001049CF805
:10FF600011109CF910000194F3F78AFF03B030BD23
:10FF70002DE9F043816B85B0804C1023056806465F
:10FF80007F4A4FF0960990F83500B4FBF1F189B241
:10FF9000FEF708F94388002107462846B4FBF3F42E
:10FFA0003464FFF729F980226B212846FFF7D6F940
:10FFB00004F0D2FF0446884604F0CEFF031B61EB39
:10FFC0000801B3F57A7F71F10003F5D3B9F10109A6
:10FFD000EED10322682128464FF09609FFF7BEF9BB
:10FFE00004F0BAFF0446884604F0B6FF031B61EB39
:10FFF0000801B3F57A7F71F10003F5D3B9F1010976
:020000040805ED
:10000000EED103226B212846FFF7A8F904F0A4FFE4
:100010000446884604F0A0FF031B61EB08010F2B88
:1000200071F10003F6D310226A212846FFF796F9F2
:1000300004F092FF0446884604F08EFF031B61EB38
:1000400008010F2B71F10003F6D300226C21284622
:10005000FFF784F904F080FF0446884604F07CFF33
:10006000031B61EB08010F2B71F10003F6D37A79C2
:1000700019212846FFF772F904F06EFF04468846FE
:1000800004F06AFF031B61EB08010F2B71F1000301
:10009000F6D318221B212846FFF760F904F05CFF15
:1000A0000446884604F058FF031B61EB08010F2B40
:1000B00071F10003F6D318221C212846FFF74EF9F0
:1000C00004F04AFF0446884604F046FF031B61EB38
:1000D00008010F2B71F10003F6D33A791A21284653
:1000E000FFF73CF904F038FF07460C4604F034FFF4
:1000F0008C4208BF8742F9D003212846FFF77CF8DD
:10010000062302AA43213068FFF70EFF28B3BDF88B
:100110000810BDF80A30BDF80C20C9BADBBA07EEEA
:10012000901AD2BAF8EEE76A07EE102A07EE903A74
:10013000B8EEC77AF8EEE77AC6ED076A86ED097A77
:10014000C6ED087AFDEEE77ACDED017A9DF904302F
:10015000013305D005B0BDE8F083D6ED087AF1E7AC
:10016000D6ED077AFDEEE77ACDED017A9DF9043000
:100170000133EFD1062005F0D3FB00BF40420F0052
:1001800098B40B0870B5066882B00546F469002C77
:100190003FD03379221D012B06D0022B2DD0002316
:1001A0001846A37002B070BDB368717C03F0010300
:1001B00096F91000009201930C231A46F3F760FEA3
:1001C000A0700028EED0B4F9043007EE903AF8EEB3
:1001D000E77AC5ED077AB4F9063007EE903AF8EE03
:1001E000E77AC5ED087AB4F9083007EE903AF8EEF0
:1001F000E77AC5ED097A02B070BDB368304613F0F6
:10020000010F4FF00C030CBF8C211946FFF72AFE9B
:10021000D6E709211420FDF7EFFEF06104462E68B1
:10022000B7E700BF70B5066882B00546F469002CD8
:100230003FD03379E21C012B06D0022B2DD00023B6
:100240001846A37002B070BDB368717C03F001035F
:1002500096F9100000920C2201930D23F3F710FE83
:10026000A0700028EED0B4F90A3007EE903AF8EE0C
:10027000E77AC5ED077AB4F90C3007EE903AF8EE5C
:10028000E77AC5ED087AB4F90E3007EE903AF8EE49
:10029000E77AC5ED097A02B070BDB368304613F055
:1002A000010F4FF00D0314BF0C218C21FFF7DAFD75
:1002B000D6E709211420FDF79FFEF06104462E6861
:1002C000B7E700BF006810B5037984B00C46012B76
:1002D00019D0022B14D1836803AA13F0010F4FF039
:1002E000030314BF2221A221FFF7BCFD30B1BDF9E9
:1002F0000D3003EB83031B12E633238004B010BDE3
:10030000002004B010BD836803AA417C03F0010300
:1003100090F910000092222201930323F3F7B0FD1D
:100320000028E4D1EAE700BF70B5066882B0054650
:10033000F469002C3FD03379221D012B06D0022B0B
:100340002DD000231846A37002B070BDB368717C35
:1003500003F0010396F9100000923B2201930E2353
:10036000F3F78EFDA0700028EED0A389DBBA07EE6C
:10037000903AF8EEE77AC5ED077AE389DBBA07EE43
:10038000903AF8EEE77AC5ED087A238ADBBA07EEF1
:10039000903AF8EEE77AC5ED097A02B070BDB3681D
:1003A000304613F0010F4FF00E0314BF3B21BB2169
:1003B000FFF758FDD6E709211420FDF71DFE04467E
:1003C000F061B8E7006810B5037984B0012B10D054
:1003D000022B0BD103AAF621FFF744FD20B1BDF893
:1003E0000C300B4A5BBA938304B010BD002004B0FC
:1003F00010BD826803AC417C022302F0010290F937
:100400001000CDE90042F622F3F73AFDE6E700BF1F
:1004100080620024006810B5037984B0012B1DD0E0
:10042000022B18D1032303AAF621FFF71BFD80B18D
:100430009DF80D309DF80CC01B020F499DF80E2051
:1004400043EA0C431343B1F93C20C2F10802D34004
:100450000B6404B010BD002004B010BD826803AC72
:10046000417C032302F0010290F91000CDE9004223
:10047000F622F3F705FDDAE780620024006810B584
:10048000037984B0012B30D0022B24D1062302AA99
:10049000F721FFF7E7FCF0B19DF809209DF808C0AF
:1004A00012019DF80A109DF80C3042EA0C329DF8BA
:1004B0000BE01B0142EA1112134943EA0E334A666C
:1004C000C1F87C2C9DF80D2043EA12134B64C1F84F
:1004D000803C04B010BD0C4B0020D3F87C1CD3F83A
:1004E000802C59665A6404B010BD826802AC417C0D
:1004F000062302F0010290F91000CDE90042F72234
:10050000F3F7BEFCC7E700BF80620024006810B5A7
:10051000037984B0012B1CD0022B0AD1836803AA73
:1005200013F0010F4FF0030314BF00218021FFF7E8
:1005300099FC9DF80D3001209DF80CC01B029DF820
:100540000E100B4A43EA0C430B43C2F8883004B048
:1005500010BD826803AC417C032302F0010290F9D4
:100560001000CDE900420022F3F78AFCE1E700BF6A
:1005700080620024006810B5037984B0012B1CD080
:10058000022B0AD1836803AA13F0010F4FF0030373
:1005900014BF00218021FFF765FC9DF80D3001207C
:1005A0009DF80CC01B029DF80E100B4A43EA0C4349
:1005B0000B43C2F89C3004B010BD826803AC417C90
:1005C000032302F0010290F91000CDE9004200225D
:1005D000F3F756FCE1E700BF80620024006810B525
:1005E000037984B0012B28D0022B23D1836803AA7E
:1005F00013F0010F4FF003030CBF83211946FFF7DF
:1006000031FCA8B19DF80C309DF90C109DF80D201F
:100610001B0400299DF80EC043EA02230E4AB4BF12
:100620004FF07F41002143EA0C030B43C2F8D03066
:1006300004B010BD002004B010BD8268032303ACD9
:10064000417C02F0010290F91000CDE900421A4607
:10065000F3F716FCD5E700BF80620024006810B5F0
:10066000037984B0012B28D0022B23D1836803AAFD
:1006700013F0010F4FF0030314BF00218021FFF797
:10068000F1FBA8B19DF80C309DF90C109DF80D20E0
:100690001B0400299DF80EC043EA02230E4AB4BF92
:1006A0004FF07F41002143EA0C030B43C2F8B43002
:1006B00004B010BD002004B010BD826803AC417CC2
:1006C000032302F0010290F91000CDE9004200225C
:1006D000F3F7D6FBD5E700BF8062002490F9103015
:1006E000F0B503EB4303274E154683B056F833604D
:1006F000044683689A0718D5FF230DF106028DF88A
:10070000061030460DF107018DF807300123F3F78D
:10071000E5FE0123002229463046F3F7DFFEA368F9
:100720009B0716D5012003B0F0BD43691BB19A8821
:10073000186812048261144B144A1868144BC000E4
:100740005768A3FB003080095368DB1B9842FBD23B
:10075000D2E70D4A4FF4FA700D4B12680B4900FBBB
:1007600002F24868A3FB023292094B681B1A9A42B4
:10077000FBD26369002BD5D01A6801209B88936156
:1007800003B0F0BD2C02002430300024001000E043
:10079000D34D621010B5037982B08E46012B0DD077
:1007A000022B08D18368DB0758BF41F0800102B0FB
:1007B000BDE8104092E7002002B010BD81681446E9
:1007C0007246009401F00104417C90F910000194FC
:1007D000F3F756FB02B010BDF0B5044600210068E7
:1007E00083B0FEF709FD15227E2120686427FEF7FD
:1007F000B5FD04F0B1FB05460E4604F0ADFB431B0E
:1008000061EB0602B3F57A7F72F10003F5D3013F85
:10081000EFD111227E2120680527FEF79FFD04F00D
:100820009BFB05460E4604F097FB431B61EB06025B
:10083000B3F57A7F72F10003F5D3013FEFD10DF1EB
:10084000070203212068FFF7A5FF9DF8073003F09A
:100850003C03142B40F09B800C2240212068FEF7C3
:100860007DFD04F079FB05460E4604F075FB431B45
:1008700061EB0602B3F57A7F72F10003F5D3454DC3
:100880000923A16B444A94F83500B5FBF1F189B214
:10089000FDF788FC0346422120685A88B5FBF2F533
:1008A00025641A79FEF75AFD04F056FB05460E46FC
:1008B00004F052FB431B61EB0602B3F57A7F72F141
:1008C0000003F5D3082241212068FEF747FD04F01C
:1008D00043FB05460E4604F03FFB431B61EB06025B
:1008E000B3F57A7F72F10003F5D30022432120682B
:1008F000FEF734FD04F030FB05460E4604F02CFBF9
:10090000431B61EB0602B3F57A7F72F10003F5D366
:10091000102251212068FEF721FD04F01DFB054641
:100920000E4604F019FB431B61EB0602B3F57A7F18
:1009300072F10003F5D30A2253212068FEF70EFD61
:1009400004F00AFB05460E4604F006FB431B61EB70
:100950000602B3F57A7F72F10003F5D380225621A7
:100960002068FEF7FBFC04F0F7FA05460E4604F09B
:10097000F3FA431B61EB0602B3F57A7F72F10003D1
:10098000F5D303212068FEF737FC03B0F0BD062045
:1009900004F0C6FF40420F00E8BC0B0870B50568C4
:1009A00084B004460E462B79012B14D0022B0FD1B4
:1009B000AB68E122DB071ED528461146FEF76CFC2A
:1009C00030B13246FF21206804B0BDE87040E1E656
:1009D000002004B070BDAA68697C02F0010295F99C
:1009E00010000DF10F050192E12200958DF80F2006
:1009F000F2F7F6FFE4E761212846FEF74DFCDFE75A
:100A000070B5056884B004460E462B79012B15D0CD
:100A1000022B10D1AB68C3222846DB074CBFE12173
:100A20006121FEF739FC30B13246FF21206804B065
:100A3000BDE87040AEE6002004B070BDAA6895F92C
:100A4000100002F00102697C01920DF10F02009288
:100A5000C3228DF80F20E122F2F7C2FFE3E700BFC7
:100A600070B5056884B004460E462B79012B19D069
:100A7000022B14D1AB68F0222846DB074CBFE121E2
:100A80006121FEF709FC50B12246FF2152F8040B08
:100A9000FFF780FE18B12379337004B070BD0020D9
:100AA00004B070BDAA6895F9100002F00102697CDB
:100AB00001920DF10F020092F0228DF80F20E12239
:100AC000F2F78EFFDFE700BFF0B583B015461C4696
:100AD00006460DF107020F46FFF75CFE9DF8072062
:100AE00005EA0203A34201D103B0F0BD22EA0502E8
:100AF00039463046224303B0BDE8F040FEF72EBC35
:100B0000F0B5044683B00D461746061D20680379EC
:100B1000012B17D0022B12D183683246FF21DB074D
:100B20005CBF3246FF21FFF7D9FD30B115B1237903
:100B3000DB07EBD40FB123793B7003B0F0BD00208D
:100B400003B0F0BD8268417C02F0010C90F9100006
:100B5000FF22CDE9006CF3F793F9E6E770B50446A0
:100B600082B0051D20680379012B13D0022B0ED112
:100B700083682A46FF21DE075CBF2A46FF21FFF774
:100B8000ADFD10B12379DB07ECD402B070BD0020BD
:100B900002B070BD8668FF22417C06F0010690F924
:100BA0001000CDE90056F3F76BF9EAE7024630B5DD
:100BB000044652F8040B83B00379012B0ED0022BAC
:100BC00009D1FF21FFF78AFD18B12079C04300F059
:100BD000010003B030BD002003B030BD8568417C0A
:100BE00005F0010590F910000092FF220195F3F73E
:100BF00047F9E9E770B5B42282B00446FF210068E6
:100C0000FEF7ACFB10B9002002B070BD2068251DB6
:100C10000379012B13D0022BF5D183682A46FF21DB
:100C2000DE075CBF2A46FF21FFF758FD0028EAD007
:100C30002379DB07E8D520680379012BEBD186689F
:100C4000FF22417C06F0010690F91000CDE9005624
:100C5000F3F716F9EAE700BF70B50A4682B004461A
:100C6000A5210068FEF77AFB10B9002002B070BD24
:100C70002068251D0379012B13D0022BF5D1836841
:100C80002A46FF21DE075CBF2A46FF21FFF726FD2B
:100C90000028EAD02379DB07E8D520680379012B07
:100CA000EBD18668FF22417C06F0010690F9100026
:100CB000CDE90056F3F7E4F8EAE700BF70B582B07B
:100CC0000446CDE90023FFF795FF10B9002002B0DC
:100CD00070BD5522A5212068FEF740FB0028F5D005
:100CE000251D2A46FF212068FFF754FD0028EDD07E
:100CF0002379DB07F5D40DF1FF350DF1070615F863
:100D0000011F2046FFF7A8FF0028DFD0B542F6D12B
:100D1000DDE700BF002A36D0013AF0B5044683B0C3
:100D20004E1E051D51FA82F716F8012FA5212068E5
:100D3000FEF714FB90B9002003B0F0BD8268417C3F
:100D400002F0010C90F91000FF22CDE9005CF3F7EE
:100D500097F80028EFD02379DB070FD520680379B7
:100D6000012BEBD0022BE6D183682A46FF21DB075B
:100D70005CBF2A46FF21FFF7B1FCEAE7B742D3D1B7
:100D8000012003B0F0BD0120704700BFF0B59622EE
:100D900083B00E460446FF210068FEF7DFFA10B963
:100DA000002003B0F0BD251D20680379012B1DD064
:100DB000022BF5D183682A46FF21DF075CBF2A4654
:100DC000FF21FFF78BFC0028EAD02379DB07EBD467
:100DD000E12220681146FEF7C1FA0028E0D0324631
:100DE000FF21206803B0BDE8F040D3E48768FF220C
:100DF000417C07F0010790F91000CDE90057F3F7A7
:100E00003FF8E0E7002A45D0013AF0B54F1C83B027
:100E100004460E46051D57FA82F79622FF212068E8
:100E2000FEF79CFA90B9002003B0F0BD8268417CC7
:100E300002F0010C90F91000FF22CDE9005CF3F7FD
:100E40001FF80028EFD02379DB070FD5206803793E
:100E5000012BEBD0022BE6D183682A46FF21DB076A
:100E60005CBF2A46FF21FFF739FCEAE7E122206850
:100E70001146FEF773FA0028D5D03246FF212068CC
:100E8000FFF788FC0028CED00136BE42C5D1012034
:100E900003B0F0BD01207047F0B50B46054616467D
:100EA000044683B087211A4655F8040BFEF756FA1C
:100EB00020680379012B17D0022B12D183682A46B0
:100EC000FF21DF075CBF2A46FF21FFF707FC30B197
:100ED0002379DA07ECD416B1C3F34013337003B0AF
:100EE000F0BD002003B0F0BD8768FF22417C07F011
:100EF000010790F91000CDE90057F2F7C1FFE6E7CE
:100F0000F0B5782183B01646044600220068FEF74B
:100F100025FA10B9002003B0F0BD251D2068037923
:100F2000012B13D0022BF5D183682A46FF21DF075E
:100F30005CBF2A46FF21FFF7D1FB0028EAD02379C6
:100F4000DA07EBD45B09337003B0F0BD8768FF228A
:100F5000417C07F0010790F91000CDE90057F2F746
:100F60008FFFEAE770B5CC2282B00446A521006865
:100F7000FEF7F4F910B9002002B070BD2068251DFD
:100F80000379012B13D0022BF5D183682A46FF2168
:100F9000DE075CBF2A46FF21FFF7A0FB0028EAD04E
:100FA0002379DB07E8D520680379012BEBD186682C
:100FB000FF22417C06F0010690F91000CDE90056B1
:100FC000F2F75EFFEAE700BF70B5B42282B00446D4
:100FD000FF210068FEF7C2F910B9002002B070BD11
:100FE000251D20680379012B21D0022BF5D18368C0
:100FF0002A46FF21DE075CBF2A46FF21FFF76EFB72
:101000000028EAD02379DA07EBD4CC212046FFF779
:1010100023FE0028E1D002E02379DB07DED52A4653
:10102000FF212068FFF7B6FB0028F5D1D5E78668D9
:10103000FF22417C06F0010690F91000CDE9005630
:10104000F2F71EFFDCE700BF2DE9F04F82468BB0C0
:1010500000200AF1040B069104905C460590CDE94E
:101060000823049B5046089ADD0002EBC303039358
:10107000FFF7C0FD28B90CE09AF8043013F0010B1B
:101080000DD02246FF21DAF80000FFF783FB00288D
:10109000F2D1099B049A1A700BB0BDE8F08F9B0740
:1010A000F7D5F0215046FFF7D7FD0028F1D0083DD5
:1010B000089B0126D9462B44B0460793069B003B6C
:1010C00018BF01230293029FB8F1080F8CBF0027BD
:1010D00007F00107002F5AD008F1FF35069B43FAAD
:1010E00005F505F00105EA017821DAF80000FEF7C0
:1010F00035F90028CDD0DAF800000379012B3AD079
:10110000022B36D183682246FF21DB075CBF2246D3
:10111000FF21FFF7E3FA0028BBD09AF8043013F060
:101120000102E8D199094FEA531E4FEAD31C01EAA4
:101130005313DB074DD485EA0C052F4078D1BCF161
:10114000000F31D0039911F80930334301F8093009
:10115000760008F1010816F0FF065FFA88F8B2D1B0
:1011600009F101095FFA89F9B9F1080F31D00126B7
:10117000A9E700208DE78268417C02F0010C90F91C
:101180001000FF22CDE9004CF2F77AFEC3E7049B82
:10119000C3B1059B434515D9079B13F809301E427F
:1011A00014BF012500259EE74EEA010111F0010F51
:1011B000039911F8093008BFC34623EA060301F872
:1011C0000930C5E7059BA3EB0805B5FA85F56D0960
:1011D00089E7B8F1400F06D8099B049A1B7893421F
:1011E0003FF63FAF55E7039BDF795E1E03F1060C28
:1011F00016F8011F082382EA01055208013B49083D
:1012000015F0010F82F08C0518BFEAB213F0FF034E
:10121000F1D1B445ECD19742DED1049B0133DBB26E
:101220000493BBF1000F3FF434AFCDF814B0D3E713
:1012300038462EE730B5056885B004462B79012B7A
:1012400000F09380022B08D1AB6802AA2846DB0786
:101250004CBF08218821FFF741FA9DF8083013F0B0
:10126000100302D1184605B030BD062302AA0021A2
:101270002068FEF759FE0028F5D09DF80920B6EE4B
:10128000002A9DF8081012029DF80A30DFED3D6A31
:1012900002EB01429DF80C10134414024FEA0121A5
:1012A0009DF80B4048BF03F17F439DF80D2001EBF3
:1012B000044107EE903A344B0A440902B8EEE77A4B
:1012C00048BF02F17F42C7EE265A07EE902AB3F9D3
:1012D0007C2002EE902AB3F9782005EE102AF8EE71
:1012E000E22AF8EEE77AB3F97420B8EEC55A04EEB4
:1012F000902AB3F97A2087EEA64AD3ED1C7A03EE42
:10130000102AB3F9762006EE902AB3F96A20B8EED7
:10131000E76AD3ED1B7AF8EEE44A07EE102AA5EE51
:10132000A25AB3F96820F8EEE77AB8EEC33A03EEB2
:10133000902AF8EEE66AB8EEC77AF8EEE33AA5EE40
:10134000856AE5EE836A27EE047A25EE843AE5EEB7
:10135000867AA3EE827AE4EE247A83ED217AE3EEB4
:10136000267AC3ED207A05B030BDAA68697C02F008
:10137000010295F91000019202AA00920822F2F7E8
:101380007FFD6AE7000078488062002410B50446BB
:10139000006882B003796A46022B4FF006030CBF47
:1013A00043210321FEF7C0FD68B1BDF80010BDF870
:1013B0000220BDF8043049BA52BA5BBAE1866287AE
:1013C000238702B010BDE086A06302B010BD00BF4D
:1013D00030B5002385B004460221C3860DF1070213
:1013E00083630068FFF7D6F918B19DF80730DB0773
:1013F00003D40025284605B030BD0623032102AAE8
:101400002068FEF791FD0DF1070209212068FFF722
:10141000C1F905460028ECD09DF8073013F00C0FF9
:10142000E7D1BDF80820BDF80C30BDF80A10C2EBBA
:101430008232C3EB8333206889009B0092002187AE
:1014400063870A21E2860122FDF788FF284605B05E
:1014500030BD00BF10B50446002221210068FDF711
:101460007DFFFC2220212068FDF778FF4022242107
:101470002068FDF773FF0C2223212068FDF76EFF23
:10148000002222212068FDF769FF012010BD00BF66
:1014900010B5044694220B210068FDF75FFF71220E
:1014A00001212068FDF75AFF002204212068FDF782
:1014B00055FFC82205212068FDF750FF00220621B4
:1014C0002068FDF74BFFC82207212068FDF746FF83
:1014D000002208212068FDF741FFC8220921206869
:1014E000FDF73CFF012010BD01207047044B002296
:1014F000002101201A605A609A60D960704700BFCD
:10150000C0D80024104B11491A680346C868121A43
:10151000FA2A16D8D1ED006A012091ED017AFDEE8C
:10152000E66AD1ED027ABDEEC77AFDEEE77A16EEF5
:10153000902ADA8617EE102A1A8717EE902A5A8711
:1015400070470020704700BF4C3E0024C0D80024E4
:10155000014B1B695B681847C0D80024024B083058
:101560001B699B68184700BFC0D800240120704742
:10157000012070470120704701207047012070470B
:1015800031B10B4BD3ED057AF8EEE77AC1ED007A75
:101590006AB10749074B8969DFED076A0B4407EE1B
:1015A000903AF8EEE77A87EEA67A82ED007A7047F5
:1015B000C0D800244D95FFFF0000C84201207047AD
:1015C00001207047704700BF034B03EB8000C369E5
:1015D0000BB19B6819607047C0D80024044B03EB23
